:1000000055C7000084C7000082C7000080C70000F9
:100010007EC700007CC700007AC7000078C70000D8
:1000200076C7000074C7000072C7000070C70000E8
:100030006EC700000C9452726AC7000068C70000C7
:1000400066C7000064C7000062C7000060C7000008
:100050005EC700005CC700005AC700000C945E81B8
:1000600056C700000C9439850C946F8550C700006A
:100070004EC700004CC700004AC7000048C7000038
:1000800046C7000044C7000042C7000040C7000048
:100090003EC700003CC700003AC700000C946D5DED
:1000A00036C7000034C7000032C7000030C7000068
:1000B0002EC700002CC700002AC7000028C7000078
:1000C00026C7000024C7000022C700000C94E48566
:1000D0000C941A861CC700000C948F860C94C5865D
:1000E00016C700007D455D458F458F458F458F457F
:1000F0008F458F458F458F458F458F456E44804492
:1001000087448E4495449C44A144AA44B144C844C5
:10011000CB448F45CF44D244D444D744F144F34434
:10012000FA44014514451B452245AB82AE829D82AF
:10013000A182A782E582B282B682BC82C082C482DA
:10014000CA82CE82D282E582D882DC82E082084AEC
:10015000D73B3BCE016E84BCBFFDC12F3D6C7431DB
:100160009ABD56833DDA3D00C77F11BED9E4BB4C32
:100170003E916BAAAABE000000803F07634236B7DB
:100180009BD8A71A39685618AEBAAB558C1D3CB728
:10019000CC5763BD6DEDFD753EF6177231BF0000A3
:1001A00000803F08000000BE922449123EABAAAA7C
:1001B0002ABECDCCCC4C3E00000080BEABAAAAAA81
:1001C0003E00000000BF000000803F000000000073
:1001D000084178D3BB4387D1133D190E3CC3BD42C0
:1001E00082AD2B3E68EC8276BED98FE1A93E4C8071
:1001F000EFFFBE01C4FF7F3F0000000000003E4D46
:100200006F74696F6E20627920756C747261736FA0
:100210006E632073656E736F723A0A00696E707553
:10022000742044535463616C6962726174653A006E
:100230004E6F20445320546865726D6F6D65746510
:1002400072210050726573732061206B6579004CD8
:100250004344206F6E00234E6F2073656E736F7280
:1002600020666F7220504D21004E6F2073656E73B3
:100270006F722100504D313A322E353A3130004DF7
:100280006561737572696E672E2E004F3220436F61
:100290006E6300434F3220436F6E630070482076D8
:1002A000616C756500547572626964697479004E99
:1002B0006F2073656E736F72210049522054656D13
:1002C0007065726174757265004D656173757269F0
:1002D0006E672E2E004C6967687420496E74656ED7
:1002E0007369747900416E676C65732F006765747C
:1002F00053656C665465737442697428293A20000A
:100300006973496E74657272757074456E61626C62
:1003100065642831293A2000676574496E746572F6
:10032000727570744D617070696E672831293A205A
:1003300000676574496E74657272757074536F7579
:100340007263652831293A2000676574496E7465C7
:100350007272757074536F7572636528293A200044
:100360006765745261746528293A20332E3134311F
:1003700035393F00616363656C2E69734C6F77504C
:100380006F77657228293A2000616363656C2E6976
:100390007341736C65657028293A20006163636559
:1003A0006C2E6973546170536F757263654F6E5A2A
:1003B00028293A2000616363656C2E69735461706B
:1003C000536F757263654F6E5928293A2000616337
:1003D00063656C2E6973546170536F757263654FFA
:1003E0006E5828293A2000616363656C2E69734159
:1003F00063746976697479536F757263654F6E5A69
:1004000028293A2000616363656C2E697341637427
:100410006976697479536F757263654F6E592829CF
:100420003A200069734163746976697479536F7512
:100430007263654F6E5828293A20006973546170C1
:10044000446574656374696F6E4F6E5A28293B204A
:1004500066616C73653F2000697354617044657414
:10046000656374696F6E4F6E5A28293B20747275EC
:10047000653F2000697354617044657465637469F5
:100480006F6E4F6E5928293B2066616C73653F2063
:10049000006973546170446574656374696F6E4F6D
:1004A0006E5928293B20747275653F20006973548A
:1004B0006170446574656374696F6E4F6E58282966
:1004C0003B2066616C73653F200069735461704422
:1004D0006574656374696F6E4F6E5828293B20748C
:1004E0007275653F2000676574537570707265732F
:1004F0007342697428293B2066616C73653F200054
:1005000067657453757070726573734269742829D6
:100510003B20747275653F2000697341637469768E
:10052000697479416328293A20006973496E6163CF
:100530007469766974795A456E61626C65642829BC
:100540003A20006973496E616374697669747959F8
:10055000456E61626C656428293A20006973496EB2
:10056000616374697669747958456E61626C65641B
:1005700028293A2000697341637469766974795A4D
:10058000456E61626C656428293A20006973416395
:1005900074697669747959456E61626C656428295D
:1005A0003A20006973416374697669747958456EBD
:1005B00061626C656428293A20006765744672653B
:1005C0006546616C6C4475726174696F6E28293A76
:1005D00020006765744672656546616C6C5468728C
:1005E0006573686F6C6428293A20006765745469E4
:1005F0006D65496E616374697669747928293A205A
:1006000000676574496E61637469766974795468CA
:10061000726573686F6C6428292000676574416394
:100620007469766974795468726573686F6C64284C
:10063000292000676574446F75626C65546170575A
:10064000696E646F7728292000676574446F75624E
:100650006C655461704C6174656E637928293A2029
:10066000006765745461704475726174696F6E28B7
:10067000293A2000676574417869734F666673652F
:10068000742826782C2026792C20267A293A2000D6
:100690006765745461705468726573686F6C642820
:1006A000293A200058595A2047733A200058595A7D
:1006B00020434F554E54533A2000736574206761B0
:1006C000696E735B5D3A006761696E735F6F726933
:1006D000675B5D3A00466C616D65204952004F666C
:1006E00066206169722D636F6E64210049742773FF
:1006F00020746F6F20636F6F6C210054656D7020E4
:1007000069732066696E6521004973206169722DE5
:10071000636F6E64206F6E3F00497427732071759C
:1007200069746520686F74210049742773207665A9
:10073000727920686F74210054656D702048756D62
:10074000696469747900234E6F2073656E736F72EC
:1007500020666F722074656D7020262068756D6943
:100760006469747921004E6F2053656E736F722136
:100770000054656D702048756D6964697479004F27
:100780006666206169722D636F6E6421004974276B
:100790007320746F6F20636F6F6C210054656D70F0
:1007A0002069732066696E65210049732061697252
:1007B0002D636F6E64206F6E3F0049742773207144
:1007C0007569746520686F742100497427732076F9
:1007D00065727920686F74212000616E6F7468659E
:1007E0007220495220696E7075743D006B657932D4
:1007F0003D006B6579323D00496E76616C6964201D
:100800006B657921007265706C6965733D00233AF0
:1008100053686F772F48696465204C4344002A3A37
:10082000546869732048656C700044433A436C65B2
:100830006172204C43440044423A5265736574200F
:100840004C6F676765720044373A4D6F74696F6E1D
:100850000044363A44532054656D700044353A558F
:100860005620496E74656E736974790044343A4F4A
:100870003220636F6E632E0044333A434F3220635D
:100880006F6E632E0044323A504D28313A322E3585
:100890003A3130290044323A504D28313A322E351F
:1008A0003A3130292A0044313A54757262696469D8
:1008B00074790044303A566F6C7461676500393A58
:1008C0006F7220334420616363656C2E00393A49AE
:1008D0006E636C2E20616E672E00383A7048207669
:1008E000616C756500373A49522054656D70003768
:1008F0003A49522054656D702A00363A4D61676E50
:1009000065746963206669656C6400353A47617394
:10091000204C6576656C00343A495220466C616D16
:100920006500333A4C6967687420496E742E003252
:100930003A616E642048656967687400323A5465AC
:100940006D7020507265737375726500313A54652D
:100950006D702048756D696469747900303A536F21
:10096000756E64204C6576656C00303A536F756E19
:1009700064204C6576656C2A0020202020202020F1
:100980002020202020202020002020202020202087
:100990002020202020202020002020202020202077
:1009A0002020202020202020200020202020202067
:1009B0002020202020202020202000202020202057
:1009C0002020202020202020202020002020202047
:1009D000202020202020202020202020004C6F6775
:1009E00067657220446972656374696F6E002D2DAE
:1009F0002D2D2D2D2D2D2D2D2D2D2D2D2D2D2D2D27
:100A00002D2D2D2D2D2D2D2D2D2D2D2D2D2D2D2D16
:100A10002D2D005265736F6C7574696F6E3A2020CE
:100A200020004D696E2056616C75653A20202020AB
:100A3000004D61782056616C75653A2020202000B9
:100A4000556E697175652049443A20202020004484
:100A50007269766572205665723A202020005365CF
:100A60006E736F723A20202020202020002D2D2D23
:100A70002D204D61676E657469632053656E736FD9
:100A800072202D2D2D2D2D2D2D2D2D2D2D2D2D2D5E
:100A90002D2D2D2D2D2D006E6F20484D43353838CE
:100AA00033206D61676E657469632073656E736F63
:100AB00072202E2E2E20436865636B207769726941
:100AC0006E67210020766F6C746167653D00547518
:100AD00072626964697479205570706572204C691E
:100AE0006D69743A200020766F6C746167653D0013
:100AF000547572626964697479204C6F77657220ED
:100B00004C696D69743A2000547572626964697445
:100B100079204C6F776572204C696D697420566935
:100B20006E663A2000434F32204D415820766F6C5C
:100B300074202800434F32207A65726F20766F6CE4
:100B4000742028004F322063616C6962726174699D
:100B50006F6E3A2000547572626964697479204C32
:100B60006F776572204C696D69742056313A2000A8
:100B700023506172616D6574657273002343616C0B
:100B80006962726174696F6E2050726573737572F9
:100B9000653D0023536561206C6576656C205028A7
:100BA00063616C63293D00234572726F723A707203
:100BB00065737375726520424D503038352C206353
:100BC0006865636B20776972696E672100495220FE
:100BD00054656D702073656E736F7220666F756EED
:100BE0006400504D322E352073656E736F72206C29
:100BF000696B656C7920666F756E6400536F756EF6
:100C000064204C6576656C2073656E736F72206628
:100C10006F756E640053656E736F7220736C6F74C2
:100C200020616E6420747970653A00005EBCE261F8
:100C30003FDD83C29C7E20A3FD1F41009D23BE4655
:100C4000DB65F88C11AF32CA57E97400000A0B0259
:100C5000090C0D0E0807030401000000000000004D
:100C60000000000000000000000000000000000084
:100C70000000000000000012111000000000000041
:100C80000000000000000000000000000000000064
:100C9000000102102020080810204010204080028F
:100CA00001020108040201010204081020408080B2
:100CB0004020100804020180040201804020100836
:100CC000040201080402010102040810204080010E
:100CD00002040810204080050505050705080808DE
:100CE00008020202020A0A080804040404010101BD
:100CF00001010101010303030303030303040707C5
:100D0000070C0C0C0C0C0C0C0C0202020206060662
:100D100006060606060B0B0B0B0B0B0B0B0000203D
:100D2000002300260029002C002F003200000100C3
:100D30000003010601090100002200250028002B04
:100D4000002E003100340002010000050108010BF3
:100D50000100002100240027002A002D003000336C
:100D60000001010000040107010A014E414E494EF5
:100D7000495459494E46CDCCCC3D0AD7233C17B7F0
:100D8000D13877CC2B329595E6241FB14F0A00005D
:100D900020410000C84200401C4620BCBE4CCA1B7B
:100DA0000E5AAEC59D7400407A10F35A00A0724EE0
:100DB00018090010A5D4E80000E87648170000E400
:100DC0000B54020000CA9A3B000000E1F505000048
:100DD00080969800000040420F000000A0860100AD
:100DE0000000102700000000E8030000000064007D
:100DF000000000000A0000000000010000000000E8
:100E00002C76D888DC674F0823DFC1DFAE59E1B10B
:100E1000B796E5E3E453C63AE651997696E8E6C21A
:100E20008426EB898C9B62ED407C6FFCEFBC9C9F21
:100E300040F2BAA56FA5F490055A2AF75C936B6C43
:100E4000F9676DC11BFCE0E40D47FEF520E6B50037
:100E5000D0ED902E0300943577050080841E0800A5
:100E600000204E0A000000C80C333333330F986E55
:100E700012831141EF8D2114893BE65516CFFEE612
:100E8000DB18D1844B381BF77C1D901DA4BBE424D8
:100E9000203284725E228100C9F124ECA1E53D2755
:100EA0002137845CA1854C86F786F53711241FBE57
:100EB000CFEFD1E2DEBFCDBF00E00CBF1AE0A0E073
:100EC000B2E0E4EBF6E301E00BBF02C007900D9245
:100ED000AA37B107D9F720E1AAE7BAE001C01D920D
:100EE000AB37B207E1F71EE0CAEADEE000E006C079
:100EF00022970109FE010BBF0E94CC93C03AD10793
:100F000080E00807A9F70E94FA8E0C94499B78C8E4
:100F1000CF92DF92EF92FF920F931F93E82FF92F5A
:100F200005C0015011092109310961F19081962311
:100F30009417B9F305C0015011092109310911F1C4
:100F4000908196239413F7CFC12CD12CE12CF12C56
:100F50000AC08FEFC81AD80AE80AF80A0C151D054E
:100F60002E053F0579F080818623841791F36C2D3F
:100F70007D2D8E2D9F2D1F910F91FF90EF90DF9073
:100F8000CF90089560E070E080E090E01F910F91B5
:100F9000FF90EF90DF90CF90089520EF39E0FC01B3
:100FA000318320830895089520EF39E0FC013183D7
:100FB00020830C94088F2F923F924F925F926F92F2
:100FC0007F928F929F92AF92BF92CF92DF92EF92D9
:100FD000FF920F931F93CF93DF93CDB7DEB72E977A
:100FE0000FB6F894DEBF0FBECDBF8C017E876D8734
:100FF000DC014D915C91119712962D913C911397C4
:10100000421753072CF4942F852FA901292F382F2D
:10101000D801149660E070E0CB01E2E0F0E0ED84EE
:10102000FE84EE15FF0544F5CD90DD90C216D30683
:101030005CF44901AA2497FCA094BA2C680D791D90
:101040008A1D9B1D960116C04C155D055CF44A0176
:10105000AA2497FCA094BA2C680D791D8A1D9B1DAB
:10106000A60108C0EE24D7FCE094FE2C6C0D7D1D7B
:101070008E1D9F1D3196D3CF0E94A1906B017C01E4
:101080006D857E8562507109882777FD8095982F40
:101090000E94A1909B01AC01C701B6010E94D58FAF
:1010A0006B017C012D853E85243131050CF4BFC0D8
:1010B0004801412C512C3201A12CB12CD4016D914D
:1010C0007D914D01882777FD8095982F0E94A190F2
:1010D000A70196010E940A8F9B01AC010E943592E4
:1010E0009B01AC01C301B2010E940B8F2B013C019B
:1010F000BFEFAB1ABB0AED85FE85AE16BF06F1F653
:10110000BF0161507109882777FD8095982F0E9453
:10111000A1909B01AC01C301B2010E94D58F0E9436
:10112000E8924B015C0120E030E040E85FE30E9480
:10113000769118160CF07BC018870F83212C312C68
:101140001B821C821D821E821A821982AF81B88581
:101150008D919D91B887AF839C01442737FD4095C1
:10116000542F29873A874B875C87CA01B9010E94AF
:10117000A190A70196010E940A8F2B013C0120E05B
:1011800030E0A9010E947691181624F0C301B20143
:10119000905802C0C301B201A50194010E94D18FF1
:1011A00087FF13C08B819C81AD81BE8129853A85E3
:1011B0004B855C85820F931FA41FB51F8B839C8377
:1011C000AD83BE833FEF231A330A49815A814F5FB3
:1011D0005F4F5A8349838D859E854817590709F0CB
:1011E000B5CF20E030E040EC5FE3C501B4010E94E0
:1011F00035924B015C0195E0291631040CF49CCF2B
:101200006B817C818D819E810E94A1906B017C010C
:10121000B101882777FD8095982F0E94A1909B01AE
:10122000AC01C701B6010E94D58F6B017C01C701DB
:10123000B6012E960FB6F894DEBF0FBECDBFDF917C
:10124000CF911F910F91FF90EF90DF90CF90BF90C3
:10125000AF909F908F907F906F905F904F903F9056
:101260002F900895CF93DF93EC01FB01248135810A
:101270000E94458ECE01DF91CF91089526E00C9417
:10128000B584DC01ED91FC910190F081E02D199481
:10129000EF92FF920F931F93CF93DF931F92CDB7DF
:1012A000DEB77C01FC0100811181C80169830E94C5
:1012B00048976981681719F0C8010E945097C701C3
:1012C0000F90DF91CF911F910F91FF90EF900895B4
:1012D000EF92FF920F931F93CF93DF931F921F9272
:1012E000CDB7DEB70DEB1AE08D5B9A407C01C701EC
:1012F000800F911FF80161918F019A838983CE013C
:101300000196C6DFFBE003331F0789F78DEB9AE0F8
:101310000F900F90DF91CF911F910F91FF90EF9061
:1013200008950F931F93CF93DF931F921F92CDB712
:10133000DEB702E01DE0F80160818EED93E09A8354
:101340008983CE010196A4DFF80161818FED93E0DE
:101350009A838983CE0101969BDFC8010F900F907D
:10136000DF91CF911F910F910895BF92CF92DF929D
:10137000EF92FF920F931F93CF93DF93CDB7DEB71A
:1013800062970FB6F894DEBF0FBECDBF6C017B0134
:101390008A0180919904882309F480C0809198047F
:1013A000882309F47BC077FF09C0E094F09440E003
:1013B0006E2D89EE9CE00E94C65E4CC040E060E06D
:1013C00089EE9CE00E94C65E0E94A88128EE33E070
:1013D00040E050E00E949A93BA01A9012AE0CE01B0
:1013E00001960E94548CBE016F5F7F4FCE0107961D
:1013F0000E94DD8B6AE378E0CE0107960E94688D3B
:10140000BC01CE010D960E94DD8BCE0107960E9495
:10141000F38ACE0101960E94F38ABE01635F7F4F7B
:1014200089EE9CE00E949B87B98840E06B2D89EE95
:101430009CE00E94C65EE114F10411F4EB2C06C09E
:1014400040E06E2D89EE9CE00E94C65ECE010D96B6
:101450000E94F38AB60189EE9CE00E949B876CECA7
:1014600079E089EE9CE00E947887F60164816E0D38
:1014700040E089EE9CE00E94C65E0E94A8816093D5
:10148000E50C7093E60C8093E70C9093E80CB801A0
:10149000882777FD8095982F0E94D78162960FB696
:1014A000F894DEBF0FBECDBFDF91CF911F910F919A
:1014B000FF90EF90DF90CF90BF9008954F925F9292
:1014C0006F927F92AF92BF92CF92DF92EF92FF9294
:1014D0000F931F93CF93DF93CDB7DEB762970FB60D
:1014E000F894DEBF0FBECDBF6C017B015A01809125
:1014F0009904882309F498C080919804882309F4FA
:1015000093C00E94A8810091E50C1091E60C2091F7
:10151000E70C3091E80C40908C0450908D04609062
:101520008E0470908F04040D151D261D371D06179F
:1015300017072807390708F077C0F7FE0AC08701A8
:101540000095109540E0602F89EE9CE00E94C65EF9
:1015500047C040E060E089EE9CE00E94C65E0E94C9
:10156000A88128EE33E040E050E00E949A93BA014F
:10157000A9012AE0CE0101960E94548CBE016F5F42
:101580007F4FCE0107960E94DD8B6AE378E0CE01A3
:1015900007960E94688DBC01CE010D960E94DD8BDE
:1015A000CE0107960E94F38ACE0101960E94F38A2B
:1015B000BE01635F7F4F89EE9CE00E949B87098993
:1015C0001A89E114F10441F00E0D1F1D40E0602F57
:1015D00089EE9CE00E94C65ECE010D960E94F38AC1
:1015E000B60189EE9CE00E949B876BEB79E089EE67
:1015F0009CE00E947887F6016481600F40E089EEEC
:101600009CE00E94C65E0E94A8816093E50C7093E6
:10161000E60C8093E70C9093E80CB501882777FDE2
:101620008095982F0E94D78162960FB6F894DEBFFE
:101630000FBECDBFDF91CF911F910F91FF90EF9023
:10164000DF90CF90BF90AF907F906F905F904F9062
:1016500008958F929F92AF92BF92CF92DF92EF92B6
:10166000FF920F931F93CF93DF937C016B01EA01ED
:1016700080919904882309F474C080919804882388
:1016800009F46FC077FF1CC0C094D09441E06C2D6A
:1016900089EE9CE00E94C65EB70189EE9CE00E9444
:1016A0009B876AEA79E089EE9CE00E947887F701DF
:1016B00064816C0D41E089EE9CE00E94C65E3EC0F4
:1016C0000E94A88100918C0410918D0420918E04B9
:1016D00030918F048090E10C9090E20CA090E30C8C
:1016E000B090E40C080D191D2A1D3B1D06171707A5
:1016F00028073907B0F541E06C2D89EE9CE00E9487
:10170000C65EB70189EE9CE00E949B8769E979E09B
:1017100089EE9CE00E947887F70164816C0D41E0BE
:1017200089EE9CE00E94C65E0E94A8816093E10C55
:101730007093E20C8093E30C9093E40CBE01882735
:1017400077FD8095982FDF91CF911F910F91FF909A
:10175000EF90DF90CF90BF90AF909F908F900C94C0
:10176000D781DF91CF911F910F91FF90EF90DF9084
:10177000CF90BF90AF909F908F90089580919904E3
:10178000882379F080919804882359F0E091E90C3E
:10179000F091EA0C0190F081E02D60E089EE9CE090
:1017A0001994089580919904882379F08091980480
:1017B000882359F06FED89EE9CE00E94AA8761E3CF
:1017C00075E089EE9CE00C94A9870895CF93DF9390
:1017D000EC01809199048823A1F0809198048823DA
:1017E00081F06FED89EE9CE00E94AA878C819D813B
:1017F000892B39F0BE0189EE9CE0DF91CF910C94EA
:101800009B87DF91CF91089580919904882301F1FE
:10181000809198048823E1F089EE9CE00E94C05EEC
:1018200040E060E089EE9CE00E94C65E69E879E0F5
:1018300089EE9CE00E94788741E060E089EE9CE0C0
:101840000E94C65E69E779E089EE9CE00C94788797
:101850000895CF93DF93CDB7DEB72C970FB6F894EA
:10186000DEBF0FBECDBF66EA74E0CE0107960E94D0
:101870005E8B6BED7CE0CE0107960E94578DBC011C
:10188000CE0101960E94DD8B48EC50E06FEF7FEFB8
:10189000CE0101966ADDCE0101960E94F38ACE0147
:1018A00007960E94F38A6AEA74E0CE0107960E94C6
:1018B0005E8B65ED7CE0CE0107960E94578DBC01E2
:1018C000CE0101960E94DD8B40ED57E06FEF7FEF78
:1018D000CE010196BEDECE0101960E94F38ACE01B2
:1018E00007960E94F38A8091000D9091010D019757
:1018F00019F46AE679E002C06CE579E0CE01019660
:101900000E94FC8C48EC50E06FEF7FEFCE01019617
:10191000D5DDCE0101960E94F38A6CE479E0CE0118
:1019200001960E94FC8C40ED57E06FEF7FEFCE01F7
:1019300001968FDECE0101960E94F38A6CE379E076
:10194000CE0101960E94FC8C48EC50E06FEF7FEFD7
:10195000CE010196B3DDCE0101960E94F38A6FE2BB
:1019600079E0CE0101960E94FC8C40ED57E06FEFCC
:101970007FEFCE0101966DDECE0101960E94F38AC3
:1019800062E279E0CE0101960E94FC8C48EC50E0C6
:101990006FEF7FEFCE01019691DDCE0101960E949F
:1019A000F38A67E179E0CE0101960E94FC8C40ED5C
:1019B00057E06FEF7FEFCE0101964BDECE0101962F
:1019C0000E94F38A6BE079E0CE0101960E94FC8CC4
:1019D00048EC50E06FEF7FEFCE0101966FDDCE0156
:1019E00001960E94F38A6AEF78E0CE0101960E9488
:1019F000FC8C40ED57E06FEF7FEFCE01019629DEC2
:101A0000CE0101960E94F38A8091000D9091010D04
:101A1000039719F46FEE78E002C065EE78E0CE012E
:101A200001960E94FC8C48EC50E06FEF7FEFCE01F6
:101A3000019644DDCE0101960E94F38A6AED78E0BA
:101A4000CE0101960E94FC8C40ED57E06FEF7FEFD6
:101A5000CE010196FEDDCE0101960E94F38A6DEC67
:101A600078E0CE0101960E94FC8C48EC50E06FEFCC
:101A70007FEFCE01019622DDCE0101960E94F38A0E
:101A80006EEB78E0CE0101960E94FC8C40ED57E0B1
:101A90006FEF7FEFCE010196DCDDCE0101960E9453
:101AA000F38A63EB78E0CE0101960E94FC8C48EC4F
:101AB00050E06FEF7FEFCE01019600DDCE01019681
:101AC0000E94F38A66EA78E0CE0101960E94FC8CBF
:101AD00040ED57E06FEF7FEFCE010196BADDCE010A
:101AE00001960E94F38A8091000D9091010D02975A
:101AF00019F465E978E002C065E878E0CE01019666
:101B00000E94FC8C48EC50E06FEF7FEFCE01019615
:101B1000D5DCCE0101960E94F38A68E778E0CE0119
:101B200001960E94FC8C40ED57E06FEF7FEFCE01F5
:101B300001968FDDCE0101960E94F38A6CE678E073
:101B4000CE0101960E94FC8C48EC50E06FEF7FEFD5
:101B5000CE010196B3DCCE0101960E94F38A6CE5BA
:101B600078E0CE0101960E94FC8C40ED57E06FEFCB
:101B70007FEFCE0101966DDDCE0101960E94F38AC2
:101B800061E578E0CE0101960E94FC8C48EC50E0C3
:101B90006FEF7FEFCE01019691DCCE0101960E949E
:101BA000F38A67E478E0CE0101960E94FC8C40ED58
:101BB00057E06FEF7FEFCE0101964BDDCE0101962E
:101BC0000E94F38A67E378E0CE0101960E94FC8CC4
:101BD00048EC50E06FEF7FEFCE0101966FDCCE0155
:101BE00001960E94F38A6AE278E0CE0101960E9493
:101BF000FC8C40ED57E06FEF7FEFCE01019629DDC1
:101C0000CE0101960E94F38A6EE178E0CE01019642
:101C10000E94FC8C48EC50E06FEF7FEFCE01019604
:101C20004DDCCE0101960E94F38A6EE078E0CE0191
:101C300001960E94FC8C40ED57E06FEF7FEFCE01E4
:101C4000019607DDCE0101960E94F38A2C960FB60D
:101C5000F894DEBF0FBECDBFDF91CF9108954F92B4
:101C60005F926F927F928F929F92AF92BF92CF922C
:101C7000DF92EF92FF92CF93DF93CDB7DEB72C9731
:101C80000FB6F894DEBF0FBECDBFBEDD8BEF9BE07D
:101C90000E9485622B013C018BEF9BE00E94166243
:101CA0004B015C01609138027091390280913A02D7
:101CB00090913B020E94A190AB01BC018BEF9BE095
:101CC0000E9422646B017C01C301B2010E94A190B9
:101CD00020E030E048EC52E40E94D58FAB01BC011B
:101CE00022E0CE0101960E94808CBE016F5F7F4F83
:101CF00083ED9BE00E94E58BCE0101960E94F38A62
:101D00006EE878E083ED9BE00E94358D63ED7BE02B
:101D100089ED9BE00E94C88B6AE878E0CE010196CD
:101D20000E945E8B63ED7BE0CE0101960E94578D91
:101D3000BC0183ED9BE00E94C88BCE0101960E94FE
:101D4000F38A6FE476E08FED9BE00E94FB8B21E04D
:101D5000B501A401CE0101960E94808CBE016F5F87
:101D60007F4F8FED9BE00E942F8DCE0101960E9448
:101D7000F38A6FEA74E08FED9BE00E94358D21E0DD
:101D8000B701A601CE0107960E94808CBE01695F53
:101D90007F4FCE0101960E94DD8B67EE75E0CE018C
:101DA00001960E94688DBC018FED9BE00E942F8DF3
:101DB000CE0101960E94F38ACE0107960E94F38A13
:101DC00063ED7BE0CE0101960E94DD8B66EC74E052
:101DD000CE0101960E94688D6FED7BE00E94578DC9
:101DE000BC018FED9BE00E94C88BCE0101960E9442
:101DF000F38A69ED7BE0CE0101960E94DD8B4AE01B
:101E000050E060E070E0CE010196AFDACE010196BD
:101E10000E94F38A21E0B501A401CE0101960E943F
:101E2000808CBE016F5F7F4F85EE9BE00E94E58B4B
:101E3000CE0101960E94F38A65EE7BE0CE01019609
:101E40000E94DD8B4AE050E06FEF7FEFCE010196FC
:101E500000DCCE0101960E94F38A65EB74E0CE01AE
:101E600001960E945E8BCE010196B0DCCE010196F8
:101E70000E94F38A21E0B701A601CE0107960E94D5
:101E8000808CBE01695F7F4FCE0101960E94DD8B81
:101E900067EE75E0CE0101960E94688DBC0185EE6B
:101EA0009BE00E94C88BCE0101960E94F38ACE016E
:101EB00007960E94F38A65EE7BE0CE0101960E94B0
:101EC000DD8B4AE050E068EF7FEFCE010196C1DB89
:101ED000CE0101960E94F38A8091D00B882331F0C5
:101EE00068E572E080E090E00E94D7812C960FB602
:101EF000F894DEBF0FBECDBFDF91CF91FF90EF9082
:101F0000DF90CF90BF90AF909F908F907F906F9019
:101F10005F904F900895CF93DF93EC018C819D816A
:101F2000892B61F0BE018EE99EE00E94C487BE014C
:101F300088ED9FE0DF91CF910C94C487DF91CF9122
:101F400008951F93CF93DF93CDB7DEB7A8970FB651
:101F5000F894DEBF0FBECDBF182F82E19CE00E9437
:101F6000A96B81110EC067E97AE0CE0101960E944B
:101F7000FC8CCE010196CFDFCE0101960E94F38A40
:101F8000A9C0BE016F5F7F4F82E19CE00E94876A1B
:101F9000112309F499C06DE67AE08EE99EE00E9473
:101FA000B4876EE57AE08EE99EE00E947887BE01F4
:101FB0006F5F7F4F8EE99EE00E94D4876FE47AE0E6
:101FC0008EE99EE00E9478874D855E856F857889D1
:101FD0002AE030E08EE99EE00E94B08860E47AE07A
:101FE0008EE99EE00E94788749895A896B897C89AD
:101FF0002AE030E08EE99EE00E94B08861E37AE05A
:102000008EE99EE00E94788720E030E040E251E4D3
:10201000698D7A8D8B8D9C8D0E943592AB01BC01B0
:1020200022E030E08EE99EE00E94CC8968EC74E00A
:102030008EE99EE00E94D48762E27AE08EE99EE01B
:102040000E94788720E030E040E251E46D8D7E8D83
:102050008F8D98A10E943592AB01BC0122E030E047
:102060008EE99EE00E94CC8968EC74E08EE99EE0E7
:102070000E94D48763E17AE08EE99EE00E9478872F
:1020800020E030E040E251E469A17AA18BA19CA15B
:102090000E943592AB01BC0122E030E08EE99EE067
:1020A0000E94CC8968EC74E08EE99EE00E94D4879F
:1020B0006EEE79E08EE99EE00E94B4876CE67AE0ED
:1020C0008EE99EE00E94D48764EF71E080E090E0AA
:1020D0000E94D781A8960FB6F894DEBF0FBECDBF81
:1020E000DF91CF911F9108954F925F926F927F92EF
:1020F0008F929F92AF92BF92CF92DF92EF92FF9218
:102100000F931F93CF93DF93CDB7DEB7CA54D10996
:102110000FB6F894DEBF0FBECDBF8C016CE67AE03F
:10212000CE01CD960E945E8B6CE67AE0CE01C7961A
:102130000E945E8BBE016F5F7F4F82E19CE00E9438
:10214000476C4D885E886F88788CC98CDA8CEB8CF4
:10215000FC8C8D8D9E8DAF8DB8A12B968CAF9DAFD5
:10216000AEAFBFAF2B97C8010197039708F0E2C14C
:10217000A7019601C301B20190580E947E8F2BEDFA
:102180003FE049EC5FE30E940B8F209134023091D5
:10219000350240913602509137020E940B8F4B015D
:1021A0005C0120E030E0A9010E94D18F87FD09C0C9
:1021B0008092BF0B9092C00BA092C10BB092C20B49
:1021C00010C02BED3FE049EC50E4C501B4010E9482
:1021D0000B8F6093BF0B7093C00B8093C10B9093D8
:1021E000C20B8090BF0B9090C00BA090C10BB09021
:1021F000C20B2BED3FE049EC50E4C501B4010E9455
:102200007691181684F42BED3FE049EC50E4C501BB
:10221000B4010E940A8F6093BF0B7093C00B809330
:10222000C10B9093C20B20E030E044E353E4609193
:10223000BF0B7091C00B8091C10B9091C20B0E949B
:1022400035922BED3FE049E450E40E94D58F609336
:10225000BB0B7093BC0B8093BD0B9093BE0B0E9485
:102260006E904AE0CE018B960E94298C6CEC74E053
:10227000CE0185960E945E8BBE01655D7F4FCE01CB
:1022800085960E94578D66ED74E00E94688DBC01B2
:1022900085EE9BE00E94C88BCE0185960E94F38A52
:1022A000CE018B960E94F38A8090BB0B9090BC0B62
:1022B000A090BD0BB090BE0B20E030E044EB52E4A8
:1022C000C501B4010E94D18F181694F020E030E0CF
:1022D00040E05FE3C501B4010E940B8F0E946E9045
:1022E0004AE0CE018B960E94298C6DED74E023C0EC
:1022F00020E030E044E353E4C501B4010E94D18FF3
:102300001816A4F1A501940160E070E884E393E459
:102310000E940A8F6093BB0B7093BC0B8093BD0B24
:102320009093BE0B0E946E904AE0CE018B960E9465
:10233000298C60EE74E0CE0185960E945E8BBE0112
:10234000655D7F4FCE0185960E94578DBC01CE0101
:10235000CD960E94C88BCE0185960E94F38ACE014D
:102360008B960E94F38A6CED78E063C020E030E049
:1023700047E853E4C501B4010E94D18F181604F157
:1023800020E030E044E353E4C501B4010E940A8F29
:1023900020E030E040E05FE30E940B8F6093BB0BD6
:1023A0007093BC0B8093BD0B9093BE0B0E946E90FC
:1023B0004AE0CE018B960E94298C60EE74E01FC02B
:1023C000A501940160E070E084EB93E40E940A8F21
:1023D00020E030E040E05FE30E940B8F6093BB0B96
:1023E0007093BC0B8093BD0B9093BE0B0E946E90BC
:1023F0004AE0CE018B960E94298C6DED74E0CE01EF
:1024000085960E945E8BBE01655D7F4FCE018596ED
:102410000E94578DBC01CE01CD960E94C88BCE0183
:1024200085960E94F38ACE018B960E94F38A63EE12
:1024300074E0CE01C7960E94FB8BBE01635C7F4FA8
:10244000CE0185960E94DD8B4AE050E060E070E0AE
:10245000CE0185960E94B509CE0185960E94F38A29
:102460000E94A88120918C0430918D0440918E04AB
:1024700050918F048090E50C9090E60CA090E70CB2
:10248000B090E80C280D391D4A1D5B1D2617370733
:102490004807590708F441C20E94A8810E949F90F2
:1024A0004B015C0160918C0470918D0480918E04CD
:1024B00090918F040E94A19020E030E040E85EE31C
:1024C0000E94359227966CAF7DAF8EAF9FAF279756
:1024D0006091E50C7091E60C8091E70C9091E80C0E
:1024E0000E94A1909B01AC0127966CAD7DAD8EAD95
:1024F0009FAD27970E940B8F9B01AC01C501B401D2
:102500000E94D18F87FD09C266EC74E0CE018596EA
:102510000E945E8BBE01695C7F4FCE0185960E9452
:10252000578DBC01CE01CD960E942F8DCE01859690
:102530000E94F38AC8010297029708F0C8C120E000
:1025400030E040E251E4C301B2010E9435924B01F8
:102550005C0120E030E040E251E4C701B6010E9496
:1025600035926B017C0120E030E040E251E42B9693
:102570006CAD7DAD8EAD9FAD2B970E9435922B013A
:102580003C010E94A8812091330B3091340B409183
:10259000350B5091360B621B730B840B950B0E940D
:1025A0009F9020E030E04AE754E40E94D58FAB01D1
:1025B000BC0123E0CE018B960E94808C69EF74E011
:1025C000CE0185960E945E8BBE01655D7F4FCE0178
:1025D00085960E94578D6AE378E00E94688DBC0161
:1025E00083ED9BE00E94C88BCE0185960E94F38A02
:1025F000CE018B960E94F38A63ED7BE0CE01859637
:102600000E94DD8B65EE7BE0CE0185960E94578DA2
:10261000BE01635C7F4F0E94578DBC01CE01CD96F9
:102620000E94C88BCE0185960E94F38A65EE74E005
:102630008FED9BE00E94FB8B21E0B501A401CE0150
:1026400085960E94808CBE016B5D7F4F8FED9BE075
:102650000E942F8DCE0185960E94F38A21E0B3015E
:10266000A201CE0185960E94808C21E0B701A601CF
:10267000CE01C1960E94808C66EC74E0CE018B96F0
:102680000E945E8BBE016F5C7F4FCE018B960E94D5
:10269000578D66EC74E00E94688DBE016B5D7F4FC4
:1026A0000E94578D60EF74E00E94688DBC018FED31
:1026B0009BE00E942F8DCE018B960E94F38ACE0163
:1026C000C1960E94F38ACE0185960E94F38AA501E5
:1026D0009401C501B4010E9435924B015C01A70130
:1026E0009601C701B6010E9435929B01AC01C5015C
:1026F000B4010E940B8F6B017C01A3019201C30105
:10270000B2010E9435929B01AC01C701B6010E9443
:102710000B8F0E94E8926093B70B7093B80B809375
:10272000B90B9093BA0B64EF74E08FED9BE00E94BD
:10273000358D4091B70B5091B80B6091B90B7091EA
:10274000BA0B21E0CE018B960E94808CBE01655DA4
:102750007F4FCE0185960E94DD8B69EC74E0CE013F
:1027600085960E94688DBC0185EE9BE00E94C88B17
:10277000CE0185960E94F38ACE018B960E94F38A41
:1027800065EE7BE08FED9BE00E942F8DC090B70B34
:10279000D090B80BE090B90BF090BA0B20E030E08D
:1027A0004AE754E4C701B6010E94769187FD29C02B
:1027B00020E030E04AE754E4C701B6010E94D58F1B
:1027C000AB01BC0123E0CE018B960E94AE8CBE0112
:1027D000655D7F4FCE0185960E94DD8B6AEC74E0CB
:1027E000CE0185960E94688DBC0185EE9BE00E941B
:1027F000C88BCE0185960E94F38ACE018B960E94EB
:10280000F38A20E030E64AE656E46091B70B709117
:10281000B80B8091B90B9091BA0B0E94D18FBE0179
:10282000635C7F4F87FF4FC0CE0185960E94DD8B92
:1028300068EF74E0CE0185960E94688D6FED7BE0B5
:102840000E94578DBC018FED9BE00E94C88BCE018A
:1028500085960E94F38A0330110599F46FED7BE0B1
:10286000CE0185960E94DD8BCE01859654DBCE018C
:1028700085960E94F38A6CE67AE08FED9BE00E94D9
:10288000FB8B6BEF74E0CE018B960E945E8B65EE46
:102890007BE0CE018B960E94578DBC01CE018596C0
:1028A0000E94DD8B4AE050E06FEF7FEFCE0185960E
:1028B0000E94290BCE0185960E94F38ACE018B9649
:1028C0000E94F38A04C08FED9BE00E94C88B6AE0EF
:1028D00070E080E090E00E94D781CE01C7960E9410
:1028E000F38ACE01CD960E94F38AC65BDF4F0FB606
:1028F000F894DEBF0FBECDBFDF91CF911F910F9136
:10290000FF90EF90DF90CF90BF90AF909F908F900F
:102910007F906F905F904F9008956CE67AE0CE01C3
:1029200085960E945E8BCE0185960E94E60BCE01B5
:1029300085960E94F38ABE01695C7F4F89EE9CE018
:102940000E949B87E1CD8F929F92AF92BF92CF92D0
:10295000DF92EF92FF920F931F93CF93DF9300D0FC
:1029600000D0CDB7DEB78C01C0900A02D0900B0228
:10297000E0900C02F0900D0220E030E040E450E4E2
:10298000C701B6010E94769118166CF420E030E081
:102990004AE754E4C701B6010E9435920E946E9046
:1029A0006B017C0106C080E3C82E85E7D82EE12CA0
:1029B000F12C0E94040C40E060E089EE9CE00E9453
:1029C000C65E64E075E089EE9CE00E94A98741E064
:1029D00060E089EE9CE00E94C65E65E175E089EEEC
:1029E0009CE00E94A98764E670E080E090E00E948D
:1029F000D7810E94A8816093330B7093340B80932E
:102A0000350B9093360B0E94A8818090330B9090E9
:102A1000340BA090350BB090360BDC01CB0188193C
:102A20009909AA09BB098C159D05AE05BF055CF483
:102A3000C8015ADB0E94A88164E170E080E090E068
:102A40000E94D781E0CF0130110509F041C06FED40
:102A50007BE089ED9BE00E94C88B0E94040C69ED2D
:102A60007BE0CE0101960E94DD8B4AE050E060E001
:102A700070E0CE0101960E94B509CE0101960E9438
:102A8000F38A6DED79E0CE0101960E94FC8C4AE05C
:102A900050E06FEF7FEFCE0101960E94290BCE012F
:102AA00001960E94F38A6DE175E0CE0101960E94C5
:102AB0005E8B6FED7BE0CE0101960E94578DBC01CD
:102AC0008FED9BE00E94C88BCE0101960E94F38A95
:102AD00026960FB6F894DEBF0FBECDBFDF91CF9123
:102AE0001F910F91FF90EF90DF90CF90BF90AF902C
:102AF0009F908F900895CF92DF92EF92FF92CF93A5
:102B0000DF9300D000D0CDB7DEB70E94040C6EE199
:102B100070E080E090E00E94D7818BEF9BE00E9404
:102B200016626B017C0164E670E080E090E00E9438
:102B3000D7816FE476E08FED9BE00E94FB8B21E074
:102B4000B701A601CE0101960E94808CBE016F5F85
:102B50007F4F8FED9BE00E942F8DCE0101960E944A
:102B6000F38A6FED7BE0CE0101960E94DD8B4AE097
:102B700050E060E070E0CE0101960E94B509CE0100
:102B800001960E94F38A0E94D20B60E375E08FEDFC
:102B90009BE00E94358DC092C70BD092C80BE0928B
:102BA000C90BF092CA0B20E030E040EF51E4C701BE
:102BB000B6010E94769187FD03C06AEC77E054C0AD
:102BC00020E030E040ED51E4C701B6010E9476916B
:102BD00087FD1FC06AEB77E0CE0101960E94FC8C56
:102BE0004AE050E06FEF7FEFCE0101960E94290B83
:102BF000CE0101960E94F38A80919C04882331F0D3
:102C00006CED75E080E090E00E94D7816AEA77E0A1
:102C10002BC020E030E040EB51E4C701B6010E9438
:102C2000769187FD03C06CE977E01EC06DE877E020
:102C3000CE0101960E94FC8C4AE050E06FEF7FEFDE
:102C4000CE0101960E94290BCE0101960E94F38AC3
:102C500080919C04882331F06CED75E080E090E079
:102C60000E94D7816FE777E0CE0101960E94FC8C2D
:102C70004AE050E06FEF7FEFCE0101960E94290BF2
:102C8000CE0101960E94F38A6CE271E080E090E050
:102C90000E94D78180919C04882331F068EE73E014
:102CA00080E090E00E94D78126960FB6F894DEBFB0
:102CB0000FBECDBFDF91CF91FF90EF90DF90CF900F
:102CC0000895CF92DF92EF92FF92CF93DF93CDB72B
:102CD000DEB72C970FB6F894DEBF0FBECDBF61E70D
:102CE00077E0CE0101960E94FC8C4AE050E06FEF45
:102CF0007FEFCE0101960E94290BCE0101960E9422
:102D0000F38A60916E0470916F0483E49CE00E94EA
:102D1000DF7CE12CF12C64E670E080E090E00E9422
:102D2000D78160916E0470916F0483E49CE00E94EF
:102D3000DF7C2FEFE21AF20A23E0E216F1045CF3E3
:102D40002AE0E216F1041CF4892B29F703C0892B31
:102D500009F0D4C06091450C7091460C882777FD2E
:102D60008095982F0E94A1906B017C016093C70B06
:102D70007093C80B8093C90B9093CA0B6091430C5E
:102D80007091440C882777FD8095982F0E94A19020
:102D90006093C30B7093C40B8093C50B9093C60BC9
:102DA00021E0B701A601CE0107960E94808C6FE456
:102DB00076E0CE0101960E945E8BBE01695F7F4F77
:102DC000CE0101960E94578DBC018FED9BE00E94C1
:102DD000C88BCE0101960E94F38ACE0107960E940D
:102DE000F38A4091C30B5091C40B6091C50B709155
:102DF000C60B21E0CE0107960E94808C63E375E04C
:102E0000CE0101960E945E8BBE01695F7F4FCE01AD
:102E100001960E94578DBC018FED9BE00E942F8D83
:102E2000CE0101960E94F38ACE0107960E94F38A92
:102E300069E276E08FED9BE00E94358D6CE67AE0EA
:102E4000CE0101960E945E8B44E150E060E070E0AC
:102E5000CE0101960E94B509CE0101960E94F38A27
:102E60006091C70B7091C80B8091C90B9091CA0BF0
:102E70000E946E904AE0CE0101960E94298CBE010C
:102E80006F5F7F4F89ED9BE00E94E58BCE0101963D
:102E90000E94F38A40E066E089EE9CE00E94C65EF4
:102EA00069ED7BE089EE9CE00E949B876FED89EEE7
:102EB0009CE00E94AA8765EB74E089EE9CE00E948A
:102EC000A9876091C30B7091C40B8091C50B909141
:102ED000C60B0E946E904AE050E089EE9CE00E9492
:102EE000938869E276E089EE9CE00E94A98764E617
:102EF00070E080E090E00E94D78118C066E677E03D
:102F0000CE0101960E94FC8C4AE050E060E070E047
:102F1000CE0101960E94B509CE0101960E94F38A66
:102F200066E477E08FED9BE00E94DC8C2C960FB678
:102F3000F894DEBF0FBECDBFDF91CF91FF90EF9031
:102F4000DF90CF900895CF92DF92EF92FF92CF93D0
:102F5000DF93CDB7DEB72C970FB6F894DEBF0FBE68
:102F6000CDBF68E377E0CE0101960E94FC8C4CE275
:102F700051E06FEF7FEFCE0101960E94290BCE0149
:102F800001960E94F38A60916E0470916F0483E44D
:102F90009CE00E94DF7CE12CF12C64E670E080E094
:102FA00090E00E94D78160916E0470916F0483E479
:102FB0009CE00E94DF7C2FEFE21AF20A23E0E21687
:102FC000F1045CF32AE0E216F1041CF4892B29F7E2
:102FD00003C0892B09F057C16091450C7091460CD4
:102FE000882777FD8095982F0E94A1906B017C0126
:102FF0006093C70B7093C80B8093C90B9093CA0B57
:103000006091430C7091440C882777FD8095982F30
:103010000E94A1906093C30B7093C40B8093C50B67
:103020009093C60B21E0B701A601CE0107960E943E
:10303000808C6FE476E0CE0101960E945E8BBE012B
:10304000695F7F4FCE0101960E94578DBC018FEDC5
:103050009BE00E94C88BCE0101960E94F38ACE01AC
:1030600007960E94F38A4091C30B5091C40B609164
:10307000C50B7091C60B21E0CE0107960E94808C93
:1030800063E375E0CE0101960E945E8BBE01695F2D
:103090007F4FCE0101960E94578DBC018FED9BE0C2
:1030A0000E942F8DCE0101960E94F38ACE010796D1
:1030B0000E94F38A69E276E08FED9BE00E94358DF5
:1030C0006CE67AE0CE0101960E945E8B44E150E00E
:1030D00060E070E0CE0101960E94B509CE01019634
:1030E0000E94F38A6091C70B7091C80B8091C90B45
:1030F0009091CA0B0E946E904AE0CE0101960E9408
:10310000298CBE016F5F7F4F89ED9BE00E94E58BAC
:10311000CE0101960E94F38A40E066E089EE9CE0D1
:103120000E94C65E69ED7BE089EE9CE00E949B8771
:103130006FED89EE9CE00E94AA8765EB74E089EE52
:103140009CE00E94A9876091C30B7091C40B809191
:10315000C50B9091C60B0E946E904AE050E089EE3C
:103160009CE00E94938869E276E089EE9CE00E94F0
:10317000A98764E670E080E090E00E94D7818BEE42
:103180009BE00E94E48EC090C70BD090C80BE090EB
:10319000C90BF090CA0B20E030E040EF51E4C701CA
:1031A000B6010E94769187FD03C069E277E054C0C2
:1031B00020E030E040ED51E4C701B6010E94769175
:1031C00087FD1FC069E177E0CE0101960E94FC8C6B
:1031D0004AE050E06FEF7FEFCE0101960E94290B8D
:1031E000CE0101960E94F38A80919C04882331F0DD
:1031F0006CED75E080E090E00E94D78169E077E0B7
:103200002BC020E030E040EB51E4C701B6010E9442
:10321000769187FD03C06BEF76E01EC06CEE76E022
:10322000CE0101960E94FC8C4AE050E06FEF7FEFE8
:10323000CE0101960E94290BCE0101960E94F38ACD
:1032400080919C04882331F06CED75E080E090E083
:103250000E94D7816EED76E0CE0101960E94FC8C33
:103260004AE050E06FEF7FEFCE0101960E94290BFC
:10327000CE0101960E94F38A62E370E080E090E064
:103280000E94D78101C037DC2C960FB6F894DEBFC0
:103290000FBECDBFDF91CF91FF90EF90DF90CF9029
:1032A0000895CF92DF92EF92FF921F93CF93DF9317
:1032B000CDB7DEB7AA970FB6F894DEBF0FBECDBF6D
:1032C000182F882331F06CE67AE08EE99EE00E94A8
:1032D000D48787E49CE00E94666DBE016F5F7F4FDC
:1032E00087E49CE00E94026DCE010D967C011123C3
:1032F00021F167EC76E08EE99EE00E94B487FE0142
:1033000031966F01F60141915191619171916F0177
:1033100026E030E08EE99EE00E94CC8966EC74E005
:103320008EE99EE00E94A987CE14DF0459F76CE66F
:103330007AE08EE99EE00E94D48723E938E144E8F0
:103340005FE369817A818B819C810E9435926D87D0
:103350007E878F87988B22E430E645E85FE36D81B6
:103360007E818F8198850E943592698B7A8B8B8BB9
:103370009C8B25E83BEE41E95FE369857A858B8587
:103380009C850E9435926D8B7E8B8F8B988FB701B9
:1033900087E49CE00E94E26C112309F48FC0B7011E
:1033A00087E49CE00E94026D6AEB76E08EE99EE085
:1033B0000E94B4876E01F9E1CF0ED11CF701419153
:1033C0005191619171917F0122E030E08EE99EE0A0
:1033D0000E94CC8966EC74E08EE99EE00E94A98789
:1033E000EC14FD0459F76CE67AE08EE99EE00E9449
:1033F000D4876E01F5E2CF0ED11C9601AE01495D76
:103400005F4FBE01675D7F4F87E49CE00E94526E74
:103410006DEA76E08EE99EE00E94788769A57AA53C
:103420004AE050E08EE99EE00E94938866EC74E0EA
:103430008EE99EE00E94A9876FA178A54AE050E03E
:103440008EE99EE00E94938866EC74E08EE99EE02F
:103450000E94A9876DA17EA14AE050E08EE99EE01E
:103460000E9493886CE67AE08EE99EE00E94D48701
:10347000B70187E49CE00E94906E64EA76E08EE9F2
:103480009EE00E947887F70141915191619171917D
:103490007F012AE030E08EE99EE00E94CC8966EC54
:1034A00074E08EE99EE00E94A987EC14FD0459F7B0
:1034B0006CE67AE08EE99EE00E94D48761E070E0DD
:1034C00087E49CE00E947B6D112389F060E976E03F
:1034D0008EE99EE00E94788787E49CE00E94DA6E85
:1034E0004AE050E0BC018EE99EE00E949A8824E008
:1034F00030E043E050E062E070E087E49CE00E944E
:10350000886D1123E9F164E776E08EE99EE00E9480
:1035100078879E012B5D3F4FAE01495D5F4FBE0135
:10352000675D7F4F87E49CE00E94EC6E69A57AA5F9
:103530004AE050E08EE99EE00E94938866EC74E0D9
:103540008EE99EE00E94A9876FA178A54AE050E02D
:103550008EE99EE00E94938866EC74E08EE99EE01E
:103560000E94A9876DA17EA14AE050E08EE99EE00D
:103570000E9493886CE67AE08EE99EE00E94D487F0
:1035800065E070E087E49CE00E94A56D112389F05E
:1035900061E676E08EE99EE00E94788787E49CE011
:1035A0000E942F6F4AE050E0BC018EE99EE00E942D
:1035B0009A8866E070E087E49CE00E94B26D112377
:1035C00089F069E476E08EE99EE00E94788787E4DE
:1035D0009CE00E94416F4AE050E0BC018EE99EE011
:1035E0000E949A8867E070E087E49CE00E94B56DD5
:1035F000112389F063E376E08EE99EE00E947887EC
:1036000087E49CE00E94536F4AE050E0BC018EE9E1
:103610009EE00E949A8868E070E087E49CE00E9447
:10362000C26D112389F06BE176E08EE99EE00E9485
:10363000788787E49CE00E94656F4AE050E0BC0117
:103640008EE99EE00E949A8869E070E087E49CE041
:103650000E94CF6D112389F061E076E08EE99EE053
:103660000E94788787E49CE00E94776F4AE050E0F0
:10367000BC018EE99EE00E949A886AE070E087E4CF
:103680009CE00E94DC6D112389F06BEE75E08EE901
:103690009EE00E94788787E49CE00E94896F4AE060
:1036A00050E0BC018EE99EE00E949A886BE070E0D9
:1036B00087E49CE00E94E96D112389F062ED75E0DA
:1036C0008EE99EE00E94788787E49CE00E949B6FD1
:1036D0004AE050E0BC018EE99EE00E949A886CE0CE
:1036E00070E087E49CE00E94F66D112309F48FC01E
:1036F0006AEB75E08EE99EE00E94788787E49CE0A3
:103700000E94AD6F4AE050E0BC018EE99EE00E944D
:103710009A8863EA75E08EE99EE00E94788787E4E4
:103720009CE00E94D270682F70E04AE050E08EE981
:103730009EE00E949A886CE875E08EE99EE00E9407
:10374000788787E49CE00E94D670682F70E04AE09A
:1037500050E08EE99EE00E949A8865E775E08EE968
:103760009EE00E94788787E49CE00E94DA70682FD0
:1037700070E04AE050E08EE99EE00E949A886CE595
:1037800075E08EE99EE00E94788787E49CE00E94C5
:10379000DE70682F70E04AE050E08EE99EE00E9403
:1037A0009A8863E475E08EE99EE00E94788787E45A
:1037B0009CE00E94E270682F70E04AE050E08EE9E1
:1037C0009EE00E949A886AE275E08EE99EE00E947F
:1037D000788787E49CE00E94E670682F70E04AE0FA
:1037E00050E08EE99EE00E949A8869E175E08EE9DA
:1037F0009EE00E94788787E49CE00E94EA70682F30
:1038000070E04AE050E08EE99EE00E949A8861E014
:1038100087E49CE00E94877061E087E49CE00E945E
:103820008C7061E087E49CE00E949170112391F01C
:1038300060E075E08EE99EE00E94788787E49CE076
:103840000E94EE70682F70E04AE050E08EE99EE042
:103850000E949A8860E087E49CE00E9491701123A6
:1038600091F066EE74E08EE99EE00E94788787E42E
:103870009CE00E94EE70682F70E04AE050E08EE914
:103880009EE00E949A8861E087E49CE00E94967026
:10389000112391F06AEC74E08EE99EE00E94788733
:1038A00087E49CE00E94F270682F70E04AE050E0EC
:1038B0008EE99EE00E949A8860E087E49CE00E9486
:1038C0009670112391F06DEA74E08EE99EE00E94FB
:1038D000788787E49CE00E94F270682F70E04AE0ED
:1038E00050E08EE99EE00E949A8861E087E49CE0C7
:1038F0000E949B70112391F061E974E08EE99EE0D3
:103900000E94788787E49CE00E94F670682F70E040
:103910004AE050E08EE99EE00E949A8860E087E4E9
:103920009CE00E949B70112391F064E774E08EE9A3
:103930009EE00E94788787E49CE00E94F670682FE2
:1039400070E04AE050E08EE99EE00E949A8861E0D3
:1039500087E49CE00E94A070112391F068E574E078
:103960008EE99EE00E94788787E49CE00E94FA70CE
:10397000682F70E04AE050E08EE99EE00E949A884D
:1039800060E087E49CE00E94A070112391F06BE35B
:1039900074E08EE99EE00E94788787E49CE00E94B4
:1039A000FA70682F70E04AE050E08EE99EE00E94D5
:1039B0009A8861E087E49CE00E94697061E087E496
:1039C0009CE00E946E7061E087E49CE00E9473704E
:1039D00060E087E49CE00E94787060E087E49CE00F
:1039E0000E947D7060E087E49CE00E948270112359
:1039F00009F490C063E274E08EE99EE00E9478874B
:103A000087E49CE00E94FE70682F70E04AE050E07E
:103A10008EE99EE00E949A8865E074E08EE99EE05F
:103A20000E94788787E49CE00E940271682F70E012
:103A30004AE050E08EE99EE00E949A8867EE73E0CB
:103A40008EE99EE00E94788787E49CE00E940671E0
:103A5000682F70E04AE050E08EE99EE00E949A886C
:103A60006EEC73E08EE99EE00E94788787E49CE02C
:103A70000E940A71682F70E04AE050E08EE99EE0F3
:103A80000E949A8865EB73E08EE99EE00E94788739
:103A900087E49CE00E940E71682F70E04AE050E0DD
:103AA0008EE99EE00E949A886CE973E08EE99EE0C0
:103AB0000E94788787E49CE00E941271682F70E072
:103AC0004AE050E08EE99EE00E949A8869E873E03F
:103AD0008EE99EE00E94788787E49CE00E94167140
:103AE000682F70E04AE050E08EE99EE00E949A88DC
:103AF00064E773E08EE99EE00E94788787E49CE0AB
:103B00000E941A71682F70E04AE050E08EE99EE052
:103B10000E949A8860E087E49CE00E94A57040EDD6
:103B20005FE069E470E487E49CE00E94E86F1123A1
:103B300009F449C060E673E08EE99EE00E94788750
:103B400087E49CE00E94BF6FAB01BC0122E030E043
:103B50008EE99EE00E94CD8969E473E08EE99EE0E3
:103B60000E94788787E49CE00E9423704AE050E03E
:103B7000682F8EE99EE00E94CC8861E373E08EE9B5
:103B80009EE00E94788761E087E49CE00E941E71BD
:103B9000682F70E04AE050E08EE99EE00E949A882B
:103BA00068E173E08EE99EE00E94788761E087E437
:103BB0009CE00E942271682F70E04AE050E08EE99C
:103BC0009EE00E949A8841E061E087E49CE00E94C8
:103BD000AA70112399F060E073E08EE99EE00E94E4
:103BE000788761E087E49CE00E942671682F70E08E
:103BF0004AE050E08EE99EE00E949A8841E061E050
:103C000087E49CE00E94AF7060E087E49CE00E9443
:103C100064701123B1F06DEE72E08EE99EE00E94B7
:103C2000788787E49CE00E94CE70682F70E04AE0BD
:103C300050E08EE99EE00E949A8887E49CE00E9412
:103C40002A71AA960FB6F894DEBF0FBECDBFDF91E2
:103C5000CF911F91FF90EF90DF90CF9008952F921A
:103C60003F924F925F926F927F928F929F92AF920C
:103C7000BF92CF92DF92EF92FF920F931F93CF9359
:103C8000DF93CDB7DEB7C554D1090FB6F894DEBFC8
:103C90000FBECDBF2B013C012DA33EA34FA358A7C0
:103CA0000E94A88122966CAF7DAF8EAF9FAF229706
:103CB00020E9421621E052066104710434F020E943
:103CC000422E55245394612C712C8DA19EA1AFA13D
:103CD000B8A580319742A105B1052CF030E127E26B
:103CE00090E080E004C03DA12EA19FA188A5409155
:103CF000D00B411104C03DA32EA39FA388A72296F9
:103D00006CAD7DAD8EAD9FAD229728EE33E040E0E7
:103D100050E00E949A9326962CAF3DAF4EAF5FAF16
:103D20002697F1E0FDAB19A61AA61BA61CA68E01CC
:103D3000035F1F4F22273327A9012419350946099C
:103D4000570929AB3AAB4BAB5CAB29A53AA54BA5C0
:103D50005CA58DA19EA1AFA1B8A5281739074A0778
:103D60005B070CF035C369A57AA58BA59CA50E94BD
:103D7000A19020E030E04AE754E40E94D58FAB01E7
:103D8000BC0123E0C8010E94808CB80189ED9BE052
:103D90000E94E58BC8010E94F38A8DA19EA1AFA16C
:103DA000B8A50A97A105B10594F42AE026964CAD72
:103DB0005DAD6EAD7FAD2697C8010E94548CB801F1
:103DC00089ED9BE00E94E58BC8010E94F38ABE0149
:103DD0006F5F7F4F87E49CE00E94906E69E375E01F
:103DE0008FED9BE00E94FB8BDE0111961D01C12C23
:103DF000D12C7601F10181909190A190B1901F0199
:103E0000A5019401C501B4010E9435929B01AC014A
:103E1000C701B6010E940B8F6B017C0123E0B50145
:103E2000A401CE0143960E94AE8CBE016D5E7F4F11
:103E3000C8010E94DD8B66EC74E0C8010E94688DA9
:103E4000BC018FED9BE00E942F8DC8010E94F38A78
:103E5000CE0143960E94F38A2016310659F6C70117
:103E6000B6010E94E8926B017C01FDE24F16F1E081
:103E70005F066104710444F00E94040C40E060E0BD
:103E800089EE9CE00E94C65E23E0B701A601C8014E
:103E90000E94808C68EF74E0CE0143960E945E8B96
:103EA00069ED7BE0CE0143960E94578D66E475E094
:103EB0000E94688DB8010E94578D6BE475E00E94E6
:103EC000688DBC018FED9BE00E942F8DCE01439643
:103ED0000E94F38AC8010E94F38A2DEC3CEC4CE46A
:103EE0005FE3C701B6010E94769129813A814B8137
:103EF0005C812DA73EA74FA758AB18160CF0ACC19C
:103F00002AE939E949E95FE3C701B6010E94D18F87
:103F100087FFA2C13DA9332309F49EC189849A84F5
:103F2000AB84BC8420E030E0A901C501B4010E944B
:103F3000D18FCD80DE80EF80F884882309F12DA514
:103F40003EA54FA558A9CA01B9010E9435926EAB92
:103F50007FAB88AF99AFA7019601C701B6010E9458
:103F600035929B01AC016EA97FA988AD99AD0E94E5
:103F70000B8F0E94E892A50194010E947E8F04C0DD
:103F80006BED7FE089EC9FE320EE3EE245E652E4F4
:103F90000E9435926EAB7FAB88AF99AF20E030E0E6
:103FA000A901C701B6010E94D18F882309F12DA56F
:103FB0003EA54FA558A9CA01B9010E9435926AAF22
:103FC0007BAF8CAF9DAFA5019401C501B4010E94E8
:103FD00035929B01AC016AAD7BAD8CAD9DAD0E946D
:103FE0000B8F0E94E892A70196010E947E8F04C069
:103FF0006BED7FE089EC9FE320EE3EE245E652E484
:104000000E9435926AAF7BAF8CAF9DAF20E030E06D
:10401000A9016DA57EA58FA598A90E94D18F88239F
:10402000F9F0A5019401C501B4010E9435924B013C
:104030005C01A7019601C701B6010E9435929B0160
:10404000AC01C501B4010E940B8F0E94E8922DA51E
:104050003EA54FA558A90E947E8F6B017C0108C028
:104060009BEDC92E9FE0D92E99ECE92E9FE3F92E06
:1040700069EF74E0C8010E945E8B69ED7BE0C801C6
:104080000E94578D6EE475E00E94688DBC018FED33
:104090009BE00E94C88BC8010E94F38A69EF74E01C
:1040A000C8010E945E8B69ED7BE0C8010E94578DBC
:1040B00068E675E00E94688DBC0189ED9BE00E9476
:1040C000C88BC8010E94F38A21E04EA95FA968ADA0
:1040D00079ADC8010E94808C21E04AAD5BAD6CAD2A
:1040E0007DADCE0143960E94808C20EE3EE245E6F7
:1040F00052E4C701B6010E943592AB01BC0121E038
:10410000CE014F960E94808CBE01615E7F4FCE0132
:1041100049960E94DD8B66EC74E0CE0149960E94C0
:10412000688DBE016D5E7F4F0E94578D66EC74E016
:104130000E94688DB8010E94578DBC0183ED9BE001
:104140000E94C88BCE0149960E94F38ACE014F96F9
:104150000E94F38ACE0143960E94F38AC8010E940E
:10416000F38A4DE2441641E054066104710474F48C
:1041700069A57AA58BA59CA525E030E040E050E03C
:104180000E949A93672B682B692BC1F569ED7BE040
:10419000C8010E94DD8B45E050E06FEF7FEFC80162
:1041A0000E945E0AC8010E94F38A61E775E0C801B7
:1041B0000E945E8B45E050E061EF7FEFC8010E94F6
:1041C000B509C8010E94F38A6CE67AE0C8010E9432
:1041D0005E8BC8010E94E60BC8010E94F38A63ED62
:1041E0007BE0C8010E94DD8B45E050E060E070E0BC
:1041F000C8010E94290BC8010E94F38A63ED7BE08D
:104200008FED9BE00E942F8D5FE145165104610404
:10421000710434F489A59AA5ABA5BCA5B7FD11C05E
:104220006FED7BE0C8010E94DD8BC8010E948B0FFF
:10423000C8010E94F38A6CE67AE08FED9BE00E9451
:10424000FB8BB201C30177FE04C069A97AA98BA9CF
:104250009CA90E94D781A9C023E04DA55EA56FA5AA
:1042600078A9C8010E94808C69EF74E0CE01439662
:104270000E945E8B69ED7BE0CE0143960E94578DD4
:1042800063E775E00E94688DB8010E94578D6CE469
:1042900075E00E94688DBC0189ED9BE00E94C88B8F
:1042A000CE0143960E94F38AC8010E94F38A498591
:1042B0005A856B857C8523E0C8010E94AE8C4D81B8
:1042C0005E816F81788523E0CE0149960E94AE8C95
:1042D000BE01675E7F4FCE0143960E94DD8B68E78B
:1042E00075E0CE0143960E94688DB8010E94578DFB
:1042F0006CE475E00E94688DBC0183ED9BE00E9438
:10430000C88BCE0143960E94F38ACE0149960E9443
:10431000F38AC8010E94F38A9DE2491691E059068A
:104320006104710474F469A57AA58BA59CA525E0A8
:1043300030E040E050E00E949A93672B682B692B95
:10434000F1F469ED7BE0C8010E94DD8B4AE050E0AA
:104350006FEF7FEFC8010E945E0AC8010E94F38AD6
:1043600063ED7BE0C8010E94DD8B4AE050E060E035
:1043700070E0C8010E94290BC8010E94F38A6FED0A
:104380007BE0C8010E94DD8BC8010E948B0FC80131
:104390000E94F38A6CE67AE08FED9BE00E94FB8B33
:1043A000C301B2010E94D7811DAA0E94A8819B016E
:1043B000AC0122968CAD9DADAEADBFAD2297281B52
:1043C000390B4A0B5B0B29A73AA74BA75CA7BDCCBF
:1043D00069ED7BE0CE010D960E94DD8B4AE050E056
:1043E0006FEF7FEFCE010D960E94B509CE010D96BD
:1043F0000E94F38A9DA99923B1F161E775E0CE018E
:104400000D960E945E8B45E050E061EF7FEFCE019C
:104410000D960E94B509CE010D960E94F38A8091F7
:10442000D00B882391F065EE72E0CE010D960E94CC
:10443000FC8C45E050E060E070E0CE010D960E94FB
:10444000B509CE010D960E94F38A6CE67AE0CE01A2
:104450000D960E945E8BCE010D960E94E60BCE015A
:104460000D960E94F38A63ED7BE0CE010D960E94CB
:10447000DD8B4AE050E06FEF7FEFCE010D960E949A
:10448000290BCE010D960E94F38ACB5BDF4F0FB64E
:10449000F894DEBF0FBECDBFDF91CF911F910F917A
:1044A000FF90EF90DF90CF90BF90AF909F908F9054
:1044B0007F906F905F904F903F902F900895CF9294
:1044C000DF92EF92FF920F931F93CF93DF93CDB7BD
:1044D000DEB72C970FB6F894DEBF0FBECDBF80912C
:1044E000D00B811102C00E94040C8BE39FE00E945C
:1044F000178564E670E080E090E00E94D78169EC67
:1045000072E089ED9BE00E94DC8C69ED7BE0CE01DE
:1045100001960E94DD8B44E150E060E070E0CE0146
:1045200001960E94B509CE0101960E94F38A6AEBBA
:1045300072E089ED9BE00E94DC8C69ED7BE0CE01AE
:1045400001960E94DD8B44E150E06FEF7FEFCE01DA
:1045500001960E94290BCE0101960E94F38A60E029
:1045600070E08AEC9CE00E946A656B017C0104E0CB
:1045700010E0A7019601C701B6010E942993882384
:1045800009F43DC00150110909F011C16FEA72E050
:1045900089ED9BE00E94DC8C69ED7BE0CE01019609
:1045A0000E94DD8B4AE050E060E070E0CE010196B1
:1045B0000E94B509CE0101960E94F38A6BE775E06F
:1045C000CE0101960E945E8B69ED7BE0CE010196E3
:1045D0000E94578DBC018FED9BE00E94C88BCE01DD
:1045E00001960E94F38A8091000D9091010D03972E
:1045F00009F0CCC01092010D1092000DC7C021E04F
:10460000B701A601CE0107960E94808C6DE875E087
:10461000CE0101960E945E8BBE01695F7F4FCE0185
:1046200001960E94578DBC018FED9BE00E94C88BC4
:10463000CE0101960E94F38ACE0107960E94F38A6A
:104640006FED7BE0CE0101960E94DD8B42E350E0EE
:104650006FEF7FEFCE0101960E94290BCE010196EC
:104660000E94F38A0E94D20B60E375E08FED9BE01D
:104670000E94358D60E070E08AEC9CE00E946865E5
:104680006B017C0104E010E0A7019601C701B601AF
:104690000E942993882359F00150110909F096C00E
:1046A0006CE67AE085EE9BE00E94FB8B50C021E037
:1046B000B701A601CE0107960E94808C6FE476E0D8
:1046C000CE0101960E945E8BBE01695F7F4FCE01D5
:1046D00001960E94578DBC0185EE9BE00E94C88B1D
:1046E000CE0101960E94F38ACE0107960E94F38ABA
:1046F00066EC74E0CE0101960E945E8B65EE7BE075
:10470000CE0101960E94578DBC0189ED9BE00E946D
:10471000C88BCE0101960E94F38A69ED7BE0CE0141
:1047200001960E94DD8B4AE050E060E070E0CE012F
:1047300001960E945E0ACE0101960E94F38A0E94B1
:10474000D20B60E375E085EE9BE00E94358D65EE4F
:104750007BE0CE0101960E94DD8B66EC74E0CE0119
:1047600001960E94688D6FED7BE00E94578DBC0121
:104770008FED9BE00E94C88BCE0101960E94F38AC8
:1047800083E090E09093010D8093000D64E670E06B
:1047900080E090E00E94D7818091D00B882329F19E
:1047A00060E273E080E090E00E94D7811EC064E682
:1047B00070E080E090E00E94D78160E070E08AECD9
:1047C0009CE00E946A656B017C01D3CE68EC70E0CE
:1047D00080E090E00E94D78160E070E08AEC9CE08D
:1047E0000E9468656B017C014FCF2C960FB6F89440
:1047F000DEBF0FBECDBFDF91CF911F910F91FF9014
:10480000EF90DF90CF9008951F93CF93DF93182FF1
:10481000C7E6DBE0812F0E946D82899399936CE358
:1048200070E080E090E00E94D7818BE0C73BD80722
:1048300089F768E270E087E69BE00E94DB0720E0F2
:1048400030E040EA50E40E94359220E030E040E859
:104850005AE30E943592DF91CF911F9108954F92B4
:104860005F926F927F928F929F92AF92BF92CF9200
:10487000DF92EF92FF920F931F93CF93DF93CDB709
:10488000DEB764970FB6F894DEBF0FBECDBF7C01D4
:104890008B0165EA72E089ED9BE00E94DC8C0E944E
:1048A000040C69ED7BE0CE0101960E94DD8B4AE0AD
:1048B00050E06FEF7FEFCE0101960E94B509CE0167
:1048C00001960E94F38AC7019FDF698B7A8B8B8BDD
:1048D0009C8B40901A0250901B0260901C027090BA
:1048E0001D02A3019201609116027091170280913E
:1048F0001802909119020E940A8F4B015C0120E07E
:1049000030E0A9010E94D18F882309F451C0C090E2
:104910002202D0902302E0902402F090250220E0B1
:1049200030E0A901C701B6010E94D18F18160CF022
:104930003FC080911E0290911F02A0912002B09171
:1049400021028D879E87AF87B88B9C01AD01C7017F
:10495000B6010E94D18F882359F1A70196016D8578
:104960007E858F8598890E94D58F0E94C2916D8720
:104970007E878F87988BA301920169897A898B89B9
:104980009C890E940A8FA50194010E94D58F2D85D4
:104990003E854F8558890E9435920E9442909B0126
:1049A000AC01C701B6010E9435926B017C0103C0C6
:1049B000C12CD12C760169ED7BE0CE0101960E94DD
:1049C000DD8B4AE050E060E070E0CE0101960E948D
:1049D000B509CE0101960E94F38A20E030E64AEE46
:1049E00056E4C701B6010E94769118163CF466E9B8
:1049F00075E08FED9BE00E94FB8B44C00115110513
:104A0000B9F421E0B701A601CE0107960E94808C7F
:104A100065EA75E0CE0101960E945E8BBE01695F7A
:104A20007F4FCE0101960E94578D69EA75E01BC049
:104A30000230110539F522E049895A896B897C8950
:104A4000CE0107960E94808C65EA75E0CE01019642
:104A50000E945E8BBE01695F7F4FCE0101960E946E
:104A6000578D6DEA75E00E94688DBC018FED9BE06B
:104A70000E94C88BCE0101960E94F38ACE01079650
:104A80000E94F38A6FED7BE0CE0101960E94DD8BE0
:104A90004AE050E06FEF7FEFCE0101960E94290BB4
:104AA000CE0101960E94F38A64E670E080E090E017
:104AB0000E94D7818091D00B882331F060E273E0AF
:104AC00080E090E00E94D78164960FB6F894DEBF34
:104AD0000FBECDBFDF91CF911F910F91FF90EF904F
:104AE000DF90CF90BF90AF909F908F907F906F900E
:104AF0005F904F9008954F925F926F927F928F9246
:104B00009F92AF92BF92CF92DF92EF92FF92CF939C
:104B1000C82F8091920A81110DC00E94A8816093D4
:104B2000860A7093870A8093880A9093890A81E0A5
:104B30008093920A80918A0A81110DC00E94A881F7
:104B40006093820A7093830A8093840A9093850A03
:104B500081E080938A0A1092660B1092650BE090B8
:104B6000650BF090660B88E2E816F1040CF08AC041
:104B70008C2F0E946D82F701EE0FFF1FE959F44F51
:104B80009183808368E270E087E69BE00E94DB0708
:104B900020E030E040EA50E40E94359220E030E02E
:104BA00040E85AE30E9435926B017C0160937E0AD3
:104BB00070937F0A8093800A9093810A40902A0222
:104BC00050902B0260902C0270902D02A301920154
:104BD000609126027091270280912802909129020B
:104BE0000E940A8F9B01AC0160E070E080EC90E4D1
:104BF0000E940A8F4B015C0120E030E0A9010E9475
:104C0000D18F20E030E040E650E4811105C0C701BB
:104C1000B6010E9435921EC0C701B6010E943592AE
:104C2000A30192010E940B8F20E030E040E850E4A5
:104C30000E940A8FA50194010E94D58F20E030E0E8
:104C400040EC50E40E94359220E030E040E850E42F
:104C50000E940B8F60937A0A70937B0A80937C0A80
:104C600090937D0A64E170E080E090E00E94D7813B
:104C70008091650B9091660B01969093660B8093E3
:104C8000650B6DCF60917A0A70917B0A80917C0AE6
:104C900090917D0ACF91FF90EF90DF90CF90BF90E1
:104CA000AF909F908F907F906F905F904F900895FE
:104CB000CF92DF92EF92FF92CF93DF93CDB7DEB723
:104CC0002C970FB6F894DEBF0FBECDBF6CE972E033
:104CD00089ED9BE00E94DC8C69ED7BE0CE010196C2
:104CE0000E94DD8B4AE050E060E070E0CE0101966A
:104CF0000E94B509CE0101960E94F38A809181023B
:104D000090918202F8DE6B017C0120E030E0A90185
:104D10000E94769187FD22C022E0B701A601CE0154
:104D200007960E94808C6FEA75E0CE0101960E9482
:104D30005E8BBE01695F7F4FCE0101960E94578D49
:104D4000BC018FED9BE00E94C88BCE0101960E94B2
:104D5000F38ACE0107960E94F38A06C063EB75E0E2
:104D60008FED9BE00E94FB8B6FED7BE0CE01019607
:104D70000E94DD8B4AE050E06FEF7FEFCE0101969D
:104D80000E94290BCE0101960E94F38A2C960FB641
:104D9000F894DEBF0FBECDBFDF91CF91FF90EF90B3
:104DA000DF90CF9008952F923F924F925F926F9233
:104DB0007F928F929F92AF92BF92CF92DF92EF92AB
:104DC000FF920F931F93CF93DF9300D01F92CDB725
:104DD000DEB76B017C015A8349835901FA012081B6
:104DE0003181428153810E94D18F181614F0F50150
:104DF00083C010E00150104C000F111F000F111F55
:104E0000E981FA81E00FF11F2081318142815381D4
:104E1000C701B6010E94769187FF6BC011E0612E39
:104E2000712C4301880C991C880C991CE981FA812A
:104E3000E80DF91D2080318042805380A20191014C
:104E4000C701B6010E947691181614F41F5FE7CFD0
:104E5000A2019101C701B6010E94D18F8501080D01
:104E6000191D811102C0F80147C0C3018150904C47
:104E7000880F991F880F991FA981BA81A80FB91FA0
:104E80002D913D914D915C9129833A834B835C83B5
:104E9000F501E80FF91F80809180A280B380C701DF
:104EA000B6010E940A8F6B017C01A5019401F801F3
:104EB00060817181828193810E940A8F9B01AC0184
:104EC000C701B6010E9435926B017C0129813A81AC
:104ED0004B815C81C201B1010E940A8F9B01AC0130
:104EE000C701B6010E94D58FA50194010E940B8FC6
:104EF00007C0F501E00FF11F60817181828193810C
:104F00000F900F900F900F90DF91CF911F910F9105
:104F1000FF90EF90DF90CF90BF90AF909F908F90D9
:104F20007F906F905F904F903F902F900895CF9219
:104F3000DF92EF92FF921F93CF93DF93182FCAE077
:104F4000D0E0C12CD12C7601812F0E946D82BC0152
:104F5000882777FD8095982F0E94A1909B01AC0136
:104F6000C701B6010E940B8F6B017C0162E370E008
:104F700080E090E00E94D781219731F720E030E077
:104F800040E251E4C701B6010E94D58F20E030E035
:104F900040EA50E40E94359220E030E040E85AE3D5
:104FA0000E943592DF91CF911F91FF90EF90DF909B
:104FB000CF9008952F923F924F925F926F927F927F
:104FC0008F929F92AF92BF92CF92DF92EF92FF9219
:104FD0000F931F93CF93DF93CDB7DEB73A0118013C
:104FE0002901A50194010E94D58F4B015C0120E0AD
:104FF00030E040EC5FE3C201B1010E9435929B01B9
:10500000AC01C501B4010E947691181694F120E01C
:1050100030E040E05FE3C701B6010E9435929B019A
:10502000AC01C501B4010E94D18F87FD22C0F301FC
:105030002481358146815781C501B4010E940A8FC0
:10504000F30120853185428553850E94D58FF30178
:1050500020813181428153810E940B8F9B01AC01E1
:1050600060E070E080E291E40E9498920E946E906D
:1050700003C06FEF7FEFCB01DF91CF911F910F91B5
:10508000FF90EF90DF90CF90BF90AF909F908F9068
:105090007F906F905F904F903F902F9008954F9228
:1050A0005F926F927F928F929F92AF92BF92CF92B8
:1050B000DF92EF92FF920F931F93CF93DF93CDB7C1
:1050C000DEB7A0970FB6F894DEBF0FBECDBF2FDFBF
:1050D000698F7A8F8B8F9C8F40904502509046024B
:1050E0006090470270904802C0904102D090420206
:1050F000E0904302F09044028090490290904A026E
:10510000A0904B02B0904C0289829A82AB82BC8202
:105110004D825E826F827886A7019601C301B2013B
:105120000E940A8F6D8F7E8F8F8F98A320913D02F2
:1051300030913E0240913F0250914002C501B401BE
:105140000E940A8F9B01AC016D8D7E8D8F8D98A181
:105150000E94D58F69877A878B879C87812C912CB9
:1051600078E0A72E71E4B72E93018201AE014F5F64
:105170005F4F698D7A8D8B8D9C8D1CDF6B017C015F
:105180000E94040C63E972E089ED9BE00E94DC8CD4
:1051900069ED7BE0CE010D960E94DD8B42E350E08D
:1051A00060E070E0CE010D960E94B509CE010D962B
:1051B0000E94F38A2AE0B701A601CE0143960E941D
:1051C000548C62EC75E0CE010D960E945E8BBE01A0
:1051D0006D5E7F4FCE010D960E94578D67EC75E096
:1051E0000E94688DBC018FED9BE00E94C88BCE01B0
:1051F0000D960E94F38ACE0143960E94F38A6FEDCA
:105200007BE0CE010D960E94DD8B42E350E06FEF14
:105210007FEFCE010D960E94290BCE010D960E94C4
:10522000F38A8091D00B882331F060E273E080E054
:1052300090E00E94D781A0960FB6F894DEBF0FBE13
:10524000CDBFDF91CF911F910F91FF90EF90DF9035
:10525000CF90BF90AF909F908F907F906F905F9016
:105260004F900895FC0120E030E0772767FD7095AE
:10527000AB0142505109DF01A81BB90BA417B507B8
:1052800024F4A1912A0F311DF6CFA9014E5B5F4F87
:10529000860F971FFC013297208130E0322F2227A2
:1052A00031968081280F311D81E04217530709F0A4
:1052B00080E008952F923F924F925F926F927F927B
:1052C0008F929F92AF92BF92CF92DF92EF92FF9216
:1052D0000F931F93CF93DF93CDB7DEB763970FB6CE
:1052E000F894DEBF0FBECDBF8B8B60E00E94E682DC
:1052F0008091D00B811105C08FE090E0A0E0B0E07C
:1053000004C082E090E0A0E0B0E08F87988BA98B8A
:10531000BA8B67ED75E08FED9BE00E94FB8B6FED24
:105320007BE0CE0101960E94DD8B4AE050E06FEFFA
:105330007FEFCE0101960E94B509CE0101960E9431
:10534000F38AC12CD12C7601312C1D861E86212C8E
:1053500002E310E0412C512C32018B890E946D82B6
:10536000AA2797FDA095BA2F480E591E6A1E7B1ECC
:1053700065E070E080E090E00E94D7810150110963
:1053800061F78090120290901302A0901402B090E6
:105390001502C301B2010E94A19020E030E040EA72
:1053A00050E40E94359220E030E040E85AE30E9449
:1053B000359220E030E048E452E40E94D58FA50108
:1053C00094010E940A8F20E030E040E751E40E94FF
:1053D00035922B013C01A50194016AE979E989E341
:1053E00090E40E940A8F9B01AC01C301B2010E94AC
:1053F000D58F20E030E0A9010E940B8F20E030E043
:1054000040E251E40E9435925B018C01232D3D85E1
:105410004E85522D0E947691181624F43A2CBD86A2
:105420000E87212E20E030E0A901B501C8010E94BD
:10543000D18F87FF04C0A12CB12C00E010E022E046
:10544000A501B801CE0107960E94808CBE01695F5C
:105450007F4FCE0101960E94DD8B64EE75E0CE0198
:1054600001960E94688DBC0189ED9BE00E94C88B6B
:10547000CE0101960E94F38ACE0107960E94F38A1C
:1054800069ED7BE0CE0101960E94DD8B4AE050E0A1
:1054900060E070E0CE0101960E94290BCE010196DA
:1054A0000E94F38A0E94A88180908C0490908D04C1
:1054B000A0908E04B0908F040091E10C1091E20C4A
:1054C0002091E30C3091E40C800E911EA21EB31EBD
:1054D00086169706A806B90608F4DEC00E94A881C1
:1054E0000E949F904B015C0160918C0470918D042F
:1054F00080918E0490918F040E94A19020E030E072
:1055000040E85EE30E9435922B013C016091E10C82
:105510007091E20C8091E30C9091E40C0E94A190B8
:105520009B01AC01C301B2010E940B8F9B01AC0136
:10553000C501B4010E94D18F87FDAEC06CE370E05D
:1055400080E090E00E94D7819FEFC91AD90AE90A4A
:10555000F90A8F859889A989BA898C159D05AE05A8
:10556000BF050CF0F5CE64E670E080E090E00E94AC
:10557000D7810E94040C64E670E080E090E00E9415
:10558000D78169EE75E089ED9BE00E94FB8B69EDA8
:105590007BE0CE0101960E94DD8B44E150E060E0AB
:1055A00070E0CE0101960E94B509CE0101960E94DD
:1055B000F38A22E0432D5D856E85722DCE0107961C
:1055C0000E94808CBE01695F7F4FCE0101960E94D0
:1055D000DD8B64EE75E0CE0101960E94688DBC0102
:1055E00089ED9BE00E94C88BCE0101960E94F38A50
:1055F000CE0107960E94F38A69ED7BE0CE01019609
:105600000E94DD8B42E350E06FEF7FEFCE01019609
:105610000E94290BCE0101960E94F38A0E94BE0BC4
:1056200062E370E080E090E00E94D78161EF75E076
:10563000CE0101960E945E8B69ED7BE0CE01019662
:105640000E94578D65EF75E00E94688D6FED7BE0DD
:105650000E94578DBC018FED9BE00E94C88BCE014C
:1056600001960E94F38A63960FB6F894DEBF0FBED0
:10567000CDBFDF91CF911F910F91FF90EF90DF9001
:10568000CF90BF90AF909F908F907F906F905F90E2
:105690004F903F902F9008950E94BE0B4FCFFF92E6
:1056A0000F931F93CF93DF93F82E0AE010E0C0E032
:1056B000D0E08F2D0E946D82C80FD91F65E070E089
:1056C00080E090E00E94D7810150110991F7CE014E
:1056D0006AE070E00E945193CB01DF91CF911F915E
:1056E0000F91FF9008950F931F93CF93DF93CDB742
:1056F000DEB72E970FB6F894DEBF0FBECDBF8D87F5
:105700009E870E94040C8D859E85C9DF8C0162E313
:1057100070E080E090E00E94D781B801882777FD93
:105720008095982F0E94A19020E030E040EA50E45C
:105730000E94359220E030EC4FE754E40E94D58F70
:10574000AB01BC0123E0CE0107960E94808C62EF82
:1057500075E0CE0101960E945E8BBE01695F7F4FAE
:10576000CE0101960E94578D6BEF75E00E94688D07
:10577000BC018FED9BE00E94C88BCE0101960E9478
:10578000F38ACE0107960E94F38A6EEF75E089EDE9
:105790009BE00E94FB8B69ED7BE0CE0101960E94AD
:1057A000DD8B4AE050E068E070E0CE0101960E9497
:1057B000B509CE0101960E94F38A6FED7BE0CE0120
:1057C00001960E94DD8B4AE050E06FEF7FEFCE0143
:1057D00001960E94290BCE0101960E94F38A69ED81
:1057E0007BE08FED9BE00E942F8D8091D00B882372
:1057F00031F060E273E080E090E00E94D7812E9665
:105800000FB6F894DEBF0FBECDBFDF91CF911F91D1
:105810000F910895CF93DF93CDB7DEB72C970FB6D6
:10582000F894DEBF0FBECDBF3ADF9093CC0B8093D0
:10583000CB0B62E370E080E090E00E94D781609142
:10584000CB0B7091CC0B4AE0CE0101960E94298CC3
:10585000BE016F5F7F4F8FED9BE00E94E58BCE0115
:1058600001960E94F38A8091410C9091420C892B01
:1058700009F45FC06DE37CE0CE0107960E94DD8BEA
:10588000BE01695F7F4FCE0101960E94DD8B44E12E
:1058900050E060E070E0CE0101960E94B509CE01B3
:1058A00001960E94F38A66E076E0CE0101960E949E
:1058B0005E8B6FED7BE0CE0101960E94578DBC019F
:1058C00089ED9BE00E94C88BCE0101960E94F38A6D
:1058D00069ED7BE0CE0101960E94DD8B44E150E052
:1058E0006FEF7FEFCE0101960E94290BCE0101964A
:1058F0000E94F38ABE01695F7F4FCE0101960E942C
:10590000DD8B66EC74E0CE0101960E94688D69ED36
:105910007BE00E94578DBC018FED9BE00E94C88BFD
:10592000CE0101960E94F38ACE0107960E94F38A67
:1059300054C061E176E089ED9BE00E94FB8B69ED4C
:105940007BE0CE0101960E94DD8B44E150E060E0F7
:1059500070E0CE0101960E94B509CE0101960E9429
:10596000F38A65E176E0CE0101960E945E8B6FEDD1
:105970007BE0CE0101960E94578DBC0189ED9BE032
:105980000E94C88BCE0101960E94F38A69ED7BE0EC
:10599000CE0101960E94DD8B44E150E06FEF7FEF76
:1059A000CE0101960E94290BCE0101960E94F38A36
:1059B00066E076E0CE0101960E945E8B6FED7BE0A3
:1059C000CE0101960E94578DBC018FED9BE00E9495
:1059D000C88BCE0101960E94F38A8091D00B882358
:1059E00031F060E273E080E090E00E94D7812C9675
:1059F0000FB6F894DEBF0FBECDBFDF91CF910895F3
:105A00000F931F93CF93DF93CDB7DEB72C970FB6CD
:105A1000F894DEBF0FBECDBF8C0181E00E946A8288
:105A200064E670E080E090E00E94D7810E94040C60
:105A3000C80135DE60E074E0681B790B4AE0CE01F6
:105A400007960E94298C65E176E0CE0101960E94BE
:105A50005E8BBE01695F7F4FCE0101960E94578D1C
:105A6000BC018FED9BE00E94C88BCE0101960E9485
:105A7000F38ACE0107960E94F38A40E066E089EE41
:105A80009CE00E94C65E65ED76E0CE0101960E9424
:105A9000FC8C42E350E068E070E0CE0101960E9489
:105AA000B509CE0101960E94F38A6FED7BE0CE012D
:105AB00001960E94DD8B42E350E06FEF7FEFCE0155
:105AC00001960E94290BCE0101960E94F38A6CE197
:105AD00076E0CE0101960E945E8B6FED7BE0CE01F9
:105AE00001960E94578DBC018FED9BE00E94C88BF0
:105AF000CE0101960E94F38A8091D00B882331F069
:105B000060E273E080E090E00E94D7812C960FB6AF
:105B1000F894DEBF0FBECDBFDF91CF911F910F91E3
:105B200008950F9390E0BBDDBC01882777FD809539
:105B3000982F0E94A1902DE038E643E55BE30E9498
:105B4000359206E021E532E049E652E02CD920E02A
:105B500030E048EC52E40E94359220E030E048EA20
:105B600051E40E94359220914D0230914E024091B5
:105B70004F02509150020E94D58F0F910895CF92FD
:105B8000DF92EF92FF92CF93DF93CDB7DEB72C97E2
:105B90000FB6F894DEBF0FBECDBFC3DF6B017C0133
:105BA0006BE872E089ED9BE00E94DC8C69ED7BE0A4
:105BB000CE0101960E94DD8B42E350E060E070E090
:105BC000CE0101960E94B509CE0101960E94F38A8A
:105BD00022E0B701A601CE0107960E94808C63ECFB
:105BE00075E0CE0101960E945E8BBE01695F7F4F1A
:105BF000CE0101960E94578D66E276E00E94688D84
:105C0000BC018FED9BE00E94C88BCE0101960E94E3
:105C1000F38ACE0107960E94F38A6FED7BE0CE01F6
:105C200001960E94DD8B42E350E06FEF7FEFCE01E3
:105C300001960E94290BCE0101960E94F38A809161
:105C4000D00B882331F060E273E080E090E00E94A6
:105C5000D7812C960FB6F894DEBF0FBECDBFDF9173
:105C6000CF91FF90EF90DF90CF900895CF92DF9289
:105C7000EF92FF920F9390E012DDBC01882777FD31
:105C80008095982F0E94A1902DE038E643E55BE3D4
:105C90000E94359206E021E532E049E652E083D8E1
:105CA00020E030E048EC52E40E9435926B017C0128
:105CB00020E030E0A9010E94D18F181634F0C12CE9
:105CC000D12C48EAE42E41E4F42EC0924D02D09249
:105CD0004E02E0924F02F09250020F91FF90EF902F
:105CE000DF90CF9008959F92AF92BF92CF92DF92B4
:105CF000EF92FF920F931F93CF93DF935C01C0E568
:105D0000D4E00EE314E057EFE52E5AE0F52ECC2454
:105D1000C394D12C75E1972E80913C0490913D0461
:105D20008C159D050CF49DC081E0A816B10429F4E2
:105D3000F70180819181F80108C0F2E0AF16B1044B
:105D400031F4F80180819181F70191838083F8011A
:105D500080819181009739F48881998190936104C1
:105D60008093600422C08130910539F48881998143
:105D700090936F0480936E0418C08230910539F4BB
:105D80008881998190936D0480936C040EC0039771
:105D900061F48881998190936304809362046CE636
:105DA0007AE08DE39CE00E94FB8BF8012191319118
:105DB0008F012430310539F48881998190938202D2
:105DC0008093810228C02530310539F4888199817A
:105DD00090936B0480936A041EC02630310539F419
:105DE0008881998190936704809366041EC0273050
:105DF000310539F488819981909365048093640416
:105E000028C02A30310539F488819981909369043A
:105E1000809368041EC02531310539F48881998149
:105E2000909371048093700414C02B3031058CF072
:105E3000888199819093630480936204929EB0015B
:105E4000939E700D11246D577D4F8DE39CE00E9451
:105E5000FB8BFFEFCF1ADF0A229682E0E80EF11CDF
:105E60005BCFDF91CF911F910F91FF90EF90DF906B
:105E7000CF90BF90AF909F90089581E08093980459
:105E800089EE9CE00C94025F89EE9CE00E94FC5E2F
:105E9000109298040895CF93DF9300D000D0CDB72F
:105EA000DEB780919904811141C061E080919A042C
:105EB0000E941F83E091E90CF091EA0C0480F581C7
:105EC000E02D20E042E060E189EE9CE0199540E998
:105ED00054E060E089EE9CE00E94825F81E0809364
:105EE00099046FE472E0CE0101960E94FC8C4AE0B6
:105EF00050E060E070E0CE0101960E94B509CE014D
:105F000001960E94F38A63E472E0CE0101960E943A
:105F1000FC8C4AE050E060E070E0CE0101960E9407
:105F2000290BCE0101960E94F38A0DC0809198043E
:105F3000882349F0A9DF60E080919A040E941F83C2
:105F40001092990401C099DF26960FB6F894DEBF2F
:105F50000FBECDBFDF91CF9108954F925F926F92A8
:105F60007F92AF92BF92CF92DF92EF92FF920F9308
:105F70001F93CF93DF93CDB7DEB7EA970FB6F894B0
:105F8000DEBF0FBECDBF182F6CE67AE0CE01C596FE
:105F90000E945E8B612FCE0145960E94A066BE01D5
:105FA0006B5E7F4FCE0101960E94BA7DCE010196B5
:105FB0000E94177FCE0101960E94A8806CE0CE015E
:105FC00001960E940780CE0101960E94C37D082F92
:105FD00010E00330110509F453C16BE276E0CE0105
:105FE000C5960E94FB8B6CE67AE08FED9BE00E94E9
:105FF000FB8BBE016B5C7F4FCE0183960E94DD8BD5
:106000004AE050E060E070E0CE0183960E94B5095E
:10601000CE0183960E94F38A41E060E089EE9CE025
:106020000E94C65E6FE476E0CE01C5960E94FB8BAF
:10603000EBE3AE2EEBE0BE2ECC24C394D12CE12CAE
:10604000F12CE016F1060CF0E1C06E2DCE010196A8
:106050000E943581F50121913191419151915F016A
:106060000E940B8F2B013C0120E030E04CEF52EC02
:106070000E94D18F87FF25C04AE0B601CE018996E4
:106080000E94298C6BE677E0CE0183960E945E8B9E
:10609000BE01675D7F4FCE0183960E94578D65E3F9
:1060A00076E00E94688DBC018FED9BE00E942F8DF1
:1060B000CE0183960E94F38ACE0189960E94F38ACC
:1060C00049C022E0B301A201CE0183960E94808CD8
:1060D0004AE0B601CE018F960E94298C6BE677E0EC
:1060E000CE0189960E945E8BBE01615D7F4FCE011D
:1060F00089960E94578D63E178E00E94688DBE0109
:106100006D5D7F4F0E94578DBC0183ED9BE00E9427
:10611000C88BCE0189960E94F38ACE018F960E9489
:10612000F38ACE0183960E94F38A63ED7BE0CE0171
:1061300083960E94DD8B66EC74E0CE0183960E940C
:10614000688DBC018FED9BE00E942F8DCE01839660
:106150000E94F38A0130110559F4E114F10409F0A9
:106160004EC06FED7BE0CE01C5960E94C88B47C044
:106170000230110511F522E0B301A201CE0189968A
:106180000E94808CBE01675D7F4FCE0183960E9486
:10619000DD8B66EC74E0CE0183960E94688DBC01B5
:1061A000CE01C5960E942F8DCE0183960E94F38A60
:1061B000CE0189960E94F38A22C063ED7BE0CE0176
:1061C00083960E94DD8B44E150E06FEF7FEFCE01BC
:1061D00083960E94290BCE0183960E94F38A0E9427
:1061E000D20B80919904882351F0809198048823E0
:1061F00031F060ED77E080E090E00E94D781FFEF22
:10620000EF1AFF0A8FEFC81AD80A1BCFCE01C59626
:106210000E94888E01151105C9F460E372E08FEDCC
:106220009BE00E94DC8C61E476E0CE0183960E94C4
:106230005E8B4AE050E06FEF7FEFCE0183960E94C5
:10624000290BCE0183960E94F38AD6C00430110533
:106250000CF0EBC0BE016B5C7F4FCE0183960E94B9
:10626000DD8B4AE050E06FEF7FEFCE0183960E9416
:10627000290BCE0183960E94F38A0E94D20BD5C0CF
:106280006CE476E0CE01C5960E94FB8BBE016B5C90
:106290007F4FCE0183960E94DD8B4AE050E060E0A4
:1062A00070E0CE0183960E94B509CE0183960E94CC
:1062B000F38A6CE67AE08FED9BE00E94FB8B6FED3A
:1062C0007BE0CE01C5960E94C88B00E010E0602FF5
:1062D000CE0101960E9435816B017C0122E0AB0169
:1062E000BC01CE010115110569F483960E94808CD2
:1062F000BE016D5D7F4F89EE9CE00E949B87CE01C1
:1063000083961BC089960E94808CBE01675D7F4F7B
:10631000CE0183960E94DD8B66EC74E0CE018396FD
:106320000E94688DBC01CE01C5960E942F8DCE01C2
:1063300083960E94F38ACE0189960E94F38A22E016
:10634000B701A601CE0189960E94808CBE01675DCF
:106350007F4FCE0183960E94DD8B66EC74E0CE0108
:1063600083960E94688DBC018FED9BE00E942F8D6B
:10637000CE0183960E94F38ACE0189960E94F38A09
:106380000F5F1F4F0330110509F0A1CFCE01C59655
:106390000E94888EBE016B5C7F4FCE0183960E9467
:1063A000DD8B4AE050E06FEF7FEFCE0183960E94D5
:1063B000290BCE0183960E94F38A0E94D20B8FEDA7
:1063C0009BE00E94888E62E576E0CE0183960E9473
:1063D0005E8B6FED7BE0CE0183960E94578D6CE55E
:1063E00076E00E94688DBC018FED9BE00E94C88B17
:1063F000CE0183960E94F38ACE01C5960E94F38A4D
:10640000EA960FB6F894DEBF0FBECDBFDF91CF91F5
:106410001F910F91FF90EF90DF90CF90BF90AF90C2
:106420007F906F905F904F9008956CE576E08FEDD0
:106430009BE00E94358DE0CF8F929F92AF92BF92EA
:10644000CF92DF92EF92FF920F931F93CF93DF9340
:10645000CDB7DEB7A2970FB6F894DEBF0FBECDBFA3
:106460005C016A017B01122F6CE172E08EE99EE013
:106470000E9478874AE050E0B5018EE99EE00E94D4
:10648000938866EC74E08EE99EE00E94A98722E082
:1064900030E0B701A6018EE99EE00E94CD89612F10
:1064A000CE0145960E94A066BE016B5E7F4FCE0175
:1064B00001960E94BA7DCE0101960E94177FCE01FF
:1064C00001960E94A8806CE0CE0101960E94078090
:1064D000CE0101960E94C37D082F10E00B301105FC
:1064E00014F00AE010E08BE5A816B10408F44FC0E0
:1064F0009BE3892E9BE0992EC12CD12C7601A12CF7
:10650000B12CA016B106BCF46A2DCE0101960E94F2
:1065100035819B01AC01F401619371938193919357
:106520004F01C701B6010E940B8F6B017C01FFEF89
:10653000AF1ABF0AE6CFB801882777FD8095982F5C
:106540000E94A1909B01AC01C701B6010E94D58FAA
:106550006B017C018BE3882E8BE0982EA12CB12C53
:10656000A016B1060CF052C0F401208131814281A5
:106570005381C701B6010E940A8FF40161937193A0
:10658000819391934F01FFEFAF1ABF0AE9CFA11496
:10659000B10439F4BBE38B2EBBE09B2EA12CB12CB4
:1065A0001DC00A151B050CF0850101501109602F53
:1065B000CE0101960E9435819B01AC01000F111F95
:1065C000000F111F055C144FC701B6010E940A8F0E
:1065D000F801608371838283938318C0A016B1068B
:1065E000ACF46A2DCE0101960E9435819B01AC016D
:1065F000C701B6010E940A8FF401619371938193E0
:1066000091934F01FFEFAF1ABF0AE8CFA2960FB6E2
:10661000F894DEBF0FBECDBFDF91CF911F910F91D8
:10662000FF90EF90DF90CF90BF90AF909F908F90B2
:10663000089560E08DE30E941F8382E090E00E9455
:10664000FD8161E08DE30E941F838AE090E00E945B
:10665000FD8160E08DE30E941F8320E432E44FE07F
:1066600050E061E08EE30E947C830E949F9020E0D6
:1066700030E048EC52E40E94D58F2091D10C30914B
:10668000D20C4091D30C5091D40C0E94359220E052
:1066900030E44CE156E40E94D58F20E030E040E049
:1066A0005FE30C9435920895CF92DF92EF92FF92C0
:1066B000C0DF6B017C0120E030E040E050E40E944C
:1066C000769118161CF4B5DF6B017C0120E030E0F8
:1066D00040E050E4C701B6010E94769118161CF400
:1066E000A8DF6B017C0120E030E040E050E4C7010E
:1066F000B6010E94769118161CF49BDF6B017C0199
:1067000020E030E040E050E4C701B6010E947691FD
:1067100018162CF4FF90EF90DF90CF908ACFC7012E
:10672000B601FF90EF90DF90CF9008954F925F9267
:106730006F927F928F929F92AF92BF92CF92DF9291
:10674000EF92FF92CF93DF9300D01F92CDB7DEB7C9
:10675000ABDF9B01AC0169833A834B835C830E946E
:10676000B4812B013C016EE170E080E090E00E947A
:10677000D7819ADF6B017C010E94B4814B015C01DF
:1067800084189508A608B70829813A814B815C8155
:1067900081ED881687E09806A104B1040CF43DC091
:1067A000C701B6010E940A8F6B017C0120E030E036
:1067B000A9010E94769118165CF426EA3BE944ECA4
:1067C0005BE3C701B6010E94D18F87FF0BC025C0D4
:1067D00026EA3BE944EC5BEBC701B6010E947691E7
:1067E0001816DCF0C501B40128EE33E040E050E0BB
:1067F0000E949A93CA01B9010E94A1904B015C01C9
:1068000020E030E04AE754E4C701B6010E94359227
:10681000A50194010E94D58F03C060E070E0CB0118
:106820000F900F900F900F90DF91CF91FF90EF900E
:10683000DF90CF90BF90AF909F908F907F906F90A0
:106840005F904F90089523E333E948E853E40E94B2
:10685000D58F20E030E040E85FE30E940B8F0E947C
:10686000E89226E636EA45EA53E40E9435926093C0
:10687000D10C7093D20C8093D30C9093D40C0895C8
:106880004F925F926F927F928F929F92AF92BF9240
:10689000CF92DF92EF92FF92CF93DF93CDB7DEB727
:1068A0006C970FB6F894DEBF0FBECDBF6B017C01B5
:1068B0000E94A8816D8B7E8B8F8B988F61E08DE31A
:1068C0000E94E68260E08EE30E94E6828BEF9BE00E
:1068D0000E9416626093CD0C7093CE0C8093CF0C07
:1068E0009093D00CB0DFE0DE6D877E878F87988B2A
:1068F0000E94B481698B7A8B8B8B9C8B6AE070E0F1
:1069000080E090E00E94D7816EEF71E08FED9BE018
:106910000E94DC8C20E030E04AE754E4C701B60175
:106920000E943592698F7A8F8B8F9C8F412C512CCE
:106930003201C12CD12C7601C701B6010E94A19071
:10694000298D3A8D4B8D5C8D0E94D18F87FF87C139
:106950000E94A8812D893E894F89588D621B730B37
:10696000840B950B0E949F9020E030E04AE754E4AE
:106970000E94D58FAB01BC0123E0CE0101960E949D
:10698000808CBE016F5F7F4F89ED9BE00E94E58B9D
:10699000CE0101960E94F38A87DE6B017C010E9482
:1069A000B4814B015C0189899A89AB89BC89881AB9
:1069B000990AAA0ABB0A91ED891697E09906A104E3
:1069C000B1040CF441C020E030E0A901C701B601D8
:1069D0000E94769118165CF426EA3BE944EC5BE3EE
:1069E000C701B6010E94D18F87FF0BC02DC026EAD8
:1069F0003BE944EC5BEBC701B6010E9476911816A7
:106A00001CF1C501B40128EE33E040E050E00E94E3
:106A10009A93CA01B9010E94A1904B015C012D8596
:106A20003E854F855889C701B6010E940A8F20E034
:106A300030E04AE754E40E943592A50194010E9497
:106A4000D58F4B015C0103C0812C912C540169ED61
:106A50007BE0CE0101960E94DD8B67E776E0CE01F8
:106A600001960E94688DBC0189ED9BE00E94C88B55
:106A7000CE0101960E94F38A23E0B701A601CE0160
:106A800007960E94808CBE01695F7F4FCE01019600
:106A90000E94DD8B6EE676E0CE0101960E94688D45
:106AA000BC0183ED9BE00E94C88BCE0101960E9441
:106AB000F38ACE0107960E94F38A22E0B501A40171
:106AC000CE0101960E94808C69EF74E0CE0107969A
:106AD0000E945E8B69ED7BE0CE0107960E94578D88
:106AE00061E776E00E94688D63ED7BE00E94578D40
:106AF00061E876E00E94688DBE016F5F7F4F0E9463
:106B0000578D65E776E00E94688DBC018FED9BE0B4
:106B10000E942F8DCE0107960E94F38ACE01019626
:106B20000E94F38A20E030E0A901C501B4010E946F
:106B3000769187FD06C066EC74E083ED9BE00E94D1
:106B4000358D22E0B501A401CE0107960E94808C0C
:106B5000BE01695F7F4FCE0101960E94DD8B65E724
:106B600076E0CE0101960E94688DBC0183ED9BE02A
:106B70000E942F8DCE0101960E94F38ACE010796C6
:106B80000E94F38A6FED7BE0CE0101960E94DD8BBF
:106B9000CE0101960E948B0FCE0101960E94F38ACE
:106BA000C301B20125E030E040E050E00E949A933A
:106BB000672B682B692B21F569E776E0CE010196FA
:106BC0000E945E8B45E050E060E070E0CE010196EF
:106BD0000E94B509CE0101960E94F38A63ED7BE025
:106BE000CE0101960E94DD8B45E050E06FEF7FEF14
:106BF000CE0101960E94290BCE0101960E94F38AD4
:106C00006CE67AE08FED9BE00E94FB8B65E070E024
:106C100080E090E00E94D7810E94A8816B017C01F6
:106C20002D893E894F89588DC21AD30AE40AF50A84
:106C30003BDD6D877E878F87988B0E94B481698B3F
:106C40007A8B8B8B9C8B6AE070E080E090E00E94F6
:106C5000D7813FEF431A530A630A730A6DCE60E08F
:106C60008DE30E94E6826C960FB6F894DEBF0FBEED
:106C7000CDBFDF91CF91FF90EF90DF90CF90BF908D
:106C8000AF909F908F907F906F905F904F900895FE
:106C9000CF93DF93CDB7DEB72C970FB6F894DEBF56
:106CA0000FBECDBF61E08DE30E94E68260E08EE31F
:106CB0000E94E6828BEF9BE00E9416626093CD0CEF
:106CC0007093CE0C8093CF0C9093D00CBCDDECDC99
:106CD000AB01BC0123E0CE0107960E94808CBE016F
:106CE000695F7F4FCE0101960E94DD8B67EE75E0F4
:106CF000CE0101960E94688DBC0189ED9BE00E9447
:106D0000C88BCE0101960E94F38ACE0107960E949D
:106D1000F38A62E776E0CE0101960E945E8B69ED10
:106D20007BE0CE0101960E94578DBC018FED9BE068
:106D30000E94C88BCE0101960E94F38AF7DCAB015A
:106D4000BC0122E0CE0107960E94808CBE01695FE3
:106D50007F4FCE0101960E94DD8B65E776E0CE0184
:106D600001960E94688DBC0183ED9BE00E94C88B58
:106D7000CE0101960E94F38ACE0107960E94F38A03
:106D800060E876E0CE0101960E945E8B63ED7BE0C9
:106D9000CE0101960E94578DBC018FED9BE00E94B1
:106DA0002F8DCE0101960E94F38A66EC74E0CE012D
:106DB00001960E945E8B63ED7BE0CE0101960E94FE
:106DC000578DBC0189ED9BE00E942F8DCE0101966D
:106DD0000E94F38A69E776E0CE0101960E945E8BFD
:106DE0004AE050E060E070E0CE0101960E94B509F3
:106DF000CE0101960E94F38A69ED7BE0CE010196F7
:106E00000E94DD8B45E050E06FEF7FEFCE010196F1
:106E10000E94290BCE0101960E94F38A64E876E075
:106E20008FED9BE00E94358D60E08DE30E94E6824D
:106E30002C960FB6F894DEBF0FBECDBFDF91CF9179
:106E400008958F929F92AF92BF92CF92DF92EF926E
:106E5000FF920F9322E0C22E33E0E32E04E025E000
:106E60004BE06CE089EE9CE00E94686067E976E0A8
:106E70008BED9CE00E945E8B6DE976E085ED9CE0F9
:106E80000E945E8B20E141E168E18AEC9CE00E9477
:106E9000736444E0E42E22E734E046E754E06AE716
:106EA00074E08BE59CE00E94816787E49CE00E948F
:106EB000C56C6CE67AE08DE39CE00E945E8B80916D
:106EC00066049091670490933C0C80933B0C8090F7
:106ED000450290904602A0904702B090480220914F
:106EE0004102309142024091430250914402C50157
:106EF000B4010E940A8F6B017C016093370C709380
:106F0000380C8093390C90933A0C6091490270913F
:106F10004A0280914B0290914C0260932B0C70932B
:106F20002C0C80932D0C90932E0C80922F0C909211
:106F3000300CA092310CB092320C20913D02309175
:106F40003E0240913F02509140020E940A8F9B01F5
:106F5000AC01C701B6010E94D58F6093330C7093CA
:106F6000340C8093350C9093360C4FEF5FEFBA01E1
:106F700082E19CE00E94D46A8BEF9BE00E940B614F
:106F80006CE67AE081EF9BE00E945E8B6CE67AE033
:106F90008BEE9BE00E945E8B6CE67AE085EE9BE0D8
:106FA0000E945E8B6CE67AE08FED9BE00E945E8B28
:106FB0006CE67AE089ED9BE00E945E8B6CE67AE0FD
:106FC00083ED9BE00E945E8B6091320270913302F0
:106FD0008CEB9AE00F91FF90EF90DF90CF90BF90F5
:106FE000AF909F908F900C94FE7283ED9BE00E9477
:106FF000F38A89ED9BE00E94F38A8FED9BE00E946B
:10700000F38A85EE9BE00E94F38A8BEE9BE00E9460
:10701000F38A81EF9BE00E94F38A80EF99E09093DE
:10702000130C8093120C8DE39CE00E94F38A85ED93
:107030009CE00E94F38A8BED9CE00C94F38A6F92A3
:107040007F928F929F92AF92BF92CF92DF92EF92F8
:10705000FF920F931F93CF93DF93CDB7DEB7E897DF
:107060000FB6F894DEBF0FBECDBF4B015C018BE3C2
:107070009FE00E94178564E670E080E090E00E9447
:10708000D78140E855E260E070E08BE39FE00E942A
:107090003E0964E670E080E090E00E94D7816FE7EF
:1070A00072E089ED9BE00E94DC8C69ED7BE0CE0113
:1070B00001960E94DD8B42E350E06FEF7FEFCE013F
:1070C00001960E94B509CE0101960E94F38A64E7F9
:1070D00072E089ED9BE00E94DC8C69ED7BE0CE01E3
:1070E00001960E94DD8B42E350E06FEF7FEFCE010F
:1070F00001960E94290BCE0101960E94F38A80918D
:10710000000D9091010D8D7F712CC12CD12CE12CA3
:10711000F12C00E010E0019709F459C0E2E46E2E72
:107120000E94A881681979098A099B09683B7B40FC
:107130008105910508F04BC08BE39FE00E94A88376
:10714000892BF1F14CED55E060E070E08BE39FE0BE
:107150000E940B8A68AE41E050E0BE01685C7F4F40
:107160008BE39FE00E94F28A882351F14FE150E0C7
:10717000BE016F5F7F4F8BE39FE00E94118A898180
:107180008D34F1F46FE1CE0101960E9432298823FB
:10719000B9F00C8110E0102F00278D81080F111D10
:1071A000EE80F12CFE2CEE248F81E80EF11CC884B9
:1071B000D12CDC2CCC248985C80ED11C7724739467
:1071C00062E370E080E090E00E94D781A9CF0E9446
:1071D000A881681979098A099B09683B7B40810568
:1071E000910510F47110C3C00E94040C69ED7BE09E
:1071F000CE0180960E94DD8B42E350E066E070E0B5
:10720000CE0180960E94B509CE0180960E94F38A35
:10721000772009F4D1C082E090E09093010D809333
:10722000000D4AE0B601CE0180960E94298C4AE00A
:10723000B701CE0186960E94298C4AE0B801CE01A2
:10724000C2960E94298CBE016E5C7F4FCE018C9647
:107250000E94DD8B67E279E0CE018C960E94688DFA
:10726000BE016A5D7F4F0E94578D67E279E00E9400
:10727000688DBE01605E7F4F0E94578DBC018FED0F
:107280009BE00E94C88BCE018C960E94F38ACE01AF
:10729000C2960E94F38ACE0186960E94F38ACE019E
:1072A00080960E94F38A6FED7BE0CE0180960E946B
:1072B000DD8B4AE050E06FEF7FEFCE0180960E94B9
:1072C000290BCE0180960E94F38A65EA76E089EE6A
:1072D0009CE00E94A9876BEA76E08FED9BE00E941C
:1072E000FB8B4AE0B601CE0180960E94298C4AE0D1
:1072F000B701CE0186960E94298C4AE0B801CE01E2
:10730000C2960E94298CBE016E5C7F4FCE018C9686
:107310000E94DD8B66EC74E0CE018C960E94688D35
:10732000BE016A5D7F4F0E94578D66EC74E00E943B
:10733000688DBE01605E7F4F0E94578D65EA76E0E2
:107340000E94688DBC018FED9BE00E942F8DCE01C5
:107350008C960E94F38ACE01C2960E94F38ACE01D7
:1073600086960E94F38ACE0180960E94F38A62E399
:1073700070E080E090E00E94D7818BE39FE00E9464
:10738000178562E370E080E090E00E94D781E89684
:107390000FB6F894DEBF0FBECDBFDF91CF911F9126
:1073A0000F91FF90EF90DF90CF90BF90AF909F90A4
:1073B0008F907F906F90089569E672E08FED9BE06B
:1073C0000E94DC8C6FED7BE0CE0180960E94DD8B0D
:1073D0004AE050E060E070E0CE0180960E94290B08
:1073E000CE0180960E94F38A66E572E08FED9BE005
:1073F0000E94DC8C8091000D9091010D029709F0A4
:10740000B6CF1092010D1092000DB1CF7F928F92E6
:107410009F92AF92BF92CF92DF92EF92FF920F9323
:107420001F93CF93DF9300D000D0CDB7DEB74C01D0
:107430008BE39FE00E94178540E052EC61E070E032
:107440008BE39FE00E943E094CED55E060E070E068
:107450008BE39FE00E940B8A64E670E080E090E09E
:107460000E94D781A12CB12C712CA814B9040CF066
:1074700051C065E070E080E090E00E94D78100E0BC
:1074800010E0C12CD12C760171100FC08BE39FE06E
:107490000E94A883892B31F485E1C816D104E10448
:1074A000F1041CF40330110554F08FEFA81AB80A48
:1074B00064E670E080E090E00E94D781D6CF8BE355
:1074C0009FE00E94A883892B69F08BE39FE00E94D4
:1074D000C183E1E0F0E0EC0FFD1FE00FF11F8083BE
:1074E0000F5F1F4F65E070E080E090E00E94D78161
:1074F000023011054CF089818B3B31F47724739471
:107500008A818A3A09F0712C8FEFC81AD80AE80AE2
:10751000F80ABACF872D26960FB6F894DEBF0FBEB5
:10752000CDBFDF91CF911F910F91FF90EF90DF9032
:10753000CF90BF90AF909F908F907F9008958F9243
:107540009F92AF92BF92CF92DF92EF92FF920F93F2
:107550001F93CF93DF93CDB7DEB72C970FB6F89478
:10756000DEBF0FBECDBF61E080919A040E94E6822B
:1075700061E080919A040E941F83E091E90CF091F0
:10758000EA0C0480F581E02D20E042E060E189EE24
:107590009CE0199540E954E060E089EE9CE00E948F
:1075A000825F0E943D2F8EED93E09093640B809359
:1075B000630B0E9448978093020D8FED93E00E9429
:1075C00048978093030D8091020D9091030D18163A
:1075D000190654F410929C04019731F41092030D93
:1075E0001092020D0E9491096BEB76E089EE9CE00F
:1075F0000E94A98740E855E260E070E08EE99EE0D5
:107600000E943E0940E855E260E070E088ED9FE0AE
:107610000E943E0964E670E080E090E00E94D7811D
:1076200080919C04882331F068EE73E080E090E064
:107630000E94D7818EE99EE00E94C183182F823775
:1076400009F42DC11092640B1092630B8DEBC82EC0
:107650008AE0D82EE12CF12CC7010E944897D60170
:107660008D936D01BFEFEB1AFB0AE6E7EE16F1040E
:1076700099F78091BD0A9091BE0AA091BF0AB0917E
:10768000C00A85369105A105B1050CF408C18093A7
:10769000380290933902A0933A02B0933B02809152
:1076A000C10A9091C20AA091C30AB091C40A809302
:1076B000340290933502A0933602B0933702809142
:1076C000C50A9091C60AA091C70AB091C80A8093D2
:1076D0002E0290932F02A0933002B093310269EDF5
:1076E0007AE0CE0101960E945E8BBE016F5F7F4FF4
:1076F0008BED9CE00E94E58BCE0101960E94F38AFF
:107700008091C90A9091CA0AA091CB0AB091CC0A83
:107710008093220290932302A0932402B093250227
:107720008091CD0A9091CE0AA091CF0AB091D00A53
:1077300080931E0290931F02A0932002B093210217
:107740008091D10A9091D20AA091D30AB091D40A23
:1077500080931A0290931B02A0931C02B0931D0207
:107760008091D50A9091D60AA091D70AB091D80AF3
:107770008093160290931702A0931802B0931902F7
:107780008091E10A9091E20AA091E30AB091E40AA3
:107790008093450290934602A0934702B09348021B
:1077A0008091E50A9091E60AA091E70AB091E80A73
:1077B0008093410290934202A0934302B09344020B
:1077C0008091E90A9091EA0AA091EB0AB091EC0A43
:1077D0008093490290934A02A0934B02B0934C02CB
:1077E0008091ED0A9091EE0AA091EF0AB091F00A13
:1077F00080933D0290933E02A0933F02B0934002DB
:107800008091F10A9091F20AA091F30AB091F40AE2
:1078100080934D0290934E02A0934F02B09350027A
:10782000C090070BD090080BE090090BF0900A0B6A
:10783000A7019601C701B6010E942993811108C0D2
:10784000C0921202D0921302E0921402F09215023A
:10785000BBE0AB2EBBE0BB2E0BE3802E0BE0902EEB
:10786000D501CD90DD90ED90FD905D01A7019601D1
:10787000C701B6010E942993811105C0F401C0829D
:10788000D182E282F382F4E08F0E911C83E3A8168A
:107890008BE0B80629F781E090E00E94732E0EE895
:1078A000010F023070F08091BD0A9091BE0AA09144
:1078B000BF0AB091C00A85369105A105B1050CF04B
:1078C00032C18091380290913902A0913A02B09170
:1078D0003B028093BD0A9093BE0AA093BF0AB09367
:1078E000C00A8091340290913502A0913602B09185
:1078F00037028093C10A9093C20AA093C30AB0933F
:10790000C40A80912E0290912F02A0913002B09172
:1079100031028093C50A9093C60AA093C70AB09318
:10792000C80A123751F420E030E048E050E069ED39
:107930007AE08BED9CE00E94C48D809122029091B0
:107940002302A0912402B09125028093C90A90934A
:10795000CA0AA093CB0AB093CC0A80911E029091E0
:107960001F02A0912002B09121028093CD0A909332
:10797000CE0AA093CF0AB093D00A80911A029091B8
:107980001B02A0911C02B0911D028093D10A90931A
:10799000D20AA093D30AB093D40A80911602909190
:1079A0001702A0911802B09119028093D50A909302
:1079B000D60AA093D70AB093D80A80914502909135
:1079C0004602A0914702B09148028093E10A909349
:1079D000E20AA093E30AB093E40A809141029091F5
:1079E0004202A0914302B09144028093E50A909331
:1079F000E60AA093E70AB093E80A809149029091C1
:107A00004A02A0914B02B0914C028093E90A9093F4
:107A1000EA0AA093EB0AB093EC0A80913D029091A0
:107A20003E02A0913F02B09140028093ED0A9093F4
:107A3000EE0AA093EF0AB093F00A80914D02909164
:107A40004E02A0914F02B09150028093F10A9093A0
:107A5000F20AA093F30AB093F40A80911202909173
:107A60001302A0911402B09115028093070B90931A
:107A7000080BA093090BB0930A0BEBE3FBE02BE0A0
:107A80003BE04191519161917191D9014D935D9389
:107A90006D937D939D01BBE0E336FB0791F765E1B4
:107AA0007CE08EE99EE00E94B487F5EFAF2EFAE00D
:107AB000BF2EACE3CA2EA4E0DA2EE12CF12C80918B
:107AC0003C0490913D048E159F051CF14601F60182
:107AD000819191916F01D5018D939D935D014AE054
:107AE00050E0B7018EE99EE00E9493886CEC76E04E
:107AF0008EE99EE00E94A987F401608171814AE0CD
:107B000050E08EE99EE00E949A88FFEFEF1AFF0A8C
:107B1000D6CF023040F41092640B1092630B80E0D9
:107B200090E00E94680964E670E080E090E00E94C6
:107B3000D7818CEB9AE00E94037361ED76E0CE0171
:107B400001960E945E8B4AE050E06FEF7FEFCE011E
:107B500001960E94B509CE0101960E94F38A66EA59
:107B600074E0CE0107960E945E8B6BED7CE0CE0147
:107B700007960E94578DBC01CE0101960E94DD8BB5
:107B80004AE050E06FEF7FEFCE0101960E94290B93
:107B9000CE0101960E94F38ACE0107960E94F38AD5
:107BA0006FEC76E0CE0107960E945E8B6BED7CE079
:107BB000CE0107960E94578D61EE76E00E94688D97
:107BC000BC01CE0101960E94DD8BCE0101960E9480
:107BD0008B0FCE0101960E94F38ACE0107960E9478
:107BE000F38A64E670E080E090E00E94D78184E050
:107BF0009DE00E94FB5B64E670E080E090E00E9404
:107C0000D78163E270E084E09DE00E940E5C61E059
:107C100070E084E09DE00E94410984E09DE00E94C4
:107C2000825C83E090E09093010D8093000D60E012
:107C300070E08AEC9CE00E946A656B017C0162E363
:107C400070E080E090E00E94D781A7019601C70113
:107C5000B6010E942993882309F465C060E070E0B2
:107C60008AEC9CE00E9468656B017C0162E370E035
:107C700080E090E00E94D781A7019601C701B6017C
:107C80000E942993882309F44EC081E090E09093EC
:107C9000010D8093000D40E052EC61E070E08BE359
:107CA0009FE00E943E0964E670E080E090E00E9460
:107CB000D78182E090E0AADB882339F06CEF7BE08B
:107CC0008EE99EE00E94B4872EC01092010D1092A2
:107CD000000D8BE39FE00E94178564E670E080E072
:107CE00090E00E94D78140E855E260E070E08BE3CD
:107CF0009FE00E943E098BE39FE00E94A883892BAE
:107D000091F062EE7BE08EE99EE00E94B48782E013
:107D100090E09093010D8093000D64E670E080E0A8
:107D200090E00E94D7818091000D9091010D039702
:107D300031F46DEC7BE08EE99EE00E94B48763E055
:107D40008BEF9BE00E94B861811111C067EA7BE074
:107D5000CE0101960E94FC8CCE0101960E948B0FF1
:107D6000CE0101960E94F38A10923C0293C063E90F
:107D70007BE08FED9BE00E94DC8C40E050E0BA019C
:107D80008BEF9BE00E94D8630E94A19020E030E03E
:107D900048EC52E40E94D58FAB01BC0122E0CE0139
:107DA00007960E94808CBE01695F7F4FCE010196CD
:107DB0000E94DD8B6EE878E0CE0101960E94688D0E
:107DC000BC018FED9BE00E942F8DCE0101960E9499
:107DD000F38ACE0107960E94F38A6FED7BE08EE96D
:107DE0009EE00E94C4876CE77BE08FED9BE00E94E1
:107DF000DC8C609138027091390280913A02909146
:107E00003B020E94A19020E030E048EC52E40E9446
:107E1000D58FAB01BC0122E0CE0107960E94808C79
:107E2000BE01695F7F4FCE0101960E94DD8B6EE837
:107E300078E0CE0101960E94688DBC018FED9BE039
:107E40000E942F8DCE0101960E94F38ACE010796E3
:107E50000E94F38A6FED7BE08EE99EE00E94C4876A
:107E6000113629F481E00E94511981E011C08EE998
:107E70009EE00E94C183182F64E670E080E090E0ED
:107E80000E94D781113671F380E00E94511980E081
:107E90000E94A10F64E670E080E090E00E94D7812C
:107EA00080919C04882331F068EE73E080E090E0DC
:107EB0000E94D7816DE477E08BEE9BE00E94FB8B04
:107EC00082E090E09093CE0B8093CD0B80919C0448
:107ED00081110E94A3172C960FB6F894DEBF0FBE37
:107EE000CDBFDF91CF911F910F91FF90EF90DF9069
:107EF000CF90BF90AF909F908F9008952F923F9218
:107F00004F925F926F927F928F929F92AF92BF92A9
:107F1000CF92DF92EF92FF920F931F93CF93DF9355
:107F2000CDB7DEB72B970FB6F894DEBF0FBECDBF2F
:107F30001C018BEB8F838AEA888781E0898784E63E
:107F4000829D9001839D300D11243B872A87E12C6F
:107F5000F12CC12CD12C812C912C5401C214D304AE
:107F600094F1C501B4010E94A19020E030E040E20C
:107F700051E40E94D58F6B017C01B101882777FD08
:107F80008095982F0E94A1909B01AC01C701B6017A
:107F90000E94D58F2B960FB6F894DEBF0FBECDBFD3
:107FA000DF91CF911F910F91FF90EF90DF90CF90D5
:107FB000BF90AF909F908F907F906F905F904F9009
:107FC0003F902F9008952A853B85E216F3064CF6E4
:107FD000C7016AE070E00E946593892B79F4E09113
:107FE0003B0FF0913C0F0280F381E02D43E050E025
:107FF000BE01695F7F4F8BE39FE0199565E070E0FC
:1080000080E090E00E94D7813FEFE31AF30A00E09E
:1080100010E0412C512C32018BE39FE00E94A88399
:10802000892B39F424E042165104610471040CF0E8
:1080300095CF063011050CF091CF8BE39FE00E94A5
:10804000A883892B69F08BE39FE00E94C183E1E064
:10805000F0E0EC0FFD1FE00FF11F80830F5F1F4F5B
:1080600065E070E080E090E00E94D7810630110565
:1080700001F599818F8198131CC09A818885981386
:1080800018C09B818985981314C02C818D8190E044
:10809000A0E0B0E0BA2FA92F982F8827820F911D5A
:1080A000A11DB11D880E991EAA1EBB1E8FEFC81AF6
:1080B000D80A9FEF491A590A690A790AADCFCF92B7
:1080C000DF92EF92FF92CF93DF93CDB7DEB72C977D
:1080D0000FB6F894DEBF0FBECDBF8BE39FE00E94CA
:1080E000178540E052EC61E070E08BE39FE00E9476
:1080F0003E094CED55E060E070E08BE39FE00E94AC
:108100000B8A64E670E080E090E00E94D78163E033
:1081100077E08FED9BE00E94FB8B6FED7BE08EE9BB
:108120009EE00E94C48762E370E080E090E00E94DD
:10813000D7816FED7BE0CE0101960E94DD8B42E39B
:1081400050E06FEF7FEFCE0101960E94B509CE019E
:1081500001960E94F38A6FE077E089ED9BE00E9430
:10816000FB8B69ED7BE0CE0101960E94DD8B44E143
:1081700050E06FEF7FEFCE0101960E94290BCE01F8
:1081800001960E94F38A8091000D9091010D019754
:1081900031F484E090E0B2DE6B017C0103C0C12CBD
:1081A000D12C76018091000D9091010D892B29F43D
:1081B00081E090E0A3DE6B017C0120E030E040EA4A
:1081C00051E4C701B6010E947691181664F521E0CA
:1081D000B701A601CE0107960E94808C6FEC75E076
:1081E000CE0101960E945E8BBE01695F7F4FCE017A
:1081F00001960E94578D6CEC75E00E94688DBC0161
:108200008FED9BE00E94C88BCE0101960E94F38AFD
:10821000CE0107960E94F38A81E090E09093010DD1
:108220008093000D10C06BE177E08FED9BE00E9422
:10823000FB8B8091000D9091010D019721F410921C
:10824000010D1092000D6FED7BE0CE0101960E94B2
:10825000DD8B4AE050E060E070E0CE0101960E94C4
:10826000B509CE0101960E94F38A6FED7BE0CE0145
:1082700001960E94DD8B66EC74E0CE0101960E94AF
:10828000688D69ED7BE00E94578DBC018FED9BE00E
:108290000E94C88BCE0101960E94F38A8BE39FE077
:1082A0000E9417858091D00B882331F060E273E043
:1082B00080E090E00E94D7812C960FB6F894DEBF44
:1082C0000FBECDBFDF91CF91FF90EF90DF90CF90A9
:1082D0000895FF920F931F93CF93DF93CDB7DEB72F
:1082E0002C970FB6F894DEBF0FBECDBF1092D10B06
:1082F0006CE67AE081EF9BE00E94FB8B11E08EE957
:108300009EE00E94A8832091D10B1816190684F5CF
:1083100021112EC08EE99EE00E94C1838093D20B72
:108320008A3041F08D3031F0682F81EF9BE00E9460
:10833000448D17C01093D10B67E277E0CE01019610
:108340000E945E8B61EF7BE0CE0101960E94578D0B
:10835000BC018EE99EE00E94C487CE0101960E9476
:10836000F38A6AE070E080E090E00E94D781C7CF96
:10837000222361F02091D10B8091F50B9091F60BA7
:1083800021116CC0009709F069C0B0C000E010E096
:10839000FF24F39488ED9FE00E94A8831816190625
:1083A000A4F588ED9FE00E94C1838093D20B8A30B0
:1083B00071F08D3061F09091D10B911108C0682F50
:1083C00081EF9BE00E94448D0F5F1F4F17C080918B
:1083D000F50B9091F60B892B89F0F092D10B88ED7B
:1083E0009FE00E94A8831816190644F46CE67AE010
:1083F00081EF9BE00E94FB8B1092D10B6FE070E04D
:1084000080E090E00E94D781C5CF62E370E080E019
:1084100090E00E94D781012B09F4ACCF60E377E0B4
:10842000CE0101960E945E8B61EF7BE0CE0101964A
:108430000E94578DBC018EE99EE00E94C487CE0148
:1084400001960E94F38A88ED9FE00E94308464E6E2
:1084500070E080E090E00E94D7818CCF019709F016
:1084600069C067E776E0CE0107960E945E8BBE0189
:10847000695F7F4F81EF9BE00E94A48D811115C041
:1084800065E377E0CE0101960E945E8BBE016F5FCF
:108490007F4F81EF9BE00E94A48D11E0811110E0DD
:1084A000CE0101960E94F38A01C010E0CE0107962A
:1084B0000E94F38A112399F040E050E061EF7BE0E5
:1084C000CE0101960E943209BE016F5F7F4F8BEE95
:1084D0009BE00E94E58BCE0101960E94F38A64E145
:1084E00070E080E090E00E94D78124C064E670E0F4
:1084F00080E090E00E94D7810E94A881CB0168EEC5
:1085000073E00E946593CB0164E670E00E9465937E
:10851000823691057CF08091D00B81110BC08BEEDF
:108520009BE00E94E48E613071058105910511F494
:108530000E94A3172C960FB6F894DEBF0FBECDBFD6
:10854000DF91CF911F910F91FF9008954F925F920D
:108550006F927F928F929F92AF92BF92CF92DF9253
:10856000EF92FF92CF93DF93CDB7DEB760970FB650
:10857000F894DEBF0FBECDBF8091D00B811105C036
:108580008EE190E0A0E0B0E004C082E090E0A0E0E6
:10859000B0E08D879E87AF87B88B65ED72E08FED79
:1085A0009BE00E94DC8C6FED7BE0CE0101960E9487
:1085B000DD8B4AE050E06FEF7FEFCE0101960E9425
:1085C000290BCE0101960E94F38A812C912C540133
:1085D000C12CD12C760163E270E084E09DE00E9422
:1085E0000E5C67E070E084E09DE00E94410984E059
:1085F0009DE00E94825C66E970E080E090E00E946D
:10860000D78163E270E084E09DE00E940E5C60E24E
:1086100070E084E09DE00E94410984E09DE00E94BA
:10862000825C66E970E080E090E00E94D78142E0E1
:1086300050E063E270E084E09DE00E94805C412CA9
:10864000512C320184E09DE00E94665B18161906E9
:108650006CF484E09DE00E946E5B762C652C542CBB
:108660004424480E511C611C711CECCFC301B201A3
:108670000E94A1902AE939E949E95FE30E94D58F78
:108680000E946E90AB01BC01C416D506E606F70643
:1086900014F46A017B012AE0CE0107960E94548CF3
:1086A000BE01695F7F4FCE0101960E94DD8B67E3BB
:1086B00077E0CE0101960E94688DBC0189ED9BE0B8
:1086C0000E94C88BCE0101960E94F38ACE010796C4
:1086D0000E94F38A69ED7BE0CE0101960E94DD8B5A
:1086E0004EE150E060E070E0CE0101960E945E0A2B
:1086F000CE0101960E94F38A9FEF891A990AA90A6E
:10870000B90A8D859E85AF85B88988159905AA0512
:10871000BB050CF060CF2AE0B701A601CE01079699
:108720000E94548CBE01695F7F4FCE0101960E946A
:10873000DD8B67E377E0CE0101960E94688DBC0176
:1087400089ED9BE00E94C88BCE0101960E94F38ABE
:10875000CE0107960E94F38A69ED7BE0CE01019677
:108760000E94DD8B4AE050E060E070E0CE010196AF
:108770000E94B509CE0101960E94F38A2AE0B70152
:10878000A601CE0107960E94548C6BE377E0CE01E0
:1087900001960E945E8BBE01695F7F4FCE010196FC
:1087A0000E94578D6EE377E00E94688D6FED7BE04D
:1087B0000E94578DBC018FED9BE00E94C88BCE01BB
:1087C00001960E94F38ACE0107960E94F38A62E323
:1087D00070E080E090E00E94D78160960FB6F89438
:1087E000DEBF0FBECDBFDF91CF91FF90EF90DF9046
:1087F000CF90BF90AF909F908F907F906F905F9041
:108800004F9008958F929F92AF92BF92CF92DF9236
:10881000EF92FF920F931F93CF93DF9300D000D07E
:10882000CDB7DEB78C01E090CD0BF090CE0B65E0BC
:1088300078E08EE99EE00E9478874AE050E0B80137
:108840008EE99EE00E949A88C8010596059718F166
:108850008091CD0B9091CE0B8017910719F10E945A
:10886000040C1093CE0B0093CD0B89EE9CE00E947C
:10887000025F4AE0B801CE0101960E94298CBE0138
:108880006F5F7F4F8BEE9BE00E94E58BCE010196E0
:108890000E94F38A07C00E3F8FEF1807A9F40E94C9
:1088A0004B2F9EC166EC74E0CE0101960E945E8B58
:1088B0004AE050E06FEF7FEFCE0101960E945E0A22
:1088C000CE0101960E94F38AF8017996E332F10510
:1088D00008F025C1EE58FF4F0C94B6938091D00B51
:1088E000882319F00E94483648C160910A027091AD
:1088F0000B0280910C0290910D020E9440343DC108
:1089000080918A0490918B040E94AD2F36C1809192
:108910007004909171040E945A292FC180916404BF
:10892000909165040E94BF2D28C1809166049091AA
:1089300067040E944F2821C10E94A8810E941F380D
:108940001CC160E070E080916A0490916B040E9409
:108950002F2413C180916004909161040E94732BB5
:108960000CC18091CF0B91E089278093CF0B809130
:10897000D00B882331F06FED7BE088ED9FE00E9403
:10898000C48768EC70E080E090E00E94D781F5C079
:108990001092D00BF2C081E08093D00BEEC00E9409
:1089A000290CEBC08CDBE9C00E946116E6C0809107
:1089B0003C02882309F4E1C06CE67AE0CE0101961E
:1089C0000E945E8B4AE050E061E070E0CE010196CB
:1089D0000E94B509CE0101960E94F38A0E942F0ED3
:1089E000CCC0B4DDCAC080916C0490916D040E942B
:1089F000002DC3C080916204909163040E940A2CF0
:108A0000BCC080913C02882309F4B7C08091D00B90
:108A1000882329F082E090E00E947410AEC083E0C9
:108A200090E00E94A314A9C00E945F2288ED9FE0FD
:108A30000E943084A2C080918102909182020E94A3
:108A400058269BC080913C02882309F496C08091EF
:108A5000D00B811127C0C0900A02D0900B02E09089
:108A60000C02F0900D0220E030E04AE754E4C70128
:108A7000B6010E9435920E946E904B015C0120E08D
:108A800030E040EA50E4C701B6010E94359220E090
:108A900030E040EA50E40E940B8F0E946E90A501E6
:108AA000940108C021E030E040E050E06AE070E06E
:108AB00080E090E00E942F1E60C08091020D909196
:108AC000030D892BA1F481E090E09093030D809336
:108AD000020D8EED93E09093640B8093630B0E94E4
:108AE000910968EC70E080E090E00E94D781E0910D
:108AF0009A0AF0919B0A199540C0E091E90CF09117
:108B0000EA0C0480F581E02D20E042E060E189EE8E
:108B10009CE019950E943D2F0E94040C2EC0F092FB
:108B2000CE0BE092CD0B68EF77E08FED9BE00E94DB
:108B3000DC8C6CE67AE0CE0101960E945E8B4AE006
:108B400050E060E070E0CE0101960E94B509CE01D0
:108B500001960E94F38A6FED7BE0CE0101960E94A0
:108B6000DD8B4AE050E06FEF7FEFCE0101960E946F
:108B7000290BCE0101960E94F38A8091E30B90911C
:108B8000E40B009799F0419718F402301105ACF40A
:108B90006FED7BE0CE0101960E94DD8BCE01019648
:108BA0000E948B0FCE0101960E94F38A64E670E06A
:108BB00080E090E00E94D78113C06FED7BE0CE0192
:108BC00001960E94DD8B4AE050E06FEF7FEFCE010F
:108BD00001960E94290BCE0101960E94F38AD8CFFC
:108BE00026960FB6F894DEBF0FBECDBFDF91CF91B2
:108BF0001F910F91FF90EF90DF90CF90BF90AF90BB
:108C00009F908F900895FF920F931F93CF93DF93C0
:108C100000D000D0CDB7DEB7823409F472C0D4F4EE
:108C2000803309F48EC07CF4833209F481C08A3227
:108C300009F0A5C06FE477E081EF9BE00E94FB8B19
:108C40008FEF9FEFF8C0813309F48AC0813409F4B3
:108C50004DC095C0813609F449C034F4833409F419
:108C60005BC0843449F08BC0833609F455C00CF4E2
:108C700048C0843609F083C08091EF0B9091F00BCF
:108C8000892B09F4DAC08BEE9BE00E94E48E97FDFD
:108C9000D4C062EF77E08EE99EE00E9478876BEEA9
:108CA0007BE08EE99EE00E94C4878BEE9BE00E94F1
:108CB000E48EDC01CB014AEF5FEF6FEF7FEF481BE3
:108CC000590B6A0B7B0B2AE0CE0101960E94548C53
:108CD000BE016F5F7F4F8BEE9BE00E94E58BCE0164
:108CE00001960E94F38A8BEE9BE0A2C063E477E0DA
:108CF00081EF9BE00E94FB8B8091CD0B9091CE0B7E
:108D00009AC066E477E081EF9BE00E94FB8B1092B3
:108D1000D00B8CEF9FEF8FC069E477E081EF9BE091
:108D20000E94FB8B81E08093D00B8DEF9FEF83C07F
:108D30006CE477E081EF9BE00E94FB8B8EEF9FEF6E
:108D40007AC06DE577E08BEE9BE00E94FB8B6DE5D2
:108D500077E081EF9BE00E94FB8B80E090E06BC0AE
:108D600060E577E08BEE9BE00E94FB8B60E577E0AF
:108D700081EF9BE00E94FB8B81E090E05CC0682F5C
:108D8000CE0101960E94118CBE016F5F7F4F8BEE6A
:108D90009BE00E94E58BCE0101960E94F38A8BEE48
:108DA0009BE00E94E48ECB012DDD64E670E080E064
:108DB00090E00E94D78149C00F5F1F4F093E83E0BA
:108DC000180769F06EE170E080E090E00E94D781C2
:108DD0008BE59CE00E945A6AF82EFF2069F36AE254
:108DE00070E06F197109F7FC73954AE0CE010196A6
:108DF0000E94298CBE016F5F7F4F81EF9BE00E9434
:108E0000E58BCE0101960E94F38A61EF7BE08BEE49
:108E10009BE00E94C88B6CEE77E08EE99EE00E949A
:108E200078876F2D8EE99EE00E94E48781EF9BE0BA
:108E30000E94E48ECB01E6DC08C08BE59CE00E943A
:108E40005A6AF82E00E010E0C8CF26960FB6F894C4
:108E5000DEBF0FBECDBFDF91CF911F910F91FF906D
:108E600008950F931F93CF93DF9300D000D0CDB719
:108E7000DEB74091B00A5091B10A6091B20A709188
:108E8000B30A20E130E08EE99EE00E94E188809103
:108E9000B00A9091B10AA091B20AB091B30A883099
:108EA00025E09207A105B10509F4F8C108F08DC0CD
:108EB000893421E09207A105B10509F4F2C1E0F57A
:108EC000843421E09207A105B10509F4DBC1E8F47F
:108ED000813421E09207A105B10509F4C4C138F439
:108EE00080349140A105B10509F4AEC1DDC18234E1
:108EF00021E09207A105B10509F4BEC18334914078
:108F0000A105B10509F4BBC1CFC1863421E09207A8
:108F1000A105B10509F4BCC108F4B7C1873421E04B
:108F20009207A105B10509F4B6C188349140A105A5
:108F3000B10509F4B3C1B8C1823025E09207A1059B
:108F4000B10509F499C1E8F4843721E09207A1053D
:108F5000B10509F444C138F482379140A105B10547
:108F600009F448C1A1C1811525E09207A105B10509
:108F700009F46AC181309540A105B10509F473C1B6
:108F800093C1853025E09207A105B10509F47DC1A3
:108F900070F4833025E09207A105B10509F46FC193
:108FA00084309540A105B10509F46CC17DC18630BE
:108FB00025E09207A105B10509F46AC18730954003
:108FC000A105B10509F467C16FC18D3B22E4920789
:108FD0002FEFA207B10509F428C108F04BC08F3E5E
:108FE00020E192072FEFA207B10509F454C118F54B
:108FF000823325E09207A105B10509F4FBC038F4DE
:1090000089309540A105B10509F44BC14DC18433A8
:1090100025E09207A105B10509F4E1C08D3F92401A
:10902000AF4FB10509F040C163E477E081EF9BE009
:109030000E94FB8BDCC08D3D22E292072FEFA2073E
:10904000B10509F4CCC038F4873E9841AF4FB10563
:1090500009F41BC129C18F3C20E392072FEFA2071F
:10906000B10509F40FC1873C9843AF4FB10509F42E
:1090700015C11AC1873928E692072FEFA207B1055B
:1090800009F4F1C048F58D3A22E592072FEFA207C7
:10909000B10509F4BBC038F4853B9A44AF4FB10524
:1090A00009F4D2C001C1853A2AE592072FEFA20741
:1090B000B10509F4F6C08D399246AF4FB10509F0FC
:1090C000F3C066E477E081EF9BE00E94FB8B109297
:1090D000D00B8CEF9FEF81C0873528EA92072FEFE6
:1090E000A207B105F9F078F485382AE792072FEF47
:1090F000A207B10509F4CCC087369849AF4FB10536
:1091000009F4BAC0D1C08F3420EB92072FEFA20729
:10911000B10509F4B4C08D33924CAF4FB10509F4D9
:1091200069C0C2C08CEB9AE00E941A7300E010E0A4
:109130006CE97AE08CEB9AE00E94CF73892B39F4CA
:109140000F5F1F4F093E83E0180709F09CC16AEDCD
:1091500077E08EE99EE00E9478874091A00A5091C6
:10916000A10A6091A20A7091A30A2AE030E08EE978
:109170009EE00E94E1888091A00A9091A10AA091AE
:10918000A20AB091A30A853025E09207A105B10596
:1091900009F4B9C008F0C0C0873421E09207A105E6
:1091A000B10509F4D9C008F0DAC0833421E0920790
:1091B000A105B10509F4E3C008F09EC0813421E0A7
:1091C0009207A105B10509F0E3C062E577E08BEEF7
:1091D0009BE00E94FB8B89EF9FEF14DB7EC063E472
:1091E00077E081EF9BE00E94FB8B1092D00B8BEF1E
:1091F0009FEFF3CF69E477E081EF9BE00E94FB8B68
:1092000081E08093D00B8DEF9FEFE7CF6CE477E0A8
:109210008BEE9BE00E94FB8B6CE477E081EF9BE0A0
:109220000E94FB8B8EEF9FEFD8CF6FE477E08BEE41
:109230009BE00E94FB8B6FE477E081EF9BE00E9454
:10924000FB8B8FEF9FEFC9CF6DE577E08BEE9BE057
:109250000E94FB8B6DE577E081EF9BE00E94FB8B2A
:1092600080E090E0BACF60E577E08BEE9BE00E9473
:10927000FB8B81E090E0B1CF82E090E0AECF83E065
:1092800090E0ABCF84E090E0A8CF85E090E0A5CF60
:1092900086E090E0A2CF87E090E09FCF88E090E06A
:1092A0009CCF89E090E099CF40E050E061EF7BE017
:1092B000CE0101960E943209BE016F5F7F4F8BEE97
:1092C0009BE00E94E58BCE0101960E94F38A64E642
:1092D00070E080E090E00E94D7818CEB9AE00E94E1
:1092E0001A7326960FB6F894DEBF0FBECDBFDF917E
:1092F000CF911F910F910895853421E09207A10528
:10930000B10509F054C06FE577E08BEE9BE00E9459
:10931000FB8B85EF9FEF61CF8F3C20E392072FEF10
:10932000A207B10509F448C008F04FC0883025E015
:109330009207A105B10509F46FC008F080C086301E
:1093400025E09207A105B10509F45DC0873095407D
:10935000A105B10509F0BBCF83EF9FEF3ECF813070
:1093600025E09207A105B10509F42FCF08F44EC0FE
:10937000833025E09207A105B10509F059C068E5E1
:1093800077E08BEE9BE00E94FB8B87EF9FEF25CF72
:1093900082349140A105B10509F099CF65E577E0E8
:1093A0008BEE9BE00E94FB8B88EF9FEF16CF8634FD
:1093B0009140A105B10538F56BE577E08BEE9BE0B8
:1093C0000E94FB8B86EF9FEF08CF873928E6920734
:1093D0002FEFA207B10509F4F8CE08F447C087368D
:1093E00028E992072FEFA207B105C1F28F3420EBD5
:1093F00092072FEFA207B10511F285389A47AF4FB8
:10940000B10509F064CF84EF9FEFE7CE883421E007
:109410009207A105B10519F482EF9FEFDECE8934E2
:109420009140A105B10509F052CF81EF9FEFD5CE54
:1094300084309540A105B10508F4B0CFBDCF8F3E73
:1094400020E192072FEFA207B10509F485CF873EEF
:1094500028E192072FEFA207B10509F454CF893014
:109460009540A105B10509F032CFDFCF873C28E355
:1094700092072FEFA207B10579F2853A9A45AF4FCF
:10948000B10599F224CF6EE170E080E090E00E9497
:10949000D7814ECE8F929F92AF92BF92CF92DF92A2
:1094A000EF92FF920F931F93CF93DF93CDB7DEB769
:1094B000A6970FB6F894DEBF0FBECDBF6CEA7AE078
:1094C0008CEB9AE00E94CF73892BC9F00E943D2F4C
:1094D0000E94040C66EC74E0CE0101960E945E8B43
:1094E0004AE050E060E070E0CE0101960E94B509CC
:1094F000CE0101960E94F38AB4DC0C94DE5A6CE62D
:109500007AE081EF9BE00E94FB8B0E9469416AE058
:1095100070E080E090E00E94D7818091F50B9091FF
:10952000F60B009711F40C94C35A019709F046C04A
:1095300069EF75E0CE010F960E945E8BBE01615F00
:109540007F4F81EF9BE00E94A48D81112AC06DECBA
:1095500075E0CE0109960E945E8BBE01675F7F4F6A
:1095600081EF9BE00E94A48D811115C061E375E03D
:10957000CE0101960E945E8BBE016F5F7F4F81EF2F
:109580009BE00E94A48D11E0811110E0CE010196B4
:109590000E94F38A01C010E0CE0109960E94F38A6E
:1095A00001C010E0CE010F960E94F38A112331F022
:1095B00061EF7BE08BEE9BE00E94C88B8091F50B06
:1095C0009091F60B0497F0F563E677E0CE010196F3
:1095D0000E945E8BBE016F5F7F4F81EF9BE00E9418
:1095E000A48D182FCE0101960E94F38A112351F108
:1095F00041E050E061EF7BE0CE0109960E94320924
:10960000CE0109960E94E48EDC01CB014AEF5FEFA8
:109610006FEF7FEF481B590B6A0B7B0B2AE0CE01E3
:1096200001960E94548CBE016F5F7F4F8BEE9BE0D2
:109630000E94E58BCE0101960E94F38ACE01099625
:109640000E94F38A65E677E0CE0109960E945E8B60
:10965000BE01675F7F4F81EF9BE00E94A48D811167
:1096600016C069E677E0CE0101960E945E8BBE01CE
:109670006F5F7F4F81EF9BE00E94A48D11E081110D
:1096800001C010E0CE0101960E94F38A01C011E0F2
:10969000CE0109960E94F38A112309F4EFC260E714
:1096A0007BE0CE0101960E94FC8CCE0101960E94C7
:1096B0008B0FCE0101960E94F38A6091380270915F
:1096C000390280913A0290913B020E94A19020E0E1
:1096D00030E048EC52E40E94D58FAB01BC0122E09F
:1096E000CE010F960E94808C6DE677E0CE01099640
:1096F0000E945E8BBE01615F7F4FCE0109960E9482
:10970000578D6EE878E00E94688DBC01CE0101960D
:109710000E94DD8BCE0101960E948B0FCE01019637
:109720000E94F38ACE0109960E94F38ACE010F9619
:109730000E94F38A409134025091350260913602C2
:109740007091370224E0CE010F960E94808C62E86F
:1097500077E0CE0109960E945E8BBE01615F7F4F6C
:10976000CE0109960E94578DBC01CE0101960E9440
:10977000DD8BCE0101960E948B0FCE0101960E94D7
:10978000F38ACE0109960E94F38ACE010F960E94B9
:10979000F38A40911E0250911F0260912002709145
:1097A000210222E0CE0109960E94808C409116028F
:1097B00050911702609118027091190223E0CE01B6
:1097C0000F960E94808C409122025091230260915A
:1097D00024027091250222E0CE0145960E94808CE1
:1097E00040911A0250911B0260911C0270911D025F
:1097F00023E0CE0181960E94808C6FE977E0CE0154
:109800004B960E945E8BBE016F5D7F4FCE014B96E3
:109810000E94578D64EB77E00E94688DBE016B5EFD
:109820007F4F0E94578D67EB77E00E94688DBE01E5
:10983000615F7F4F0E94578D64EB77E00E94688DD7
:10984000BE01675F7F4F0E94578D6DEB77E00E94EE
:10985000688DBC01CE0101960E94DD8BCE01019680
:109860000E948B0FCE0101960E94F38ACE014B9687
:109870000E94F38ACE0181960E94F38ACE0145961A
:109880000E94F38ACE010F960E94F38ACE010996B8
:109890000E94F38A62EC77E0CE0109960E945E8B0B
:1098A0006BED7CE0CE0109960E94578DBC01CE0184
:1098B00001960E94DD8BCE0101960E948B0FCE0196
:1098C00001960E94F38ACE0109960E94F38A409184
:1098D000450250914602609147027091480223E090
:1098E000CE0109960E94808C2091490230914A0253
:1098F00040914B0250914C0260E070E080E291E4B4
:109900000E949892AB01BC0121E0CE0145960E94D5
:10991000AE8C63ED77E0CE010F960E945E8BBE01A8
:109920006B5E7F4FCE010F960E94578D66EE77E0FB
:109930000E94688DBE01675F7F4F0E94578D6BEF5D
:1099400075E00E94688DBC01CE0101960E94DD8BFE
:10995000CE0101960E948B0FCE0101960E94F38AE0
:10996000CE010F960E94F38ACE0145960E94F38A9B
:10997000CE0109960E94F38A409141025091420221
:10998000609143027091440223E0CE0109960E9447
:10999000808C20913D0230913E0240913F025091D7
:1099A000400260E070E080E291E40E949892AB0196
:1099B000BC0121E0CE0145960E94AE8C6CEE77E0B2
:1099C000CE010F960E945E8BBE016B5E7F4FCE0173
:1099D0000F960E94578D66EE77E00E94688DBE015B
:1099E000675F7F4F0E94578D6BEF75E00E94688D17
:1099F000BC01CE0101960E94DD8BCE0101960E9432
:109A00008B0FCE0101960E94F38ACE010F960E9421
:109A1000F38ACE0145960E94F38ACE0109960E94F0
:109A2000F38A40914D0250914E0260914F02709125
:109A3000500222E0CE010F960E94808C6FEF77E0FB
:109A4000CE0109960E945E8BBE01615F7F4FCE0101
:109A500009960E94578D65E178E00E94688DBC01EF
:109A6000CE0101960E94DD8BCE0101960E948B0FE4
:109A7000CE0101960E94F38ACE0109960E94F38AD4
:109A8000CE010F960E94F38A409112025091130268
:109A9000609114027091150222E0CE010F960E948F
:109AA000808C6CE178E0CE0109960E945E8BBE014D
:109AB000615F7F4FCE0109960E94578D6BEF75E075
:109AC0000E94688DBC01CE0101960E94DD8BCE0103
:109AD00001960E948B0FCE0101960E94F38ACE015F
:109AE00009960E94F38ACE010F960E94F38ABEE384
:109AF000CB2EB4E0DB2E01E010E085E1E82E809172
:109B00003C0490913D04801791070CF44FC0D6019E
:109B1000AD90BD906D014AE0B501CE0109960E945D
:109B2000298C4AE0B801CE0145960E94298C6FE24B
:109B300078E0CE010F960E945E8BBE016B5E7F4F78
:109B4000CE010F960E94578D6DEE74E00E94688DD5
:109B5000BE01675F7F4F0E94578D67E378E00E94E8
:109B6000688DEA9CB001EB9C700D11246D577D4F00
:109B70000E94688DBC01CE0101960E94DD8BCE0152
:109B800001960E948B0FCE0101960E94F38ACE01AE
:109B90000F960E94F38ACE0145960E94F38ACE0169
:109BA00009960E94F38A0F5F1F4FA9CF40910E02C2
:109BB00050910F02609110027091110222E0CE01CB
:109BC0000F960E94808C6DE378E0CE0109960E948A
:109BD0005E8BBE01615F7F4FCE0109960E94578D5B
:109BE00067E776E00E94688DBC01CE0101960E9475
:109BF000DD8BCE0101960E948B0FCE0101960E9453
:109C0000F38ACE0109960E94F38ACE010F960E9434
:109C1000F38A40910A0250910B0260910C027091FC
:109C20000D0222E0CE010F960E94808C6DE478E058
:109C3000CE0109960E945E8BBE01615F7F4FCE010F
:109C400009960E94578D67E776E00E94688DBC01F7
:109C5000CE0101960E94DD8BCE0101960E948B0FF2
:109C6000CE0101960E94F38ACE0109960E94F38AE2
:109C7000CE010F960E94F38A10E001C011E00E940D
:109C80003D2F0E94040C66EC74E0CE0101960E9408
:109C90005E8B4AE050E060E070E0CE0101960E94E9
:109CA0005E0ACE0101960E94F38A8091F50B909195
:109CB000F60B8330910508F06FC0019739F460E02E
:109CC00070E081EF9BE00E94C38DF82E8091F50B30
:109CD0009091F60B029709F050C063E677E0CE0151
:109CE00001960E945E8BBE016F5F7F4F81EF9BE00C
:109CF0000E94A48D182FCE0101960E94F38A112391
:109D0000E1F161E070E081EF9BE00E94C38D682F7C
:109D1000CE0101960E94118CBE016F5F7F4F8BEECA
:109D20009BE00E94F08BCE0101960E94F38A60E0D6
:109D300070E081EF9BE00E94C38DF82E68E478E02C
:109D4000CE0101960E945E8B61EF7BE0CE01019611
:109D50000E94578D66EC74E00E94688DBC018EE90C
:109D60009EE00E949B87CE0101960E94F38A6BEED3
:109D70007BE08EE99EE00E94C4878F2D0E940346FF
:109D80000E94A8816093F70B7093F80B8093F90BF6
:109D90009093FA0B0C94DE5A21E030E040E050E062
:109DA00061EF7BE0CE0101960E94458EBE016F5FA0
:109DB0007F4F89ED9BE00E94E58BCE0101960E94CA
:109DC000F38A6AE878E0CE0109960E945E8BBE01B4
:109DD000675F7F4F81EF9BE00E94A48D811116C0C9
:109DE00063E975E0CE0101960E945E8BBE016F5F54
:109DF0007F4F81EF9BE00E94A48D01E0811101C0A3
:109E000000E0CE0101960E94F38A01C001E0CE017C
:109E100009960E94F38A002309F4A7C042E050E0AB
:109E200061EF7BE0CE0101960E943209BE016F5FB7
:109E30007F4F89ED9BE00E94E58BCE0101960E9449
:109E4000F38A69ED7BE08EE99EE00E94C48789ED8C
:109E50009BE00E94EE8E20E030E048EC52E40E944D
:109E600035920E946E90AB01BC0140933802509332
:109E7000390260933A0270933B022AE030E08EE9A7
:109E80009EE00E94B0886091380270913902809102
:109E90003A0290913B028B019C0100591F452140E1
:109EA000310901341C492105310588F06DE578E060
:109EB000CE0101960E945E8B69ED7BE0CE0101969A
:109EC0000E94578D60E778E00E94688D73C1198207
:109ED0001A821B821C821D821E821F8218860E948B
:109EE000A19020E030E048EC52E40E94D58F8E0132
:109EF0000F5F1F4F22E047E00E941694BC018FEDD8
:109F00009BE00E94FB8B60E878E0CE0109960E94FE
:109F10005E8B6FED7BE0CE0109960E94578D6DE858
:109F200078E00E94688DBC018FED9BE00E94C88B99
:109F3000CE0109960E94F38A1092640B1092630B73
:109F40008091380290913902A0913A02B0913B027F
:109F50008093BD0A9093BE0AA093BF0AB093C00A33
:109F600080E090E00E9468092EC162E978E0CE01AD
:109F700009960E945E8BBE01675F7F4F81EF9BE079
:109F80000E94A48D811116C068E978E0CE01019687
:109F90000E945E8BBE016F5F7F4F81EF9BE00E944E
:109FA000A48D01E0811101C000E0CE0101960E9464
:109FB000F38A01C001E0CE0109960E94F38A0023D2
:109FC00009F46DC026E030E045E050E061EF7BE051
:109FD000CE0101960E94458EBE016F5F7F4F89EDD5
:109FE0009BE00E94E58BCE0101960E94F38A89EDE9
:109FF0009BE00E94E48E6B017C0163E178E0CE017E
:10A0000009960E945E8BBE01675F7F4F81EF9BE0E8
:10A010000E943C8EAC014F5F5F4F61EF7BE0CE0151
:10A0200001960E943209BE016F5F7F4F89ED9BE070
:10A030000E94E58BCE0101960E94F38ACE0109961B
:10A040000E94F38A89ED9BE00E94E48EDB01EEE33F
:10A05000F4E021E030E040913C0450913D0442178F
:10A0600053075CF0408151814A175B0711F411825C
:10A0700010822F5F3F4F3296EECFF601EE0FFF1F9B
:10A08000E45CFB4F7183608382E090E00E94732E5A
:10A0900061EF7BE08EE99EE00E94C48749C06EE9D3
:10A0A00078E0CE0109960E945E8BBE01675F7F4F0C
:10A0B00081EF9BE00E94A48D811116C064EA78E0D4
:10A0C000CE0101960E945E8BBE016F5F7F4F81EFD4
:10A0D0009BE00E94A48D01E0811101C000E0CE014F
:10A0E00001960E94F38A01C001E0CE0109960E9408
:10A0F000F38A002339F1EEE3F4E081E090E020916F
:10A100003C0430913D042817390774F086309105DE
:10A110001CF49183808305C09C012E5F3F4F3183E7
:10A12000208301963296EBCF82E090E00E94732E5E
:10A130001092640B1092630B80E090E00E9468091B
:10A140000C94DE5A6AEA78E0CE0109960E945E8B92
:10A15000BE01675F7F4F81EF9BE00E94A48D81115C
:10A1600016C062EB78E0CE0101960E945E8BBE01C4
:10A170006F5F7F4F81EF9BE00E94A48D01E0811112
:10A1800001C000E0CE0101960E94F38A01C001E007
:10A19000CE0109960E94F38A002391F16AEB78E0E0
:10A1A000CE0101960E945E8B65ED7CE0CE010196AA
:10A1B0000E94578DBC018FED9BE00E94C88BCE01A1
:10A1C00001960E94F38A6FEC76E0CE0109960E9418
:10A1D0005E8B6FED7BE0CE0109960E94578DBC012E
:10A1E000CE0101960E94DD8BCE0101960E948B0F5D
:10A1F000CE0101960E94F38ACE0109960C94C05AB2
:10A2000064EC78E0CE0109960E945E8BBE01675F28
:10A210007F4F81EF9BE00E94A48D811116C069ECF5
:10A2200078E0CE0101960E945E8BBE016F5F7F4F8A
:10A2300081EF9BE00E94A48D01E0811101C000E04C
:10A24000CE0101960E94F38A01C001E0CE01099679
:10A250000E94F38A002309F444C063E178E0CE0150
:10A2600009960E945E8BBE01675F7F4F81EF9BE086
:10A270000E943C8EAC014F5F5F4F61EF7BE0CE01EF
:10A2800001960E943209BE016F5F7F4F89ED9BE00E
:10A290000E94E58BCE0101960E94F38ACE010996B9
:10A2A0000E94F38A89ED9BE00E94E48E611571059E
:10A2B00021F481E08093990410C06130710519F494
:10A2C000109299040AC06230710511F00C94DE5AA4
:10A2D00081E080939904109298040E944B2F0C9473
:10A2E000DE5A6EEC78E0CE0109960E945E8BBE01CC
:10A2F000675F7F4F81EF9BE00E94A48D811116C0A4
:10A3000062ED78E0CE0101960E945E8BBE016F5F28
:10A310007F4F81EF9BE00E94A48D01E0811101C07D
:10A3200000E0CE0101960E94F38A01C001E0CE0157
:10A3300009960E94F38A002309F45CC043E050E0D0
:10A3400061EF7BE0CE0101960E943209BE016F5F92
:10A350007F4F89ED9BE00E94E58BCE0101960E9424
:10A36000F38A69ED7BE08EE99EE00E94C48710923B
:10A37000640B1092630B69ED7BE08BED9CE00E9417
:10A38000C88B20E030E048E050E069ED7AE08BEDEA
:10A390009CE00E94C48D8091630B9091640B0E949D
:10A3A000680966ED78E0CE0101960E945E8B6BED48
:10A3B0007CE0CE0101960E94578DBC01CE0109962A
:10A3C0000E94DD8BCE0101960E94F38ABE01675F79
:10A3D0007F4F88ED9FE00E949B8768EB7BE080E0E9
:10A3E00090E00E94D78169ED7AE08EE99EE00E94BC
:10A3F000D48769C06EED78E0CE0109960E945E8B2D
:10A40000BE01675F7F4F81EF9BE00E94A48D8111A9
:10A4100016C063EE78E0CE0101960E945E8BBE010D
:10A420006F5F7F4F81EF9BE00E94A48D01E081115F
:10A4300001C000E0CE0101960E94F38A01C001E054
:10A44000CE0109960E94F38A002309F43FC044E03C
:10A4500050E061EF7BE0CE0101960E943209BE011F
:10A460006F5F7F4F89ED9BE00E94E58BCE010196E7
:10A470000E94F38A68EE78E0CE0101960E945E8B1E
:10A4800069ED7BE0CE0101960E94578DBC01CE01A3
:10A4900009960E94DD8BCE0101960E94F38ABE01CF
:10A4A000675F7F4F88ED9FE00E949B8768EB7BE0B2
:10A4B00080E090E00E94D781BE01675F7F4F8EE908
:10A4C0009EE00E94C487CE01099691C76FEE78E0A6
:10A4D000CE010F960E945E8BBE01615F7F4F81EFC0
:10A4E0009BE00E94A48D81112BC062EF78E0CE0129
:10A4F00009960E945E8BBE01675F7F4F81EF9BE0F4
:10A500000E94A48D811116C065EF78E0CE010196FE
:10A510000E945E8BBE016F5F7F4F81EF9BE00E94C8
:10A52000A48D01E0811101C000E0CE0101960E94DE
:10A53000F38A01C001E0CE0109960E94F38A01C0AE
:10A5400001E0CE010F960E94F38A002309F42DC189
:10A550006AE0A62EB12CC12CD12C760188248A94D5
:10A5600073E0972E6EE170E080E090E00E94D7816A
:10A57000809181020E946D82B4010E9465938827B8
:10A5800077FD8095982F0E94A19020E030E040EA6E
:10A5900050E40E9435929B01AC01C701B6010E94B4
:10A5A0000B8F6B017C01E1E0AE1AB108D9F620E017
:10A5B00030E040E251E40E94D58F6B017C0168EFEE
:10A5C00078E0CE0109960E945E8BBE01675F7F4FE7
:10A5D00081EF9BE00E94A48D811116C06CEF78E0A2
:10A5E000CE0101960E945E8BBE016F5F7F4F81EFAF
:10A5F0009BE00E94A48D01E0811101C000E0CE012A
:10A6000001960E94F38A01C001E0CE0109960E94E2
:10A61000F38A002309F43FC020E030E040E650E434
:10A62000C701B6010E9435929B01AC0160E070E069
:10A6300080E890E40E940A8FAB01BC0140932A029B
:10A6400050932B0260932C0270932D0222E0CE01D6
:10A6500001960E94808CBE016F5F7F4F8FED9BE063
:10A660000E94E58BCE0101960E94F38A60E079E0BA
:10A67000CE0101960E945E8B6FED7BE0CE010196CC
:10A680000E94578DBC018FED9BE00E94C88BCE01CC
:10A6900001960E94F38A6FE079E0CE0109960E944C
:10A6A0005E8BBE01675F7F4F81EF9BE00E94A48DB0
:10A6B000811116C064E179E0CE0101960E945E8BA3
:10A6C000BE016F5F7F4F81EF9BE00E94A48D01E090
:10A6D000811101C000E0CE0101960E94F38A01C001
:10A6E00001E0CE0109960E94F38A002309F43FC0DD
:10A6F00020E030E040E650E4C701B6010E94359208
:10A700009B01AC0160E070E080E291E40E940A8F5E
:10A71000AB01BC01409326025093270260932802AC
:10A720007093290222E0CE0101960E94808CBE0126
:10A730006F5F7F4F8FED9BE00E94E58BCE0101960E
:10A740000E94F38A69E179E0CE0101960E945E8B56
:10A750006FED7BE0CE0101960E94578DBC018FED1D
:10A760009BE00E94C88BCE0101960E94F38A6FEC99
:10A7700076E0CE0109960E945E8B6FED7BE0CE0104
:10A7800009960E94578DBC01CE0101960E94DD8B77
:10A79000CE0101960E948B0FCE0101960E94F38A92
:10A7A000CE0109960E94F38AD6C669E279E0CE010D
:10A7B00001960E945E8BBE016F5F7F4F81EF9BE031
:10A7C0000E94A48D082FCE0101960E94F38A0023D7
:10A7D00009F46EC08091F50B9091F60B079708F481
:10A7E000BAC646E050E061EF7BE0CE0101960E94E0
:10A7F0003209BE016F5F7F4F89ED9BE00E94E58BC0
:10A80000CE0101960E94F38A89ED9BE00E94EE8EB4
:10A81000AB01BC0140930E0250930F0260931002F3
:10A820007093110221E0CE0109960E94808C6DE3A5
:10A8300078E0CE0101960E945E8BBE01675F7F4F7C
:10A84000CE0101960E94578D67E776E00E94688DE1
:10A85000BC018FED9BE00E94C88BCE0101960E9447
:10A86000F38ACE0109960E94F38A6FED7BE0CE0158
:10A8700001960E94DD8BCE0101960E948B0FCE01C6
:10A8800001960E94F38A0E94A88128EE33E040E0FE
:10A8900050E00E947893CA01B9010E949F90609392
:10A8A000370B7093380B8093390B90933A0B53C648
:10A8B00060E379E0CE0101960E945E8BBE016F5F7E
:10A8C0007F4F81EF9BE00E94A48D082FCE0101965F
:10A8D0000E94F38A0023E9F18091F50B9091F60B29
:10A8E000079708F438C646E050E061EF7BE0CE0100
:10A8F00001960E943209BE016F5F7F4F89ED9BE098
:10A900000E94E58BCE0101960E94F38A89ED9BE0BF
:10A910000E94EE8EAB01BC0140930A0250930B02E1
:10A9200060930C0270930D0221E0CE0109960E9403
:10A93000808C6DE478E0CE0101960E945E8BBE01B2
:10A94000675F7F4FCE0101960E94578D67E776E0E3
:10A950004DC367E379E0CE0109960E945E8BBE018C
:10A96000675F7F4F81EF9BE00E94A48D811116C02D
:10A970006BE379E0CE0101960E945E8BBE016F5FB2
:10A980007F4F81EF9BE00E94A48D01E0811101C007
:10A9900000E0CE0101960E94F38A01C001E0CE01E1
:10A9A00009960E94F38A002309F456C080916A0434
:10A9B00090916B040E94042460931A0270931B020E
:10A9C00080931C0290931D026093D10A7093D20A67
:10A9D0008093D30A9093D40A80E090E0A0E8BFE38C
:10A9E0008093220290932302A0932402B093250225
:10A9F0008093C90A9093CA0AA093CB0AB093CC0A59
:10AA000065E57BE08EE99EE00E94788740911A021E
:10AA100050911B0260911C0270911D0222E030E0F7
:10AA20008EE99EE00E94CD891092640B1092630B18
:10AA300080E090E00E94680940911A0250911B0248
:10AA400060911C0270911D0222E0CE0109960E94C5
:10AA5000808C6FE379E0A7C468E479E0CE010996C1
:10AA60000E945E8BBE01675F7F4F81EF9BE00E947B
:10AA7000A48D811116C06EE479E0CE0101960E948A
:10AA80005E8BBE016F5F7F4F81EF9BE00E94A48DC4
:10AA900001E0811101C000E0CE0101960E94F38A1D
:10AAA00001C001E0CE0109960E94F38A002309F457
:10AAB00065C08091F50B9091F60B0797F8F046E092
:10AAC00050E061EF7BE0CE0101960E943209BE01A9
:10AAD0006F5F7F4F89ED9BE00E94E58BCE01019671
:10AAE0000E94F38A89ED9BE00E94EE8E60934D02F6
:10AAF00070934E0280934F029093500280916404B1
:10AB00000E94362E80914D0290914E02A0914F02EC
:10AB1000B09150028093F10A9093F20AA093F30A45
:10AB2000B093F40A64E47BE08EE99EE00E947887AB
:10AB300040914D0250914E0260914F02709150022F
:10AB400022E030E08EE99EE00E94CD891092640BF5
:10AB50001092630B80E090E00E94680940914D02E2
:10AB600050914E0260914F027091500222E0CE014E
:10AB700009960E94808C64E579E015C46EE579E061
:10AB8000CE0109960E945E8BBE01675F7F4F81EF09
:10AB90009BE00E94A48D811116C063E679E0CE018E
:10ABA00001960E945E8BBE016F5F7F4F81EF9BE03D
:10ABB0000E94A48D01E0811101C000E0CE01019648
:10ABC0000E94F38A01C001E0CE0109960E94F38A37
:10ABD000002309F49BC08091F50B9091F60B06972A
:10ABE00008F145E050E061EF7BE0CE0101960E9464
:10ABF0003209BE016F5F7F4F89ED9BE00E94E58BBC
:10AC0000CE0101960E94F38A89ED9BE00E94EE8EB0
:10AC10000E94B7916093490270934A0280934B025D
:10AC200090934C0280916604909167040E9497274C
:10AC300020E030E048E051E40E94D58F6093450267
:10AC40007093460280934702909348026093E10A12
:10AC50007093E20A8093E30A9093E40A8091490298
:10AC600090914A02A0914B02B0914C028093E90A64
:10AC70009093EA0AA093EB0AB093EC0A64E37BE0BA
:10AC80008EE99EE00E9478872091490230914A0225
:10AC900040914B0250914C0260E070E080E291E400
:10ACA0000E949892AB01BC0121E030E08EE99EE069
:10ACB0000E94CC8968E679E08EE99EE00E94A9872F
:10ACC00040914502509146026091470270914802BE
:10ACD00022E030E08EE99EE00E94CD891092640B64
:10ACE0001092630B80E090E00E9468094091450259
:10ACF00050914602609147027091480223E0CE01D4
:10AD000009960E94808C6FE679E0C7C068E779E019
:10AD1000CE0109960E945E8BBE01675F7F4F81EF77
:10AD20009BE00E94A48D811116C06DE779E0CE01F1
:10AD300001960E945E8BBE016F5F7F4F81EF9BE0AB
:10AD40000E94A48D01E0811101C000E0CE010196B6
:10AD50000E94F38A01C001E0CE0109960E94F38AA5
:10AD6000002309F4A8C08091F50B9091F60B06978B
:10AD700008F145E050E061EF7BE0CE0101960E94D2
:10AD80003209BE016F5F7F4F89ED9BE00E94E58B2A
:10AD9000CE0101960E94F38A89ED9BE00E94EE8E1F
:10ADA0000E94B79160933D0270933E0280933F02F0
:10ADB0009093400280916604909167040E949727C7
:10ADC00020E030E048E051E40E94D58F60934102DA
:10ADD0007093420280934302909344026093E50A89
:10ADE0007093E60A8093E70A9093E80A80913D0207
:10ADF00090913E02A0913F02B09140028093ED0AF3
:10AE00009093EE0AA093EF0AB093F00A65E27BE01C
:10AE10008EE99EE00E94788720913D0230913E02AB
:10AE200040913F025091400260E070E080E291E486
:10AE30000E949892AB01BC0121E030E08EE99EE0D7
:10AE40000E94CC8968E679E08EE99EE00E94A9879D
:10AE5000409141025091420260914302709144023C
:10AE600022E030E08EE99EE00E94CD891092640BD2
:10AE70001092630B80E090E00E94680940914102CB
:10AE800050914202609143027091440223E0CE014E
:10AE900009960E94808C62E879E0CE0101960E94BA
:10AEA0005E8BBE01675F7F4FCE0101960E94578D7A
:10AEB0006DEA75E09BC06BE879E0CE0109960E94CF
:10AEC0005E8BBE01675F7F4F81EF9BE00E94A48D88
:10AED000811116C06FE879E0CE0101960E945E8B69
:10AEE000BE016F5F7F4F81EF9BE00E94A48D01E068
:10AEF000811101C000E0CE0101960E94F38A01C0D9
:10AF000001E0CE0109960E94F38A002309F471C082
:10AF100060E0809170040E94E68209E110E0C12C9B
:10AF2000D12C7601809170040E946D82BC0188272B
:10AF300077FD8095982F0E94A1909B01AC01C701DD
:10AF4000B6010E940B8F6B017C016AE070E080E02B
:10AF500090E00E94D7810150110921F720E030E0F4
:10AF600040EA50E4C701B6010E94359220E030E08B
:10AF700040E85AE30E94359220E030E048EC51E48A
:10AF80000E94D58F60931202709313028093140273
:10AF9000909315026093070B7093080B8093090B35
:10AFA00090930A0B1092640B1092630B80E090E078
:10AFB0000E9468094091120250911302609114029C
:10AFC0007091150222E0CE0109960E94808C6CE1FE
:10AFD00078E0CE0101960E945E8BBE01675F7F4FD5
:10AFE000CE0101960E94578D6BEF75E00E94688D2F
:10AFF000E5C163E979E0CE0109960E945E8BBE014E
:10B00000675F7F4F81EF9BE00E94A48D811116C086
:10B0100067E979E0CE0101960E945E8BBE016F5F09
:10B020007F4F81EF9BE00E94A48D01E0811101C060
:10B0300000E0CE0101960E94F38A01C001E0CE013A
:10B0400009960E94F38A002309F473C026E030E0D9
:10B0500044E050E061EF7BE0CE0101960E94458E16
:10B06000BE016F5F7F4F89ED9BE00E94E58BCE01B3
:10B0700001960E94F38A89ED9BE00E94E48E6B01A9
:10B080007C0163E178E0CE0109960E945E8BBE01EF
:10B09000675F7F4F81EF9BE00E943C8EAC014F5F6A
:10B0A0005F4F61EF7BE0CE0101960E943209BE0145
:10B0B0006F5F7F4F89ED9BE00E94E58BCE0101968B
:10B0C0000E94F38ACE0109960E94F38A00918A04B5
:10B0D00010918B0489ED9BE00E94EE8EAB01BC01C8
:10B0E0009801C6010E941C32EBE3FBE02BE03BE041
:10B0F0004191519161917191D9014D935D936D93FE
:10B100007D939D01BBE0E336FB0791F71092640B42
:10B110001092630B80E090E00E94680944E050E0E8
:10B1200061EF7BE0CE0109960E9432096BE979E07C
:10B130003AC16CEB79E0CE0109960E945E8BBE01AC
:10B14000675F7F4F81EF9BE00E94A48D811116C045
:10B1500060EC79E0CE0101960E945E8BBE016F5FCC
:10B160007F4F81EF9BE00E94A48D01E0811101C01F
:10B1700000E0CE0101960E94F38A01C001E0CE01F9
:10B1800009960E94F38A002309F456C080916A044C
:10B1900090916B040E94042460931602709317022E
:10B1A00080931802909319026093D50A7093D60A7F
:10B1B0008093D70A9093D80A80E090E5A3ECB7E497
:10B1C00080931E0290931F02A0932002B09321024D
:10B1D0008093CD0A9093CE0AA093CF0AB093D00A61
:10B1E00068E07BE08EE99EE00E947887409116023D
:10B1F00050911702609118027091190222E030E01C
:10B200008EE99EE00E94CD891092640B1092630B30
:10B2100080E090E00E946809409116025091170268
:10B22000609118027091190222E0CE0109960E94E5
:10B23000808C64EC79E0B7C06FEC79E0CE010996C0
:10B240000E945E8BBE01675F7F4F81EF9BE00E9493
:10B25000A48D811116C063ED79E0CE0101960E94A4
:10B260005E8BBE016F5F7F4F81EF9BE00E94A48DDC
:10B2700001E0811101C000E0CE0101960E94F38A35
:10B2800001C001E0CE0109960E94F38A002309F46F
:10B29000B1C08091F50B9091F60B0497F8F044E063
:10B2A00050E061EF7BE0CE0101960E943209BE01C1
:10B2B0006F5F7F4F89ED9BE00E94E58BCE01019689
:10B2C0000E94F38A89ED9BE00E94EE8E6093220239
:10B2D000709323028093240290932502809122028E
:10B2E00090912302A0912402B09125028093C90A73
:10B2F0009093CA0AA093CB0AB093CC0A60EF7AE08D
:10B300008EE99EE00E9478874091220250912302AC
:10B31000609124027091250222E030E08EE99EE0E7
:10B320000E94CC8980916A0490916B040E9404244D
:10B3300060931A0270931B0280931C0290931D026B
:10B340006093D10A7093D20A8093D30A9093D40A5F
:10B3500066EE7AE08EE99EE00E94788740911A02BC
:10B3600050911B0260911C0270911D0222E030E09E
:10B370008EE99EE00E94CD891092640B1092630BBF
:10B3800080E090E00E94680940911A0250911B02EF
:10B3900060911C0270911D0222E0CE0109960E946C
:10B3A000808C67ED79E0CE0101960E945E8BBE0134
:10B3B000675F7F4FCE0101960E94578DBC018FEDD4
:10B3C0009BE00E94C88BCE0101960E94F38ACE01B9
:10B3D00009960E94F38A6FED7BE0CE0101960E94F0
:10B3E000DD8BCE0101960E948B0FCE0101960E944B
:10B3F000F38AE4C06FED79E0CE0109960E945E8B7E
:10B40000BE01675F7F4F81EF9BE00E94A48D811199
:10B4100016C063EE79E0CE0101960E945E8BBE01FC
:10B420006F5F7F4F81EF9BE00E94A48D01E081114F
:10B4300001C000E0CE0101960E94F38A01C001E044
:10B44000CE0109960E94F38A002309F484C08091FA
:10B45000F50B9091F60B0497F8F044E050E061EFA3
:10B460007BE0CE0101960E943209BE016F5F7F4FE3
:10B4700089ED9BE00E94E58BCE0101960E94F38A44
:10B4800089ED9BE00E94EE8E60931E0270931F0276
:10B49000809320029093210280911E0290911F02BE
:10B4A000A0912002B09121028093CD0A9093CE0A00
:10B4B000A093CF0AB093D00A6EEC7AE08EE99EE0BA
:10B4C0000E94788740911E0250911F0260912002D5
:10B4D0007091210222E030E08EE99EE00E94CC894A
:10B4E00080916A0490916B040E9404246093160278
:10B4F0007093170280931802909319026093D50AF3
:10B500007093D60A8093D70A9093D80A64EC7AE0B5
:10B510008EE99EE00E9478874091160250911702B2
:10B52000609118027091190222E030E08EE99EE0ED
:10B530000E94CD891092640B1092630B80E090E022
:10B540000E946809409116025091170260911802FA
:10B550007091190221CF112389F16FEC76E0CE01B1
:10B5600001960E945E8B61EF7BE0CE0101960E9406
:10B57000578DBC018EE99EE00E94C487CE010196E2
:10B580000E94F38A1BC08BE59CE00E945A6A182F28
:10B590008823F9F06CE67AE08BEE9BE00E94FB8B4F
:10B5A00067EE79E08EE99EE00E94A987612F8EE91F
:10B5B0009EE00E94E487812F0E9403460E94A8819A
:10B5C0006093F70B7093F80B8093F90B9093FA0B41
:10B5D00049C08091D00B882309F44FC00E94A881F4
:10B5E00058EEC52E53E0D52EE12CF12CA701960183
:10B5F0000E947893CA01B9010E949F902091370B55
:10B600003091380B4091390B50913A0B0E940A8FC0
:10B6100020910E0230910F024091100250911102C0
:10B620000E94769118164CF50E94A881A7019601F8
:10B630000E947893CA01B9010E949F906093370BD2
:10B640007093380B8093390B90933A0B8091CD0B0C
:10B650009091CE0B0E94024464E170E080E090E0A3
:10B660000E94D7818091D00B8823E9F064E670E0D6
:10B6700080E090E00E94D78116C00E94A881C0900F
:10B68000F70BD090F80BE090F90BF090FA0B6C19D7
:10B690007D098E099F0968347E4E8105910510F35E
:10B6A0000E94442FDFCFA6960FB6F894DEBF0FBEE0
:10B6B000CDBFDF91CF911F910F91FF90EF90DF9061
:10B6C000CF90BF90AF909F908F9008958091340D50
:10B6D00090E02091350D821B910908952091350D40
:10B6E0008091340D281750F4E22FF0E0EA5CF24F1D
:10B6F000808190E02F5F2093350D08958FEF9FEFAD
:10B700000895E091350D8091340DE81730F4F0E0A4
:10B71000EA5CF24F808190E008958FEF9FEF0895EB
:10B720000895CF92DF92EF92FF920F931F93CF93E2
:10B73000DF937C01CB018A012091100D222389F037
:10B74000EB016B01C40ED51ECC15DD0561F06991CE
:10B75000D701ED91FC910190F081E02DC701199581
:10B76000F3CF642F91D1C801DF91CF911F910F9139
:10B77000FF90EF90DF90CF900895CF93DF931F92CB
:10B78000CDB7DEB769832091100D2223D1F020912F
:10B79000110D203240F021E030E0FC0133832283A0
:10B7A00080E090E014C08091120DE82FF0E0ED5E93
:10B7B000F24F998190838F5F8093120D8093110DCA
:10B7C00004C061E0CE0101965FD181E090E00F906E
:10B7D000DF91CF910895FC011382128248EE53E06D
:10B7E00060E070E044835583668377838EEF99E051
:10B7F0009183808308951092350D1092340D10922C
:10B80000120D1092110D83C081E08093100D609392
:10B81000330D1092120D1092110D0895F5CF0F9364
:10B82000062F21E04091110D63E17DE08091330D01
:10B83000D4D01092120D1092110D1092100D0F9184
:10B8400008958F929F92AF92BF92CF92DF92EF9224
:10B85000FF920F931F93CF93DF93EC01F62ED42E1C
:10B8600048015901EE2009F1CFDF1E2D143008F0F8
:10B8700013E01150B8F0E881F98128E0129FB0017F
:10B880001124A501940104C0569547953795279535
:10B890006A95D2F7CA01B9010190F081E02DCE017D
:10B8A0001995E7CF60E0CE01BADF4D2D413208F0A7
:10B8B00040E22C2D66E37DE08F2D47D01092350DB0
:10B8C0008093340DDF91CF911F910F91FF90EF90F6
:10B8D000DF90CF90BF90AF909F908F900895CF92C0
:10B8E000EF920F931F93C22EE12C00E010E098011D
:10B8F000A8DF1F910F91EF90CF90089521E0EFCF37
:10B9000021E0EDCF61E08BCF84E09DE064CF109229
:10B91000C30D81E08093C10D1092C00D61E084E100
:10B920000E941F8361E085E10E941F83E9EBF0E044
:10B9300080818E7F808380818D7F808388E4809367
:10B94000B80085E48093BC000895413208F043C0FC
:10B950009091C30D9111FCCF91E09093C30D209372
:10B96000C10D2FEF2093560D10929B0D240F2093A5
:10B970009A0D9093C20D9091C20D880F892B8093E0
:10B98000C20D8091C00D813061F41092C00D809184
:10B99000C20D8093BB008091BC0083FDF8CF85EC85
:10B9A00001C085EE8093BC008091C30D8130E1F32E
:10B9B00080919B0D841710F440919B0D2CE93DE084
:10B9C000FB01D9018A2F821B841718F48D91819372
:10B9D000F9CF842F089580E008950F93413208F045
:10B9E0004AC09091C30D9111FCCF92E09093C30D8A
:10B9F0000093C10D9FEF9093560D10929B0D4093B5
:10BA00009A0DFB016CE97DE0DB019A2F961B9417E0
:10BA100018F491919D93F9CF1092C20D9091C20D9F
:10BA2000880F892B8093C20D8091C00D813061F405
:10BA30001092C00D8091C20D8093BB008091BC001C
:10BA400083FDF8CF85EC01C085EE8093BC002223F6
:10BA500021F08091C30D8230E1F38091560D8F3F2C
:10BA600061F08091560D803251F08091560D8033F7
:10BA700041F483E007C081E005C080E003C082E0BC
:10BA800001C084E00F910895613298F42091C30DB4
:10BA9000243089F46093780DFC018AE79DE0DC0195
:10BAA0002A2F281B261718F421912D93F9CF80E017
:10BAB000089581E0089582E0089585ED8093BC00AB
:10BAC0008091BC0084FDFCCF1092C30D089585ECDD
:10BAD0008093BC001092C30D08951F920F920FB671
:10BAE0000F9211240BB60F922F933F934F935F93B6
:10BAF0006F937F938F939F93AF93BF93EF93FF9336
:10BB00008091B900887F803609F49DC070F5883235
:10BB100009F45CC090F4803109F455C038F48823EE
:10BB200009F4F3C0883009F44EC0F2C0883109F43A
:10BB30004DC0803209F45EC0EBC0803409F469C0A6
:10BB400050F4803309F456C0883309F0E1C0809383
:10BB5000560DBDDFDDC0803509F44FC0883509F4CE
:10BB60005DC0883409F0D4C0D2C0883909F4C3C09C
:10BB7000A8F4883709F467C038F4883609F463C03C
:10BB8000803709F460C0C4C0883809F4B4C0803973
:10BB900009F45FC0803809F0BBC05BC0803B09F48A
:10BBA00082C038F4803A09F466C0883A09F47BC050
:10BBB000AFC0803C09F4A3C0883C09F4A0C0883B16
:10BBC00009F486C0A5C08091C20D10C090919B0D54
:10BBD00080919A0D981770F5E0919B0D81E08E0F82
:10BBE00080939B0DF0E0E456F24F80818093BB0080
:10BBF00085EC82C08093560D8AC0E0919B0D81E058
:10BC00008E0F80939B0D8091BB00F0E0E456F24FC5
:10BC1000808390919B0D80919A0D6AC0E0919B0D5D
:10BC200081E08E0F80939B0D8091BB00F0E0E45685
:10BC3000F24F80838091C10D811169C081E08093B2
:10BC4000C00D84EA5DC083E08093C30D1092570D50
:10BC5000CFCF8091570D803208F04DC0E091570D45
:10BC600081E08E0F8093570D8091BB00F0E0E85A81
:10BC7000F24F8083BDCF2BDF8091570D803230F49F
:10BC8000E091570DF0E0E85AF24F10826091570DA5
:10BC900070E0E091BC0DF091BD0D88E59DE0199537
:10BCA0001092570D35C084E08093C30D1092790D2A
:10BCB0001092780DE091BE0DF091BF0D1995809115
:10BCC000780D811105C081E08093780D10927A0D76
:10BCD000E091790D81E08E0F8093790DF0E0E658C8
:10BCE000F24F80818093BB009091790D8091780D07
:10BCF000981708F47DCF85E88093BC0009C085ECD7
:10BD00008093BC001092C30D03C01092560DD5DE77
:10BD1000FF91EF91BF91AF919F918F917F916F9123
:10BD20005F914F913F912F910F900BBE0F900FBEDF
:10BD30000F901F90189508950895DC01ED91FC91E6
:10BD40000284F385E02D41E0199581E090E00895AB
:10BD5000FC01138212822EE03AE0318320830895A1
:10BD6000DC01ED91FC910084F185E02D6FEF1994D9
:10BD7000DC01ED91FC910284F385E02D40E0199403
:10BD800061E0F6DF80ED97E00C94FD81CF93DF93C7
:10BD9000CDB7DEB728970FB6F894DEBF0FBECDBF84
:10BDA0001D8220E42E8334E13F8334E538871982F5
:10BDB0002A8320E12B8320E52C83FC012781421775
:10BDC00010F04FEF420FFC01308550E0FE01E40F10
:10BDD000F51F303121F4243011F4218101C0258177
:10BDE000260F2068622F28960FB6F894DEBF0FBE8C
:10BDF000CDBFDF91CF91BCCFFC0165816B7F6583A7
:10BE00006860B6CFFC016581262F246025836C60B5
:10BE1000AFCFCF93DF93EC01423018F08C81886074
:10BE20008C834F836887222329F0413019F48C8159
:10BE300084608C8364E670E080E090E00E94D781AB
:10BE40006C8164FD31C0E881F9810284F385E02DC5
:10BE500042E063E0CE01199584E991E10E94FD8101
:10BE6000E881F9810284F385E02D42E063E0CE01B0
:10BE7000199586E990E00E94FD81E881F9810284AC
:10BE8000F385E02D42E063E0CE01199586E990E06C
:10BE90000E94FD81E881F9810284F385E02D42E072
:10BEA00062E0CE01199513C06062CE0161DF84E9C2
:10BEB00091E10E94FD816C816062CE0159DF86E9CB
:10BEC00090E00E94FD816C816062CE0151DF86E9C5
:10BED00090E00E94FD816C816062CE0149DF8CE3BD
:10BEE00090E00E94FD8184E08D83CE018BDFCE0146
:10BEF00047DF82E08E8366E0CE013ADFCE01DF913C
:10BF0000CF912ECFCF92DF92FF920F931F93CF93BB
:10BF1000DF931F921F92CDB7DEB78C01677088E068
:10BF2000689FB00111246064C80149835A8320DFEF
:10BF30008EE190E00E94FD814981C42E5A81D52E68
:10BF4000F12CD6016D916D01D801ED91FC9101901C
:10BF5000F081E02DC801199588E290E00E94FD81F2
:10BF6000F394B8E0FB12EDCF0F900F90DF91CF91DB
:10BF70001F910F91FF90DF90CF900895FC0186896B
:10BF80008F3F79F021853285662319F0232B31F418
:10BF900003C02130310511F461E001C060E00C9470
:10BFA0001F830895FF920F931F93CF93DF93EC01AC
:10BFB000F62E8A0161E08F2D0E94E682FE8A1A87A2
:10BFC0000987E881F9810084F185E02D60E0CE01E8
:10BFD000DF91CF911F910F91FF9019946F927F92F3
:10BFE0008F92AF92CF92EF92FF920F931F93CF93C6
:10BFF000DF93CDB7DEB73C01F62EFC0143872487E3
:10C000000587E686C786A08A818A8F85828B888984
:10C01000838B8989848B8A89858B00E010E0F3010A
:10C02000E00FF11F61E086850E94E6820F5F1F4FDF
:10C0300004301105A1F7FF2069F061E0F301838569
:10C040000E94E682F30184858F3F99F061E00E94AF
:10C05000E6820FC000E010E0F301E00FF11F61E0A5
:10C0600082890E94E6820F5F1F4F04301105A1F7FD
:10C07000E4CF61E0F30185850E94E682FF2019F09C
:10C08000F301148203C080E1F301848360E0F301D3
:10C0900083850E941F8360E0F30185850E941F83D2
:10C0A000F30184858F3F19F060E00E941F838FEFBA
:10C0B000F301868B12861186DF91CF911F910F912C
:10C0C000FF90EF90CF90AF908F907F906F900895FA
:10C0D0006F927F928F92AF92CF92EF920F93CF9306
:10C0E000DF9300D0CDB7DEB73C012B834A83698351
:10C0F0002FDE8EE19AE0F301918380831F921F92DD
:10C100001F921F928C2CAE2CC02E2B81E22E4A81C6
:10C11000042F2FEF6981462F61E0C3015FDF0F908D
:10C120000F900F900F900F900F900F90DF91CF9185
:10C130000F91EF90CF90AF908F907F906F90089578
:10C14000CF93DF93EC0161E08D850E941F8360E057
:10C150008D85DF91CF910C941F83CF92DF92EF9268
:10C16000FF920F931F93CF93DF931F92CDB7DEB74C
:10C170008C01C12CD12CE62EF12CC416A0F4B701F1
:10C180000C2C02C0759567950A94E2F76170F8016E
:10C19000EC0DFD1D868549830E941F838FEFC81A11
:10C1A000D80A4981EACFC8010F90DF91CF911F9142
:10C1B0000F91FF90EF90DF90CF90C2CF0F931F931E
:10C1C000CF93DF93EC01162F042F61E0413009F08B
:10C1D00060E08B850E941F838C858F3F19F060E0A3
:10C1E0000E941F83023079F08C8184FF02C048E0F6
:10C1F0000BC0612F70E084E0759567958A95E1F733
:10C2000044E0CE01AADF44E0612FCE01DF91CF915F
:10C210001F910F91A2CF0895CF92DF92EF92FF92DC
:10C22000FC0185899689481B590B61097109A3890D
:10C23000B4899A01AB010E94BC936B017C018FE031
:10C24000F594E794D794C7948A95D1F76585768558
:10C25000882777FD8095982F2BE0660F771F881F22
:10C26000991F2A95D1F727853089442737FD4095B6
:10C27000542F2C0D3D1D4E1D5F1D0E949A932C0DB9
:10C280003D1D4E1D5F1DCA01B901FF90EF90DF906B
:10C29000CF9008951F93CF93DF931F92CDB7DEB752
:10C2A000162F67E770E084E09DE04983B7DA612FDD
:10C2B00084E09DE062DA4981642F84E09DE05DDAEC
:10C2C00084E09DE00F90DF91CF911F911BCBCF9326
:10C2D000C62F67E770E084E09DE0A0DA6C2F84E071
:10C2E0009DE04BDA84E09DE00DDB67E770E084E0E1
:10C2F0009DE094DA41E050E067E770E084E09DE083
:10C30000FFDA84E09DE0EAD9C82F84E09DE0FADA04
:10C310008C2FCF910895CF93DF93C62F67E770E0FE
:10C3200084E09DE07BDA6C2F84E09DE026DA84E0F7
:10C330009DE0E8DA67E770E084E09DE06FDA42E0D4
:10C3400050E067E770E084E09DE0DADA84E09DE0A9
:10C35000C5D9D82F80E0C82F84E09DE0BFD9C82B75
:10C36000D92B84E09DE0CEDACE01DF91CF91089504
:10C37000CF93DF93EC01643008F063E0688384E0DE
:10C380009DE039DA60EDCE01A2DF853509F039C0D4
:10C390006AEACE01C0DF9A8389836CEACE01BBDFF3
:10C3A0009C838B836EEACE01B6DF9E838D8360EB28
:10C3B000CE01B1DF9A8B898B62EBCE01ACDF9C8B17
:10C3C0008B8B64EBCE01A7DF9E8B8D8B66EBCE0152
:10C3D000A2DF98878F8368EBCE019DDF9A878987DC
:10C3E0006AEBCE0198DF9C878B876CEBCE0193DFE5
:10C3F0009E878D876EEBCE018EDF988B8F8781E0D5
:10C4000001C080E0DF91CF910895CF93DF93EC01DD
:10C410004EE264EF3FDF65E070E080E090E00E9474
:10C42000D78166EFCE01DF91CF9175CFCF93DF93A8
:10C43000EC01EBDFAC0160E070E0CE01EDDE685FA7
:10C440007F4F8F4F9F4F34E09595879577956795F0
:10C450003A95D1F70E94A19020E030E040E251E40B
:10C460000E94D58FDF91CF910895CF92DF92EF9206
:10C47000FF92CF93DF93EC0148814295440F440F24
:10C48000407C4C5C64EF06DF8881811105C065E06B
:10C4900070E080E090E012C0813029F468E070E044
:10C4A00080E090E00BC0823029F46EE070E080E024
:10C4B00090E004C06AE170E080E090E00E94D781E3
:10C4C00066EFCE0128DF6C01E12CF12CFE2CED2C67
:10C4D000DC2CCC2468EFCE01FADEA7019601282BD4
:10C4E000CA01B901488128E030E0241B310904C0A9
:10C4F00096958795779567952A95D2F7DF91CF9195
:10C50000FF90EF90DF90CF9008952F923F924F923F
:10C510005F926F927F928F929F92AF92BF92CF92D3
:10C52000DF92EF92FF920F931F93CF93DF93CDB7DC
:10C53000DEB72A970FB6F894DEBF0FBECDBF9A873D
:10C54000898763DF8C0189859A858FDF6D837E8380
:10C550008F839887A80160E070E089859A855CDE0A
:10C560004B015C0180EA881A8FE0980AA108B108A3
:10C57000A5019401C501B4010E9442932B013C0125
:10C580000CE075946794579447940A95D1F7A98560
:10C59000BA8511962D903C9012971C9115960D908E
:10C5A000BC91A02D0E94C6936B017C018DE0F59497
:10C5B000E794D794C7948A95D1F7E985FA85A7813E
:10C5C000B085A30192010E94C693BB2797FDB09549
:10C5D000AB2FC80ED91EEA1EFB1EF2E0CF0ED11CF7
:10C5E000E11CF11C32E0F594E794D794C7943A9596
:10C5F000D1F780E8D80EE11CF11CE985FA85A18904
:10C60000B289A70196010E94BC93DC01CB014FE0E7
:10C61000B695A795979587954A95D1F789839A837B
:10C62000AB83BC836101EE24D7FCE094FE2C52E086
:10C63000CC0CDD1CEE1CFF1C5A95D1F7A185B285F0
:10C64000A30192010E94C6932B013C016BE07594FB
:10C650006794579447946A95D1F7A381B481A50153
:10C6600094010E94C693EBE0959587957795679521
:10C67000EA95D1F7460E571E681E791EC40CD51CCC
:10C68000E61CF71C012E04C0CC0CDD1CEE1CFF1CAC
:10C690000A94D2F792E0C90ED11CE11CF11CC7012B
:10C6A000B60124E030E040E050E00E949A938D8192
:10C6B0009E81AF81B885821B930BA40BB50B9C01A7
:10C6C000AD0160E573EC80E090E004C0969587953D
:10C6D000779567951A95D2F70E94429397FD0DC002
:10C6E000660F771F881F991F29813A814B815C81D2
:10C6F0000E94789349015A010CC029813A814B81EB
:10C700005C810E94789349015A01880C991CAA1CEB
:10C71000BB1C9927B7FC9A958B2D7A2D692D9B010F
:10C72000AC010E9442939B01AC01AEEDBBE00E94C4
:10C73000BC936C01FF24D7FCF094EF2CA3E4B3EE80
:10C74000A50194010E94C893BB2797FDB095AB2F1C
:10C75000C80ED91EEA1EFB1E9FECC90E9EE0D91E14
:10C76000E11CF11CA4E0F594E794D794C794AA9532
:10C77000D1F7C80CD91CEA1CFB1CC701B6012A96CC
:10C780000FB6F894DEBF0FBECDBFDF91CF911F91E2
:10C790000F91FF90EF90DF90CF90BF90AF909F9060
:10C7A0008F907F906F905F904F903F902F90089563
:10C7B0008F929F92AF92BF92CF92DF92EF92FF92B1
:10C7C000CF93DF9300D01F92CDB7DEB74A015B0154
:10C7D0009CDE6B017C0120E03AE24DE257E4C501AA
:10C7E000B4010E94D58F9B01AC0160E070E080E84D
:10C7F0009FE30E940A8F26EF38E248EA50E40E9445
:10C8000098929B01AC01C701B60129833A834B83FF
:10C810005C830E94A19029813A814B815C810E94B6
:10C82000D58F0E946E900F900F900F900F90DF9118
:10C83000CF91FF90EF90DF90CF90BF90AF909F90FF
:10C840008F900895CF93DF9300D01F92CDB7DEB7BE
:10C850009A01AB0129833A834B835C8356DE0E94A5
:10C86000A19029813A814B815C810E94D58F21E082
:10C870003EED42E45EE30E9498929B01AC0160E0D1
:10C8800070E080E89FE30E940A8F20E03AE24DE2E8
:10C8900057E40E9435920F900F900F900F90DF9108
:10C8A000CF910895FB016181828170E0762F662728
:10C8B000680F711D882777FD8095982F0E94A190A1
:10C8C00020E030E040E85DE30E94359223E333E965
:10C8D00048E853E40C940A8F089521E06227FC0194
:10C8E00080810C941F83CF93DF93EC01862F6883A4
:10C8F00049832A8361E00E94E68261E088810E9488
:10C900001F8360E089810E94E68260E08A810E9444
:10C91000E68261E089810E941F8361E08A810E9432
:10C920001F8360E0CE01DF91CF91D7CFFB018181E2
:10C930009081890F9281890F9381981304C081E0BF
:10C9400094819D3009F080E008952F923F924F929C
:10C950005F926F927F928F929F92AF92BF92CF928F
:10C96000DF92EF92FF920F931F93CF93DF9300D04C
:10C9700000D0CDB7DEB78C013B014E830E94A88169
:10C980001B012C0180ED280E87E0381E411C511C34
:10C9900061E0C801A2DFFE0131966F014E01F6E0B1
:10C9A0008F0E911CF60185E011928A95E9F77601C8
:10C9B00027E0A22EB12CF80181810E9454830197B7
:10C9C00039F40E94A881621573058405950598F3D2
:10C9D000F80181810E945483892B39F40E94A88137
:10C9E000621573058405950598F3F80182810E940C
:10C9F0005483892B59F0F701208181E090E00A2CC3
:10CA000001C0880F0A94EAF7282B2083F1E0AF1ABF
:10CA1000B10888F69FEFE91AF90AE814F90441F61B
:10CA20000E94A881621573058405950540F060E0B9
:10CA3000C80153DF20E030E040EC5FE72EC0898181
:10CA4000EE818E13AFCFB601C80170DF882309F4E1
:10CA5000A9CF60E0C80141DFB601C80123DFFB01B7
:10CA6000DC016A946728B9F420E030E040E151E449
:10CA7000BF01CD010E94359220E030E040EA50E451
:10CA80000E94D58F20E030E040E052E40E940B8FFE
:10CA90009B01AC0102C09F01AD01B901CA012696FC
:10CAA0000FB6F894DEBF0FBECDBFDF91CF911F91BF
:10CAB0000F91FF90EF90DF90CF90BF90AF909F903D
:10CAC0008F907F906F905F904F903F902F90089540
:10CAD00046E63BCF4CE439CFFF920F931F93CF93A1
:10CAE000DF93FC010081C181D281F8948981F02E0D
:10CAF000F0948F21898378941DE7115029F182E009
:10CB000090E00E94FD8188818023B9F3F8948A81A6
:10CB10008F218A838981802B8983789480EE91E0AC
:10CB20000E94FD81F89489818F21898386E490E0B9
:10CB30000E94FD818881802311E009F010E0789443
:10CB40008AE991E00E94FD81812FDF91CF911F91B1
:10CB50000F91FF9008951F93CF93DF93FC011081F5
:10CB6000C181D281912F909560FF12C0F8948A8183
:10CB700089238A838981812B89838AE090E00E94BE
:10CB8000FD818A81812B8A83789487E390E011C0AC
:10CB9000F8948A8189238A838981812B898381E41E
:10CBA00090E00E94FD818A81812B8A83789485E0C0
:10CBB00090E0DF91CF911F910C94FD810F931F9313
:10CBC000CF93DF93FC011081C181D281F8948981D8
:10CBD000812B89838A81012F009580238A8383E0BA
:10CBE00090E00E94FD818981802389838AE090E022
:10CBF0000E94FD81C881789485E390E00E94FD81C8
:10CC00001C2381E009F480E0DF91CF911F910F9107
:10CC10000895CF92DF92EF92FF920F931F93CF93DD
:10CC2000DF931F92CDB7DEB76C01E62E08E010E06F
:10CC3000FF24F39461E09F2D9E2109F460E0C6017A
:10CC4000498389DFFF0C0150110949810115110544
:10CC500089F7411115C0F894D6011196ED91FC9118
:10CC6000129791818C918095892381831196ED9102
:10CC7000FC91129792818C9180958923828378947C
:10CC80000F90DF91CF911F910F91FF90EF90DF9068
:10CC9000CF900895EF92FF920F931F93CF93DF935E
:10CCA0008C01C8E0D0E0F12CEE24E394C80186DFCB
:10CCB0008111FE28EE0C2197C9F78F2DDF91CF91BE
:10CCC0001F910F91FF90EF900895CF92DF92FF9206
:10CCD0000F931F93CF93DF931F92CDB7DEB78C01D5
:10CCE000F62E40E065E5798394DFCF2C7981D72E4D
:10CCF00088E0F82EF60161916F0140E0C80189DFFC
:10CD0000FA94C1F70F90DF91CF911F910F91FF908F
:10CD1000DF90CF90089540E06CEC7BCFFC01138650
:10CD20001586148627E030E0DF01A20FB31F1396AB
:10CD30001C922115310519F021503109F5CF0895C4
:10CD40001F93CF93DF93EC01162F60E0812F0E9499
:10CD5000E682612F70E0FB01EF56F34FE491E88328
:10CD6000FB01E952F34FE491F0E0EE0FFF1FE35EA9
:10CD7000F24F859194919A838983CE01DF91CF916F
:10CD80001F91CCCFAF92BF92CF92DF92EF92FF92E2
:10CD90000F931F93CF93DF931F92CDB7DEB75C0144
:10CDA000D62EE72EFC01158511115EC0498394DE55
:10CDB0004981811105C0F5011386158614866DC061
:10CDC000442319F040E060EF02C040E06CEEC50182
:10CDD00020DF01E0F12CC12C11E0C501EFDE682F4E
:10CDE000C5016983EBDE6981613019F48130B9F4E2
:10CDF00032C02F2D30E068131BC0F5018385181752
:10CE000030F4E20FF31F8381802349F402C0181726
:10CE100031F060E0193058F4F501148708C0F501CD
:10CE2000EF0DF11D8381802B838361E009C0C12E4A
:10CE3000F501E20FF31F8381902F9095892383835F
:10CE4000C50189DE1F5F000F11F4F39401E0F7E0E4
:10CE5000FF1508F0C2CF113438F0F501C386C110B8
:10CE600009C081E0858706C0F50113861586148602
:10CE700010E013C0F50183818823B1F3ED2DFE2D61
:10CE800080E090E0D501A80FB91F13962C91219353
:10CE9000019688309105B1F711E0812F0F90DF9155
:10CEA000CF911F910F91FF90EF90DF90CF90BF90A7
:10CEB000AF900895DC0180E0615088F09D91982743
:10CEC000E92FEF70F0E0E55DF34F249192959F70AC
:10CED000E92FF0E0E55CF34F84918227EDCF0895D0
:10CEE000FC0110821482138215820895862F642F0C
:10CEF0000C94E682862F642F0C941F83862F0C944B
:10CF000054834F925F926F927F928F929F92AF92D3
:10CF1000BF92CF92DF92EF920F93CF93DF93EC010A
:10CF20004B013A0159010296DBDF8EE29AE09983C8
:10CF300088836E018CE1C80ED11C26018CE3480E5B
:10CF4000511CC601CDDF86E0C80ED11CC414D50427
:10CF5000C1F7FE01EE59FF4F718260823296B182B5
:10CF6000A082329600833196E08237979182808248
:10CF700038968AE090E091838083329684EF91E046
:10CF8000918380833396118210827197108211826F
:10CF900012821382C459DF4F1882DF91CF910F9113
:10CFA000EF90DF90CF90BF90AF909F908F907F9049
:10CFB0006F905F904F9008952F923F924F925F92A3
:10CFC0006F927F928F929F92AF92BF92CF92DF9299
:10CFD000EF92FF920F931F93CF93DF93CDB7DEB7FE
:10CFE00028970FB6F894DEBF0FBECDBF98878F830A
:10CFF000F12C4C0186E6880E911C0F8118850E5984
:10D000001F4FD4018C91F816A0F4AF81B8858D9193
:10D010009C91F801A081B181AF0DB11DFC0120816F
:10D02000318142E06C918F819885F9011995F394D3
:10D03000E8CF512CEF81F885E959FF4FFA83E98356
:10D040000F8118850C591F4FC12CD12C7601C39428
:10D050008F8198858E599F4F9C838B83A981BA813C
:10D060008C91581608F088C0A52CB12CAF81B885DA
:10D070008D919C91F801A081B181AA0DBB1DFC018D
:10D080002081318141E06C918F819885F90119955A
:10D09000AF81B8858D919C91F801A081B181AA0DD5
:10D0A000BB1DFC012281338140E06C918F8198850A
:10D0B000F9011995D701C601052C04C0880F991FE5
:10D0C000AA1FBB1F0A94D2F79C011C012094309424
:10D0D000412CD4018C91EF81F88540815181481613
:10D0E00048F5642C712CEB81FC81A081B181A60DE7
:10D0F000B71DFA01448155816C918F8198852D83EC
:10D100003E83FA011995660C771C2D813E81EF81D3
:10D11000F885E60DF71D892B29F480859185822BF2
:10D12000932B04C0808591858221932191878087EC
:10D130004394CFCFF801A081B181AA0DBB1DFA01A4
:10D140002281338141E06C918F819885F901199595
:10D15000AF81B8858D919C91F801A081B181AA0D14
:10D16000BB1DFC012081318140E06C918F8198854D
:10D17000F9011995539472CF28960FB6F894DEBF33
:10D180000FBECDBFDF91CF911F910F91FF90EF9018
:10D19000DF90CF90BF90AF909F908F907F906F90D7
:10D1A0005F904F903F902F900895FC0180E090E0B9
:10D1B000258D368D2617370739F0019636968A3039
:10D1C0009105B1F78FEF9FEF0895DC0126E0629F94
:10D1D000A00DB11D112490965C934E935F9721E0B2
:10D1E00091962C939197FC01E459FF4F2081319641
:10D1F0000190F081E02D222331F0309749F0611148
:10D2000007C0DC0102C0309719F05C968C9119942C
:10D210000895CF92DF92FF920F931F93CF93DF93E6
:10D220001F92CDB7DEB76C01F62EFC0186E0689F39
:10D23000E00DF11D112411A2878D90A1813091057F
:10D24000E9F01CF4892B51F044C08230910591F132
:10D25000039709F03EC040E050E030C04423C9F1DC
:10D2600041E050E0C601B1DF0E94A881F601E85A12
:10D27000FF4F60837183828393832BC049830E9415
:10D28000A881F601E85AFF4F008111812281338184
:10D29000601B710B820B930B72960081118120E051
:10D2A00030E04981061717072807390718F442E0CC
:10D2B00050E004C041110DC043E050E06F2DC601A5
:10D2C0000F90DF91CF911F910F91FF90DF90CF9042
:10D2D0007CCF0F90DF91CF911F910F91FF90DF9046
:10D2E000CF9008952F923F924F925F926F927F92CC
:10D2F0008F929F92AF92BF92CF92DF92EF92FF9266
:10D300000F931F93CF93DF931F92CDB7DEB71C010E
:10D31000FC014AE08FEF9FEF278D30A1232B21F4F2
:10D32000148E968F858F11A2415036964111F4CFFD
:10D33000712C610126E6C20ED11C510187E6A80EB0
:10D34000B11C4101A0E68A0E911C46E0442ED60194
:10D350008C91781608F053C0612C8101070D111DC6
:10D36000070D111D085F1F4FF501E0806E1408F0D6
:10D3700044C0F80140815181062C02C05695479562
:10D380000A94E2F741707E9C70011124E60CF11CB6
:10D39000D401ED91FC91EE0DFF1D5080B701C1014C
:10D3A000498303DF498197FD02C0682F1BC00196A6
:10D3B00011F5442301F180E090E060E070E0F101BC
:10D3C000E80FF91F248D211110C0469EF001479EE1
:10D3D000F00D1124E20DF31D548EF68EE58E10A291
:10D3E000178E41E0C10115DF06C06F5F7F4F0696C3
:10D3F0006A30710521F76394B7CF7394A8CF20E00A
:10D4000030E080E0F101E20FF31F91A1911181E082
:10D410002A5F3F4F2C333105A9F70F90DF91CF9151
:10D420001F910F91FF90EF90DF90CF90BF90AF9042
:10D430009F908F907F906F905F904F903F902F9034
:10D440000895CF92DF92EF92FF920F931F93CF93A5
:10D45000DF938C010E94A881E801C45ADF4FC88085
:10D46000D980EA80FB806C197D098E099F09F8013B
:10D47000E859FF4FC080D180E12CF12CC616D706A9
:10D48000E806F90660F4C80197DDC8012BDF182F04
:10D490000E94A881688379838A839B8301C010E0FE
:10D4A000812FDF91CF911F910F91FF90EF90DF902F
:10D4B000CF9008950F931F93CF93DF93EC018C01CE
:10D4C00004591F4F81E0F8018083CE01BADF882321
:10D4D00049F089A1882331F08F8D98A1019711F42B
:10D4E0008C8D03C0F801108280E0DF91CF911F91F5
:10D4F0000F91089520EF39E0FC01318320830895D6
:10D5000020EF39E0FC01318320830C94088F0F93C6
:10D510001F93CF93DF938C01EB0188E2FB01119203
:10D520008A95E9F74BE050E064E37AE0CE010E948F
:10D53000A4961B8641E050E060E070E04C875D8778
:10D540006E877F87F801458956896789708D488B7A
:10D55000598B6A8B7B8B42E050E060E070E04C8B33
:10D560005D8B6E8B7F8B1CA21DA21EA21FA240E0B2
:10D5700050E068E474E4488F598F6A8F7B8F40E0F5
:10D5800050E068E474EC4C8F5D8F6E8F7F8F4DECB4
:10D590005CEC6CE47EE348A359A36AA37BA3DF9110
:10D5A000CF911F910F91089520E43AE0FC0131835F
:10D5B0002083458B568B678B708F0895CF93DF93B5
:10D5C0001F921F92CDB7DEB784E09DE02A83498386
:10D5D0000E94045C4981642F84E09DE00E94BD5B51
:10D5E0002A81622F84E09DE00E94BD5B84E09DE083
:10D5F0000F900F90DF91CF910C94825C0F931F934B
:10D60000CF93DF938C01EB01262F41E06EE1D6DF53
:10D61000F801D483C383C038D10509F45BC0DCF4BE
:10D62000C034D105A9F1C036D10509F442C0A09794
:10D6300009F08AC080E090E8A9E8B4E48093A104EE
:10D640009093A204A093A304B093A40480E090E07C
:10D65000A5E7B4E471C0C03CD10509F44CC0C03E9C
:10D66000D10509F459C0C03AD10509F06DC080E078
:10D6700090E0A8ECB3E48093A1049093A204A0935B
:10D68000A304B093A40480E090E0AFE7B3E454C0F7
:10D6900080E090ECA5E5B4E48093A1049093A2040B
:10D6A000A093A304B093A40480E090E0AEE3B4E4BC
:10D6B00043C080E090E8A7E2B4E48093A104909393
:10D6C000A204A093A304B093A40480E090E0A6E198
:10D6D000B4E432C080E090E0A1EEB3E48093A10412
:10D6E0009093A204A093A304B093A40480E090E0DC
:10D6F000A8ECB3E421C080E090E0A5EAB3E4809315
:10D70000A1049093A204A093A304B093A40480E086
:10D7100090E8A3E9B3E410C080E090E0A6E6B3E4AB
:10D720008093A1049093A204A093A304B093A404B3
:10D7300080E090E0ADE4B3E480939D0490939E0478
:10D74000A0939F04B093A004DF91CF911F910F91FC
:10D750000895CF93DF93EC0184E09DE00E94FB5B92
:10D7600020E042E06EE1CE0129DF60E270E0CE0110
:10D7700045DF81E0DF91CF9108956F927F928F9284
:10D780009F92AF92BF92CF92DF92EF92FF920F9350
:10D790001F93CF93DF93EC016EE184E09DE00E9444
:10D7A000045CE091040DF091050D0190F081E02DF5
:10D7B00063E084E09DE0199584E09DE00E94825C36
:10D7C00046E06EE184E09DE00E947E5C84E09DE0A6
:10D7D0000E94665B0697D4F384E09DE00E946E5B36
:10D7E000682E84E09DE00E946E5B782E84E09DE0D0
:10D7F0000E946E5BC82E84E09DE00E946E5BD82E76
:10D8000084E09DE00E946E5B882E84E09DE00E9493
:10D810006E5B982EB62CA12CA728B501882777FD22
:10D820008095982F0E94A1906D837E838F83988727
:10D83000F82CE12CE928B701882777FD8095982FEF
:10D840000E94A19069877A878B879C871C2D00E0B6
:10D850000D29B801882777FD8095982F0E94A19007
:10D860006D877E878F87988B198A1A8A1B8A1C8AF4
:10D87000DF91CF911F910F91FF90EF90DF90CF90AC
:10D88000BF90AF909F908F907F906F900895CF92B0
:10D89000DF92EF92FF920F931F93CF93DF938C0150
:10D8A000EB0184E2FB0111928A95E9F7C80165DF7B
:10D8B00084E290E0A0E0B0E088839983AA83BB83F0
:10D8C000F80185899689A789B08D8C839D83AE8365
:10D8D000BF8382E090E0A0E0B0E088879987AA87C4
:10D8E000BB87188A198A1A8A1B8AC090A104D09013
:10D8F000A204E090A304F090A404A701960165811E
:10D900007681878190850E94D58F20E030E048ECB9
:10D9100052E40E9435926C8B7D8B8E8B9F8BA7017E
:10D920009601F80161857285838594850E94D58F63
:10D9300020E030E048EC52E40E943592688F798F05
:10D940008A8F9B8F20919D0430919E0440919F046B
:10D950005091A004F80165857685878590890E949D
:10D96000D58F20E030E048EC52E40E9435926C8F75
:10D970007D8F8E8F9F8F81E0DF91CF911F910F91CF
:10D98000FF90EF90DF90CF900895FC0181E08083BD
:10D99000118243EC5BEA66E77BE342835383648353
:10D9A000758348ED5BE666E77BE3468357836087D4
:10D9B000718742EF54EE64E67BE3428753876487C6
:10D9C00075870895FC01DB014D915D916D917C910E
:10D9D0001397428353836483758314964D915D91AD
:10D9E0006D917C911797468357836087718718964E
:10D9F0004D915D916D917C911B9742875387648710
:10DA000075870895CF93DF93FC01EB014281538129
:10DA100064817581488359836A837B8346815781FA
:10DA2000608571854C835D836E837F83828593855A
:10DA3000A485B58588879987AA87BB87DF91CF9111
:10DA400008950F931F93CF93DF93082F6DEC75E02C
:10DA50008EE99EE00E94A987C7E0D0E010E0B801FF
:10DA60000C2E02C0759567950A94E2F761707727CE
:10DA700042E050E08EE99EE00E949388219778F77B
:10DA8000DF91CF911F910F9108951F93CF93DF9353
:10DA90001F92CDB7DEB7162F63E570E084E09DE0FE
:10DAA00049830E940E5C612F84E09DE00E94BD5B73
:10DAB0004981642F84E09DE00E94BD5B84E09DE08D
:10DAC0000F90DF91CF911F910C94825CCF93DF93E5
:10DAD000EC0184E09DE00E94FB5B40E06DE2CE0142
:10DAE000D4DF40E16DE2CE01D0DF48E06DE2CE014F
:10DAF000DF91CF91CACF6F3F710534F4AB0177FF4F
:10DB000005C040E050E002C04FEF50E06DE1BDCFF6
:10DB1000EF92FF921F93CF93DF931F92CDB7DEB7A3
:10DB20007C01142F462F6EE12983AFDF412F6FE177
:10DB3000C701ABDF2981422F60E2C7010F90DF915F
:10DB4000CF911F91FF90EF90A0CF6F3F710534F4FC
:10DB5000AB0177FF05C040E050E002C04FEF50E05E
:10DB600061E293CF462F62E290CF6F3F710534F4AC
:10DB7000AB0177FF05C040E050E002C04FEF50E03E
:10DB800063E283CF6F3F710534F4AB0177FF05C0CB
:10DB900040E050E002C04FEF50E064E276CF6F3FCC
:10DBA000710534F4AB0177FF05C040E050E002C0DE
:10DBB0004FEF50E065E269CF6F3F710534F4AB0180
:10DBC00077FF05C040E050E002C04FEF50E066E252
:10DBD0005CCF6F3F710534F4AB0177FF05C040E0C7
:10DBE00050E002C04FEF50E068E24FCF6F3F710549
:10DBF00034F4AB0177FF05C040E050E002C04FEFC6
:10DC000050E069E242CFAF92BF92CF92DF92EF92A3
:10DC1000FF920F931F93CF93DF938C01C62F7A014E
:10DC2000690163E570E084E09DE00E940E5C6C2F6A
:10DC300084E09DE00E94BD5B84E09DE00E94825CE8
:10DC400063E570E084E09DE00E940E5CA70163E55F
:10DC500070E084E09DE00E94805CE6015E01AC180B
:10DC6000BD0884E09DE00E94665B892B31F084E072
:10DC70009DE00E946E5B8993F1CFAE14BF0421F04A
:10DC8000F801108281E0818384E09DE0DF91CF91F3
:10DC90001F910F91FF90EF90DF90CF90BF90AF90CA
:10DCA0000C94825CCF92DF92EF92FF920F931F93BE
:10DCB000CF93DF93EC016B017A0189019C01225F14
:10DCC0003F4F46E050E062E39EDF8F8590E0982F63
:10DCD00088272E85822BF60191838083898990E0A5
:10DCE000982F88272889822BF701918380838B893D
:10DCF00090E0982F88272A89822BF80191838083CE
:10DD0000DF91CF911F910F91FF90EF90DF90CF9017
:10DD100008959B012C5F3F4FAB014E5F5F4FC2CF19
:10DD2000AF92BF92CF92DF92EF92FF920F931F9329
:10DD3000CF93DF9300D000D0CDB7DEB77C015B017D
:10DD4000BE016F5F7F4FE5DFCE0101966C01870159
:10DD500075015E0197E0A90EB11CF6016191719108
:10DD60006F01882777FD8095982F0E94A190F80178
:10DD700022813381448155810E943592F70161935C
:10DD80007193819391937F010C5F1F4FCA14DB0441
:10DD900021F726960FB6F894DEBF0FBECDBFDF91F8
:10DDA000CF911F910F91FF90EF90DF90CF90BF9098
:10DDB000AF900895CF93DF931F92CDB7DEB79E014A
:10DDC0002F5F3F4F41E050E06DE11DDF898190E022
:10DDD0000F90DF91CF910895AF92BF92CF92DF92D3
:10DDE000EF92FF920F931F93CF93DF931F92CDB7C4
:10DDF000DEB78C015B016A0179019E012F5F3F4F05
:10DE000041E050E06EE1FFDE898190E0F501918311
:10DE100080839E012F5F3F4F41E050E06FE1C801DA
:10DE2000F2DE898190E0F601918380839E012F5F6D
:10DE30003F4F41E050E060E2C801E5DE898190E0BB
:10DE4000F701918380830F90DF91CF911F910F9104
:10DE5000FF90EF90DF90CF90BF90AF900895CF9359
:10DE6000DF931F92CDB7DEB79E012F5F3F4F41E09A
:10DE700050E061E2C8DE898190E00F90DF91CF91A0
:10DE80000895CF93DF931F92CDB7DEB79E012F5F2A
:10DE90003F4F41E050E062E2B6DE898190E00F90B2
:10DEA000DF91CF910895CF93DF931F92CDB7DEB767
:10DEB0009E012F5F3F4F41E050E063E2A4DE898185
:10DEC00090E00F90DF91CF910895CF93DF931F9251
:10DED000CDB7DEB79E012F5F3F4F41E050E064E2D7
:10DEE00092DE898190E00F90DF91CF910895CF93DA
:10DEF000DF931F92CDB7DEB79E012F5F3F4F41E00A
:10DF000050E065E280DE898190E00F90DF91CF9153
:10DF10000895CF93DF931F92CDB7DEB79E012F5F99
:10DF20003F4F41E050E066E26EDE898190E00F9065
:10DF3000DF91CF910895CF93DF931F92CDB7DEB7D6
:10DF40009E012F5F3F4F41E050E068E25CDE898137
:10DF500090E00F90DF91CF910895CF93DF931F92C0
:10DF6000CDB7DEB79E012F5F3F4F41E050E069E241
:10DF70004ADE898190E00F90DF91CF910895CF9391
:10DF8000DF931F92CDB7DEB79E012F5F3F4F41E079
:10DF900050E06CE238DE69816F7070E066507109A4
:10DFA000882777FD8095982F0E94A1909B01AC0156
:10DFB00060E070E080E090E40E94989220E030E021
:10DFC00048EC50E40E9435920F90DF91CF91089574
:10DFD000EF92FF920F931F93CF93DF931F92CDB7D2
:10DFE000DEB78C01CB01BA0120E030E048EC50E410
:10DFF0000E94D58F0E946E90E12CF12C759567954B
:10E000006115710521F08FEFE81AF80AF7CF8AE061
:10E01000E816F10484F49E012F5F3F4F41E050E089
:10E020006CE2C801F0DD46E04E0D8981807F482B0F
:10E030006CE2C8012ADD0F90DF91CF911F910F9103
:10E04000FF90EF900895CF93DF931F92CDB7DEB787
:10E050009E012F5F3F4F41E050E060E3D4DD8981B6
:10E060000F90DF91CF910895DF92EF92FF920F937F
:10E070001F93CF93DF931F92CDB7DEB78C01F62E9F
:10E08000E42ED22E9E012F5F3F4F41E050E0BBDDDA
:10E09000898121E030E00E2C01C0220F0A94EAF7BA
:10E0A000DD2011F0282B02C02095282329834981E7
:10E0B0006F2DC801EADC0F90DF91CF911F910F9176
:10E0C000FF90EF90DF900895262F47E050E061E346
:10E0D000CBCF262F46E050E067E2C6CF262F45E0A3
:10E0E00050E067E2C1CF262F44E050E067E2BCCFAA
:10E0F000262F42E050E067E2B7CF262F41E050E004
:10E1000067E2B2CF262F40E050E067E2ADCF262F86
:10E1100047E050E067E2A8CF262F43E050E067E2F7
:10E12000A3CF262F43E050E06AE29ECF262F42E0A5
:10E1300050E06AE299CF262F41E050E06AE294CFA6
:10E14000262F40E050E06AE28FCF262F44E050E0D7
:10E150006CE28ACF242F462F50E06FE285CF242F28
:10E16000462F50E06EE280CF1F93CF93DF931F9234
:10E17000CDB7DEB7142F9E012F5F3F4F41E050E037
:10E1800042DD898190E002C0959587951A95E2F766
:10E1900081700F90DF91CF911F91089547E050E07B
:10E1A00061E3E2CF46E050E067E2DECF45E050E0D9
:10E1B00067E2DACF44E050E067E2D6CF42E050E0D9
:10E1C00067E2D2CF41E050E067E2CECF40E050E0DE
:10E1D00067E2CACF43E050E067E2C6CF43E050E0D9
:10E1E0006AE2C2CF42E050E06AE2BECF41E050E0D6
:10E1F0006AE2BACF40E050E06AE2B6CF46E050E0D3
:10E200006BE2B2CF45E050E06BE2AECF44E050E0CD
:10E210006BE2AACF42E050E06BE2A6CF41E050E0D3
:10E220006BE2A2CF40E050E06BE29ECF43E050E0D3
:10E230006BE29ACF44E050E06CE296CF462F50E07C
:10E2400060E392CF462F50E06FE28ECF462F50E032
:10E250006EE28ACFEF92FF920F931F93CF93DF93DB
:10E260001F92CDB7DEB77C016AE47AE08EE99EE0CA
:10E270000E94A9879E012F5F3F4F41E050E060E080
:10E28000C701C1DC8981DDDB6CE67AE08EE99EE0C6
:10E290000E94D4870DE110E061E57AE08EE99EE00E
:10E2A0000E94A98740E150E0B8018EE99EE00E94FB
:10E2B00093886CE679E08EE99EE00E94A9879E0132
:10E2C0002F5F3F4F41E050E0602FC7019CDC898108
:10E2D000B8DB6CE67AE08EE99EE00E94D4870F5F9F
:10E2E0001F4F0A331105C1F60F90DF91CF911F9197
:10E2F0000F91FF90EF900895CF92DF92EF92FF92EF
:10E30000CF93DF93EC01882777FD8095982F0E94AB
:10E31000A1906B017C0120E030E040E45FE30E94CB
:10E32000359220E030E048E452E40E94D58F0E940C
:10E330006E90C617D707ECF020E030E040EA5FE3CC
:10E34000C701B6010E94359220E030E048E452E473
:10E350000E94D58F20E030E040E85FE30E940B8F01
:10E360000E946E9021E06C177D070CF420E0822F54
:10E3700001C080E090E0DF91CF91FF90EF90DF90BF
:10E38000CF900895CF92DF92EF92FF92CF93DF93D9
:10E39000EC016C597F4F882777FD8095982F0E945C
:10E3A000A1906B017C0120E030E040E45FE30E943B
:10E3B000359220E030E048E452E40E94D58F0E947C
:10E3C0006E90C617D707ECF020E030E040EA5FE33C
:10E3D000C701B6010E94359220E030E048E452E4E3
:10E3E0000E94D58F20E030E040E85FE30E940B8F71
:10E3F0000E946E9021E06C177D070CF420E0822FC4
:10E4000001C080E090E0DF91CF91FF90EF90DF902E
:10E41000CF900895CF92DF92EF92FF92CF93DF9348
:10E42000EC0164567109882777FD8095982F0E942A
:10E43000A1906B017C0120E030E040E45FE30E94AA
:10E44000359220E030E048E452E40E94D58F0E94EB
:10E450006E90C617D707ECF020E030E040EA5FE3AB
:10E46000C701B6010E94359220E030E048E452E452
:10E470000E94D58F20E030E040E85FE30E940B8FE0
:10E480000E946E9021E06C177D070CF420E0822F33
:10E4900001C080E090E0DF91CF91FF90EF90DF909E
:10E4A000CF9008951F920F920FB60F9211240BB6C2
:10E4B0000F922F933F934F935F936F937F938F931D
:10E4C0009F93AF93BF93EF93FF938091C50D0E94ED
:10E4D00054832091C80D3091C90D2F5F3F4F309369
:10E4E000C90D2093C80D9091C70D953618F096E090
:10E4F0009093C40D9091C40D9430C9F128F49230DA
:10E5000069F09330D1F05EC0953009F451C0963077
:10E5100009F058C091E09093940E51C0811152C0FF
:10E520002091C80D3091C90D2436310508F442C040
:10E530001092940E1092C70D1CC0813009F042C099
:10E54000E091C70D91E09E0F9093C70DF0E02091F0
:10E55000C80D3091C90DEE0FFF1FE653F24F318306
:10E5600020831092C90D1092C80D94E029C081112A
:10E5700017C0E091C70D91E09E0F9093C70DF0E09A
:10E580002091C80D3091C90DEE0FFF1FE653F24FD9
:10E59000318320831092C90D1092C80D93E010C0F2
:10E5A0002091C80D3091C90D2536310558F007C0AE
:10E5B000811108C01092C90D1092C80D03C095E0DA
:10E5C0009093C40D9091C60D992329F0811102C03A
:10E5D0002F9A01C02F98FF91EF91BF91AF919F911A
:10E5E0008F917F916F915F914F913F912F910F90FC
:10E5F0000BBE0F900FBE0F901F9018956093C50D26
:10E600001092C60D0895F89482E08093B000809334
:10E61000B10094E69093B3001092B2008093700022
:10E6200078948093C40D1092C70D8091C50D60E061
:10E630000C94E68282E08093C40D1092C70D089579
:10E640008F929F92AF92BF92CF92DF92EF92FF9202
:10E650007B01BA0180E090E00E949F904B015C0139
:10E66000B70180E090E00E949F906B017C012DEC4F
:10E670003CEC4CE45FE30E9435929B01AC01C50188
:10E68000B4010E94D18F87FD17C02DEC3CEC4CE407
:10E690005FE3C501B4010E9435929B01AC01C70143
:10E6A000B6010E94D18F992787FD90958827990FF1
:10E6B000881F9927019602C080E090E0FF90EF90BC
:10E6C000DF90CF90BF90AF909F908F9008958F92E2
:10E6D0009F92AF92BF92CF92DF92EF92FF920F93F1
:10E6E0001F93CF93DF936C01EB01EC84FD8486E0F4
:10E6F000E816F1040CF443C0EE0CFF1C06E010E039
:10E7000045EC842E4DE9942E4CE1A42E41E8B42E24
:10E710008A859B85FC01E00FF11F40815181F80142
:10E720003497E80FF91F60817181C60189DFFC0110
:10E73000A501940163E971E080E091E00E944293B9
:10E740004F01AA2497FCA094BA2C86269726A826C7
:10E75000B9260E5F1F4F0E151F05D1F68C829D82C4
:10E76000AE82BF8280E290E0998788878FEF9FEF2B
:10E770009983888361E070E080E090E003C060E00E
:10E7800070E0CB01DF91CF911F910F91FF90EF903F
:10E79000DF90CF90BF90AF909F908F9008950F9390
:10E7A0001F93CF93DF938C01EB018AEC9DE09B8755
:10E7B0008A878091C70D90E09D878C878091940E09
:10E7C00090E09F878E878091C40D853009F051C0FD
:10E7D000C8011BD3882319F081E090E04CC0BE0132
:10E7E000C801B0D78111F8CFBE01C80107D7811188
:10E7F000F3CFBE01C8017ED28111EECFBE01C801A8
:10E80000CCD48111E9CFBE01C80169D58111E4CF13
:10E81000BE01C80192D38111DFCFBE01C801E3D18F
:10E820008111DACFBE01C8012DD18111D5CFBE0132
:10E83000C80145D68111D0CFBE01C8010E943D7CE0
:10E840008111CACFBE01C8011BD08111C5CFBE0145
:10E85000C801A2D08111C0CFBE01C80138DF672B2B
:10E86000682B692B09F0B8CF82E08093C40D109219
:10E87000C70D80E090E0DF91CF911F910F91089537
:10E88000AF92BF92CF92DF92EF92FF920F931F93BE
:10E89000CF93DF93EB018091C70D883510F480E0B2
:10E8A00070C0EA85FB858281938160E672E26ADD51
:10E8B000892BA9F3EA85FB858481958164E971E15F
:10E8C000A9DD892B61F3BEE1CB2ED12C1DE1E12E18
:10E8D000F12C00E010E08091C70D90E00497E8165D
:10E8E000F906ACF5EA85FB85C701880F991FE80F8B
:10E8F000F91F8081918164EF71E044DD892B79F209
:10E900005601AA0CBB1CEA85FB85EA0DFB1D808124
:10E91000918168E572E07EDD892B21F0000F111FE7
:10E9200001600DC0EA85FB85EA0DFB1D80819181A8
:10E9300064EA76E06FDD892B49F0000F111F82E059
:10E94000E80EF11C82E0C80ED11CC5CF760181E033
:10E95000E81AF108F594E794F986E8868AE2E81661
:10E96000F1040CF49CCFC801AA2797FDA095BA2FFB
:10E970008C839D83AE83BF8389E090E099838883F5
:10E9800081E0DF91CF911F910F91FF90EF90DF9089
:10E99000CF90BF90AF900895AF92BF92CF92DF9289
:10E9A000EF92FF920F931F93CF93DF93EB01809130
:10E9B000C70D803211F080E05AC0EA85FB85828164
:10E9C00093816CE271E0DEDC892BA9F3EA85FB859B
:10E9D000848195816EEE72E01DDD892B61F306E086
:10E9E00010E0C12CD12C7601EA85FB85E00FF11FE8
:10E9F000808191816CE271E0C5DC892BE1F25801E4
:10EA000082E0A80EB11CEA85FB85EA0DFB1D808122
:10EA1000918168E077E0FEDC892B39F0CC0CDD1CBD
:10EA2000EE1CFF1C6894C0F810C0EA85FB85EA0D57
:10EA3000FB1D808191816EEE72E0ECDC892B09F484
:10EA4000BACFCC0CDD1CEE1CFF1C0C5F1F4F0E332D
:10EA5000110551F68EE090E099878887CC82DD829F
:10EA6000EE82FF828FE090E09983888381E0DF91DE
:10EA7000CF911F910F91FF90EF90DF90CF90BF90BB
:10EA8000AF900895AF92BF92CF92DF92EF92FF9234
:10EA90000F931F93CF93DF93EB018091C70D8232C9
:10EAA00051F5EA85FB858281938168E572E06ADC35
:10EAB000892B09F18091C70D90E081509048880F13
:10EAC000991FEA85FB85E80FF91F8081918168E530
:10EAD00072E058DC892B79F0198618868FEF9FEF4A
:10EAE000DC018C839D83AE83BF8386E090E09983B5
:10EAF000888381E06DC0EA85FB858281938160E433
:10EB00007FE140DC892B21F08091C70D813210F428
:10EB100080E05EC0EA85FB858481958160EA7FE0C4
:10EB200079DC892BA9F358E0A52EB12C03E010E085
:10EB3000C12CD12C7601EA85FB85C801880F991F6D
:10EB4000E80FF91F8081918168E572E01BDC892B59
:10EB5000F9F2EA85FB85EA0DFB1D8081918160E475
:10EB600076E058DC892B39F0CC0CDD1CEE1CFF1C48
:10EB70006894C0F810C0EA85FB85EA0DFB1D808112
:10EB8000918166E272E046DC892B09F4C1CFCC0C9E
:10EB9000DD1CEE1CFF1C0E5F1F4F84E0A80EB11C95
:10EBA0000332110541F6EA85FB85EA5BFF4F808160
:10EBB000918168E572E0E6DB892B09F4A9CF80E159
:10EBC00090E099878887CC82DD82EE82FF828DCFAC
:10EBD000DF91CF911F910F91FF90EF90DF90CF9039
:10EBE000BF90AF900895AF92BF92CF92DF92EF9215
:10EBF000FF920F931F93CF93DF93EB018091C70D8B
:10EC0000893310F480E06BC0EA85FB8582819381B3
:10EC100060E47FE1B7DB892BA9F3EA85FB8584817A
:10EC2000958160EA7FE0F6DB892B61F338E0A32E63
:10EC3000B12C03E010E0C12CD12C7601EA85FB85D4
:10EC4000C801880F991FE80FF91F8081918168E53D
:10EC500072E098DB892BB1F2EA85FB85EA0DFB1D9A
:10EC60008081918160E476E0D5DB892B39F0CC0C92
:10EC7000DD1CEE1CFF1C6894C0F810C0EA85FB8503
:10EC8000EA0DFB1D8081918166E272E0C3DB892B76
:10EC900009F4B8CFCC0CDD1CEE1CFF1C0E5F1F4F1F
:10ECA00084E0A80EB11C0B33110541F6EA85FB8503
:10ECB000EA58FF4F8081918168E572E063DB892B20
:10ECC00009F4A0CF8CE190E099878887CC82DD821F
:10ECD000EE82FF828AE090E09983888381E0DF9171
:10ECE000CF911F910F91FF90EF90DF90CF90BF9049
:10ECF000AF9008956F927F928F929F92AF92BF9242
:10ED0000CF92DF92EF92FF920F931F93CF93DF93F7
:10ED1000EB018091C70D823208F45DC0EA85FB8566
:10ED2000828193816EE571E02DDB892B09F453C05C
:10ED300063E0A62EB12C02E010E0C12CD12C7601AC
:10ED400035018091C70D90E0A816B906CCF54801B1
:10ED5000880C991CEA85FB85E80DF91D808191815D
:10ED60006EE977E00FDB892B39F0CC0CDD1CEE1C53
:10ED7000FF1C6894C0F80FC0EA85FB85E80DF91DFB
:10ED8000808191816EEE72E0FDDA892B21F1CC0C4D
:10ED9000DD1CEE1CFF1CC501880F991FEA85FB8551
:10EDA000E80FF91F808191816EE571E033DB22E08D
:10EDB000A20EB11C892B19F00E5F1F4FC1CF83012A
:10EDC000015011091595079519870887003111051C
:10EDD00024F41986188680E009C0CC82DD82EE8298
:10EDE000FF828CE090E09983888381E0DF91CF916E
:10EDF0001F910F91FF90EF90DF90CF90BF90AF9059
:10EE00009F908F907F906F900895AF92BF92CF9216
:10EE1000DF92EF92FF920F931F93CF93DF93EB015B
:10EE2000EA85FB858281938168E273E2ABDA892B04
:10EE300011F480E077C08091C70D843009F5EA8530
:10EE4000FB85848195816AEC78E0E4DA892BC1F056
:10EE5000EA85FB858681978160E372E093DA892BEE
:10EE600079F0198618868FEF9FEFDC018C839D83E4
:10EE7000AE83BF8383E090E09983888381E052C0B2
:10EE80008091C70D8434A8F2EA85FB858481958141
:10EE900064E971E1BFDA892B61F206E010E0C12C70
:10EEA000D12C7601EA85FB85E00FF11F80819181ED
:10EEB00060E372E067DA892B09F4BBCF580182E086
:10EEC000A80EB11CEA85FB85EA0DFB1D80819181AE
:10EED0006AE976E09FDA892B39F0CC0CDD1CEE1C58
:10EEE000FF1C6894C0F810C0EA85FB85EA0DFB1D85
:10EEF0008081918160E372E08DDA892B09F499CFEA
:10EF0000CC0CDD1CEE1CFF1C0C5F1F4F06381105DE
:10EF100049F680E290E099878887CC82DD82EE8294
:10EF2000FF82A8CFDF91CF911F910F91FF90EF90BB
:10EF3000DF90CF90BF90AF9008958F929F92AF9245
:10EF4000BF92CF92DF92EF92FF920F931F93CF93D6
:10EF5000DF9300D01F92CDB7DEB74B01DB011A96CD
:10EF6000ED91FC911B97828193816EEA7DE00ADA34
:10EF7000892B11F480E08FC0D4011A96ED91FC9199
:10EF80001B978481958166ED76E0FCD9892B91F3FE
:10EF9000E6E0EE2EF12C20E030E040E050E0A12C45
:10EFA000B12CC12CD12CD4011A96ED91FC911B9758
:10EFB000EE0DFF1D8081918166EF71E029833A8318
:10EFC0004B835C83DFD9892BA9F287010E5F1F4F2A
:10EFD000D4011A96ED91FC911B97E00FF11F8081EF
:10EFE00091816CED74E016DA29813A814B815C8164
:10EFF000892B39F0B501C60101E00E94D093216050
:10F000001CC0D4011A96ED91FC911B97E00FF11FE3
:10F010008081918160E971E029833A834B835C832D
:10F02000F9D929813A814B815C81892B09F4A2CFDE
:10F03000B501C60101E00E94D0935B016C01B4E010
:10F04000EB0EF11CE6ECEE16F10409F0ACCFD401A6
:10F0500014962C93149715963C93159716964C93EB
:10F06000169717965C931797B501C60100E20E94A8
:10F07000EB9312962C93129713963C93139785E07B
:10F0800090E011969C938E9380E390E019969C9368
:10F090008E93189781E00F900F900F900F90DF9153
:10F0A000CF911F910F91FF90EF90DF90CF90BF9085
:10F0B000AF909F908F9008958F929F92AF92BF9242
:10F0C000CF92DF92EF92FF920F931F93CF93DF9334
:10F0D0007A016901DA01CD91DC91FB018485958586
:10F0E000C817D9070CF047C0CE01880F991F0284BA
:10F0F000F385E02DE80FF91FA080B180C170DD27F6
:10F10000F1E0CF27209719F484E690E002C08CE963
:10F110009FEF4801880E991EB401C501EDD8892BD7
:10F1200089F4800E911EB401C501E6D8892B69F4DB
:10F13000B401600F711FC501DFD8892BF9F023E0FE
:10F1400030E005C021E030E002C022E030E0D6012E
:10F150008D919C91119701968217930744F0F601C7
:10F1600011821082D7018D919C91119701968D93F8
:10F170009C93CE0105C081E090E002C08FEF9FEF2D
:10F18000DF91CF911F910F91FF90EF90DF90CF9083
:10F19000BF90AF909F908F9008954F925F926F9223
:10F1A0007F928F929F92AF92BF92CF92DF92EF9217
:10F1B000FF920F931F93CF93DF9300D01F92CDB791
:10F1C000DEB76C017B011C821B8281E090E09A8398
:10F1D00089838091C70D8D3010F480E06BC009E702
:10F1E00013E09E012D5F3F4FAE014F5F5F4FC601A1
:10F1F00063DF892B91F79E012D5F3F4FAE014F5F7B
:10F200005F4FB701C60158DF019739F79E012D5FA7
:10F210003F4FAE014F5F5F4FB701C6014DDF892BF6
:10F22000E1F6412C512C3201A12CB12C8091C70D5B
:10F2300090E029813A81281739078CF509E713E016
:10F240009E012D5F3F4FAE014F5F5F4FB701C6017B
:10F2500033DF4C019E012D5F3F4FAE014F5F5F4F8B
:10F26000B701C60129DF21E08216910451F4892BF0
:10F2700009F0B3CF440C551C661C771C689440F809
:10F280000AC0892809F0A9CF019709F0A6CF440C3C
:10F29000551C661C771C8FEFA81AB80AC7CFF70158
:10F2A000B186A086448255826682778281E090E0B2
:10F2B000918380830F900F900F900F90DF91CF91EB
:10F2C0001F910F91FF90EF90DF90CF90BF90AF9084
:10F2D0009F908F907F906F905F904F9008952F92A6
:10F2E0003F924F925F926F927F928F929F92AF92D6
:10F2F000BF92CF92DF92EF92FF920F931F93CF9323
:10F30000DF9300D01F92CDB7DEB76C017B011C826A
:10F310001B82DB011C968D919C911D971816190676
:10F3200014F080E0B5C0DB011A96ED91FC911B97BB
:10F3300082E090E09A838983828193816AE67AE011
:10F3400021D8892B71F3D7011A96ED91FC911B9767
:10F3500089819A819C012F5F3F4F3A832983880FCF
:10F36000991FE80FF91F8081918169E773E052D8F6
:10F37000892BB9F20CEB11E09E012D5F3F4FAE01DE
:10F380004F5F5F4FB701C60197DE892B51F69E0193
:10F390002D5F3F4FAE014F5F5F4FB701C6018CDE5F
:10F3A000019709F0BECF212C312C2101A12CB12CC9
:10F3B00029813A81F70184859585281739070CF052
:10F3C0005CC00CEB11E09E012D5F3F4FAE014F5F23
:10F3D0005F4FB701C60170DE3C01B3E0AB16B1046C
:10F3E00089F00CEB11E09E012D5F3F4FAE014F5FA6
:10F3F0005F4FB701C60160DE4C01E3E0AE16B10419
:10F40000F9F40FC00CEB11E09E012D5F3F4FAE01F0
:10F410004F5F5F4FB701C6014FDE6816790609F3EB
:10F4200080CF0CEB11E09E012D5F3F4FAE014F5F8F
:10F430005F4FB701C60140DE8816990609F071CF0B
:10F440006114710459F48A94892809F06ACF220C56
:10F45000331C441C551C689420F80BC06A94672820
:10F4600009F05FCF892809F05CCF220C331C441CC3
:10F47000551CAFEFAA1ABA0A9BCFB186A086248288
:10F4800035824682578282E090E09183808381E0DA
:10F490000F900F900F900F90DF91CF911F910F91D0
:10F4A000FF90EF90DF90CF90BF90AF909F908F90A4
:10F4B0007F906F905F904F903F902F900895AF9204
:10F4C000BF92CF92DF92EF92FF920F931F93CF9351
:10F4D000DF93EB01EA85FB858281938168E873E124
:10F4E0000E94C271892B11F480E07DC08091C70D0C
:10F4F000843019F5EA85FB85848195816AEC78E092
:10F500000E940A72892BC9F0EA85FB858681978162
:10F5100060E372E00E94C271892B79F01986188627
:10F520008FEF9FEFDC018C839D83AE83BF8387E0E9
:10F5300090E09983888381E056C08091C70D843420
:10F5400098F2EA85FB858481958168E873E10E94E1
:10F550000A72892B49F206E010E0C12CD12C760109
:10F56000EA85FB85E00FF11F8081918160E372E005
:10F570000E94C271892B09F4B7CF580182E0A80E0E
:10F58000B11CEA85FB85EA0DFB1D8081918160E459
:10F5900076E00E940A72892B39F0CC0CDD1CEE1C3F
:10F5A000FF1C6894C0F811C0EA85FB85EA0DFB1DBD
:10F5B0008081918160E372E00E940A72892B09F4D4
:10F5C00093CFCC0CDD1CEE1CFF1C0C5F1F4F0638CC
:10F5D000110531F680E290E099878887CC82DD8240
:10F5E000EE82FF82A4CFDF91CF911F910F91FF9008
:10F5F000EF90DF90CF90BF90AF9008958F929F9241
:10F60000AF92BF92CF92DF92EF92FF920F931F9330
:10F61000CF93DF93EB018091C70D8A3108F47AC054
:10F62000EA85FB85808191818032934050F4198670
:10F6300018868FEF9FEFDC018C839D83AE83BF83A1
:10F640006FC0828193816CEA7DE00E94C271892B38
:10F6500009F460C0EA85FB85848195816CEA7DE0D0
:10F660000E94C271892B09F455C054E0A52EB12C1B
:10F6700003E010E0C12CD12C76018091C70D90E001
:10F68000A816B906E4F5EA85FB85C801880F991F1D
:10F69000E80FF91F8081918166EB73E00E940A7286
:10F6A000892B61F14501880C991CEA85FB85E80DE1
:10F6B000F91D8081918160E679E00E94C271892BF9
:10F6C00039F0CC0CDD1CEE1CFF1C6894C0F810C097
:10F6D000EA85FB85E80DF91D808191816CEB72E074
:10F6E0000E94C271892BB1F0CC0CDD1CEE1CFF1CFA
:10F6F0000E5F1F4F82E0A80EB11CBFCF85010150E5
:10F70000110915950795198708870C30110524F400
:10F710001986188680E009C0CC82DD82EE82FF82E5
:10F720008BE090E09983888381E0DF91CF911F91F6
:10F730000F91FF90EF90DF90CF90BF90AF909F9090
:10F740008F9008958F929F92AF92BF92CF92DF9247
:10F75000EF92FF920F931F93CF93DF93EB01809172
:10F76000C70D8A3108F471C0EA85FB8580819181DB
:10F77000843F914060F4198618868FEF9FEFDC017B
:10F780008C839D83AE83BF838BE090E066C08281D3
:10F79000938160E679E00E94C271892B09F455C01B
:10F7A00073E0A72EB12C02E010E0C12CD12C760121
:10F7B0008091C70D90E0A816B906E4F5EA85FB85AF
:10F7C000C801880F991FE80FF91F8081918168E5B2
:10F7D00072E00E940A72892B61F14501880C991C24
:10F7E000EA85FB85E80DF91D8081918160EB74E06D
:10F7F0000E94C271892B39F0CC0CDD1CEE1CFF1C61
:10F800006894C0F810C0EA85FB85E80DF91D808179
:10F81000918168E572E00E94C271892BB1F0CC0C35
:10F82000DD1CEE1CFF1C0E5F1F4F82E0A80EB11CFA
:10F83000BFCF8501015011091595079519870887D4
:10F840000C30110524F41986188680E009C0CC829A
:10F85000DD82EE82FF8284E090E09983888381E0FC
:10F86000DF91CF911F910F91FF90EF90DF90CF909C
:10F87000BF90AF909F908F900895AF92BF92CF921C
:10F88000DF92EF92FF920F931F93CF93DF93EB01E1
:10F890008091C70D863410F480E086C0EA85FB8530
:10F8A000828193816EEE72E00E94C271892BA1F376
:10F8B000EA85FB85848195816EEE72E00E940A7272
:10F8C000892B51F3EA85FB858681978162E27BE093
:10F8D0000E94C271892B01F3EA85FB8580859185A1
:10F8E00062E27BE00E940A72892BB1F25CE0A52EF5
:10F8F000B12C05E010E0C12CD12C7601EA85FB8506
:10F90000C801880F991FE80FF91F808191816EEE61
:10F9100072E00E94C271892B09F4BECFEA85FB8593
:10F92000EA0DFB1D8081918166E678E00E940A72F3
:10F93000892B39F0CC0CDD1CEE1CFF1C6894C0F840
:10F9400011C0EA85FB85EA0DFB1D808191816EEE79
:10F9500072E00E940A72892B09F49ECFCC0CDD1C48
:10F96000EE1CFF1C0E5F1F4F84E0A80EB11C053477
:10F97000110521F6EA85FB85E657FF4F80819181CD
:10F980006EEE72E00E94C271892B09F485CF80E28D
:10F9900090E099878887CC82DD82EE82FF8288E0C2
:10F9A00090E09983888381E0DF91CF911F910F913F
:10F9B000FF90EF90DF90CF90BF90AF9008953F926F
:10F9C0004F925F926F927F928F929F92AF92BF926F
:10F9D000CF92DF92EF92FF920F931F93CF93DF931B
:10F9E00000D01F921F92CDB7DEB75C01562E198250
:10F9F0001A821B821C821D8261E0852DE7D560E0A2
:10FA0000852D1DD662E170E080E090E0D0D461E009
:10FA1000852D15D688E290E0F0D460E0852DD6D50E
:10FA200001E117E2852D40D6892B31F401501109EF
:10FA3000C9F78EEF9FEF69C001E117E2852D34D63B
:10FA4000019721F401501109C9F7F3CF08E210E042
:10FA5000312C37E0432E88248394912C21E1E22E2F
:10FA600027E2F22E852D20D6892B29F481E0E81A91
:10FA7000F108C1F7DECF78D46B017C0191E1692EEA
:10FA800097E2792E852D10D6019729F4E1E06E1AC0
:10FA90007108C1F7CECF68D46C197D098E099F0912
:10FAA000693271058105910578F0E1E0F0E0EC0F35
:10FAB000FD1FE30DF11D2081C401042C01C0880F3E
:10FAC0000A94EAF7282B2083411004C0339487E07E
:10FAD000482E01C04A940150110909F0BFCF298175
:10FAE000822F90E0F501918380833B81832F90E00A
:10FAF00093838283230F81E090E03D81321302C023
:10FB000080E090E09195819591090F900F900F9072
:10FB10000F900F90DF91CF911F910F91FF90EF9079
:10FB2000DF90CF90BF90AF909F908F907F906F901D
:10FB30005F904F903F900895FB018081883251F093
:10FB400028F4803139F0823239F404C08B3311F05B
:10FB5000823411F481E0089580E00895FC017783F8
:10FB6000668314821582108289E0818381E082831A
:10FB700083830895CF93DF93EC01F0DF1B8A1A8A09
:10FB8000DF91CF910895FC0185810895CF93DF9394
:10FB9000EB0167E0CE010E945A6791E02F8182134A
:10FBA00090E0892FDF91CF910895EF92FF920F930C
:10FBB0001F93CF93DF93EC018B01E42E8E819F8105
:10FBC0000E948E66F12C41E0B8018E819F810E94D7
:10FBD000C266882351F0FE1005C0B801CE01D6DF01
:10FBE000811104C0F394EF1470F780E0DF91CF919E
:10FBF0001F910F91FF90EF900895CF92DF92EF92B7
:10FC0000FF920F931F93CF93DF931F921F92CDB755
:10FC1000DEB76C01F42EE52EFC01868197816983A5
:10FC20007A830E946C6569817A81882311F1F601DB
:10FC3000868197810E94656640E06EEBF6018681C1
:10FC400097810E9409660F2D1E2D89E0F82EF6017E
:10FC5000868197810E944A66F80181938F01FA9408
:10FC6000B1F7F601868197810E946C6591E0813041
:10FC700009F090E0892F0F900F90DF91CF911F91A5
:10FC80000F91FF90EF90DF90CF900895CF93DF9387
:10FC9000EA01B3DF882351F068E0CE010E945A6781
:10FCA00091E02885821390E0892F01C080E0DF91E8
:10FCB000CF910895EF92FF920F931F93CF93DF930D
:10FCC000EC018B017A018E819F810E946C65B801E5
:10FCD0008E819F810E94656640E06EE48E819F81E7
:10FCE0000E94096640E0F70162818E819F810E9437
:10FCF000096640E0F70163818E819F810E94096659
:10FD0000F8018081803139F040E0F70164818E8113
:10FD10009F810E9409668E819F810E946C65B80157
:10FD20008E819F810E946566488168E48E819F81F3
:10FD30000E94096664E170E080E090E038D3888139
:10FD4000882329F06AE070E080E090E030D38E8173
:10FD50009F81DF91CF911F910F91FF90EF900C94B5
:10FD60006C65EF92FF921F93CF93DF931F921F92C8
:10FD7000CDB7DEB77C01FC018681978169837A83E8
:10FD80000E946C6569817A81F701868197810E9462
:10FD9000656640E064EBF701868197810E94096601
:10FDA000F701868197810E94DE65182FF701868111
:10FDB00097810E946C6581E0111180E00F900F9097
:10FDC000DF91CF911F91FF90EF900895CF93DF9334
:10FDD000CDB7DEB729970FB6F894DEBF0FBECDBF03
:10FDE000FB0120812031C9F0AE014F5F5F4F4EDF34
:10FDF000882379F08D818F3351F020F48F3149F4CD
:10FE000089E00CC08F3539F08F3739F002C08AE0B5
:10FE100005C080E003C08BE001C08CE029960FB6DE
:10FE2000F894DEBF0FBECDBFDF91CF910895FF9252
:10FE30000F931F93CF93DF93CDB7DEB728970FB6FD
:10FE4000F894DEBF0FBECDBF8C01FC018681978187
:10FE50000E948E66F8011482158241E0BE016F5F38
:10FE60007F4FF801868197810E94C2668823C1F185
:10FE7000BE016F5F7F4FC80189DE882371F3F801EF
:10FE80008081811107C0BE016F5F7F4FC80169DFAC
:10FE9000811122C0F801F180BE016F5F7F4FC80160
:10FEA00095DF8F1518F4F801818105C0BE016F5FE1
:10FEB0007F4FC8018BDFF801818384818F5F84834A
:10FEC000BE016F5F7F4FC80137DE882331F2F80132
:10FED00085818F5F8583C1CF81E0F8018083DACF90
:10FEE00028960FB6F894DEBF0FBECDBFDF91CF913D
:10FEF0001F910F91FF900895DF92EF92FF920F9361
:10FF00001F93CF93DF93CDB7DEB762970FB6F89408
:10FF1000DEBF0FBECDBF8C017B01D22E493028F051
:10FF2000342F4D3018F03CE001C039E0B701C80172
:10FF30003A8B4CDF3A89831709F458C0AE014F5F02
:10FF40005F4FB701C8013A8BA1DE3A89882309F4D3
:10FF50004FC0F7018081803109F448C03B3041F047
:10FF60003C3021F03A3031F48FE305C08FE703C015
:10FF70008FE501C08FE18D83AE014F5F5F4FB70109
:10FF8000C8013A8B97DEF80191813A89832F39179E
:10FF900008F4892FF8018183D11028C0381730F573
:10FFA0003183E12CF12CF801848190E0E816F90608
:10FFB000ECF44E2DBE01665F7F4FC801F6DDF801FF
:10FFC000D180BE01665F7F4FC80100DF8D1518F438
:10FFD000F801818105C0BE01665F7F4FC801F6DE72
:10FFE000F8018183FFEFEF1AFF0ADDCF81E001C046
:10FFF00080E062960FB6F894DEBF0FBECDBFDF91F2
:020000021000EC
:10000000CF911F910F91FF90EF90DF900895EF92A5
:10001000FF920F931F93CF93DF93CDB7DEB728974F
:100020000FB6F894DEBF0FBECDBF8C01693020F053
:100030006D3018F06CE001C069E0F8016183E12CDB
:10004000F12CF801848190E0E816F90694F44E2D25
:10005000BE016F5F7F4FC801A8DD21E0F80141813B
:10006000BE016F5F7F4FC80147DFFFEFEF1AFF0A46
:10007000E8CF28960FB6F894DEBF0FBECDBFDF9154
:10008000CF911F910F91FF90EF900895FC01868111
:1000900097810E94DE6591E0813009F090E0892F20
:1000A00008958F929F92AF92BF92CF92DF92EF927C
:1000B000FF920F931F93CF93DF93EC01695063304E
:1000C00048F4E62FF0E0EE0FFF1FEC5AF54F0081E9
:1000D000118102C00EEE12E08B818823D1F088815D
:1000E000811117C035D16B017C014801AA2497FC0E
:1000F000A094BA2CCE01CADF81111DC029D1681984
:1001000079098A099B096C157D058E059F0598F470
:10011000F1CFB801882777FD8095982FDF91CF9197
:100120001F910F91FF90EF90DF90CF90BF90AF9015
:100130009F908F903CC1DF91CF911F910F91FF90C5
:10014000EF90DF90CF90BF90AF909F908F900895E9
:10015000CF93DF93EC018E819F810E946C658E812D
:100160009F810E948B66488164E48E819F810E94FA
:1001700009668A81882329F06981CE01DF91CF91B8
:1001800090CFDF91CF910895FA01208148E0249F1C
:1001900090011124818190E0982F8827990F990F61
:1001A000990F282B392BDB018C918031C1F46781A9
:1001B00070E08681AB01481B5109CA019695982FC2
:1001C0008827979587950E94659360517109207FD4
:1001D00053E0220F331F5A95E1F7260F371FC9014D
:1001E0000895EF92FF920F931F93CF93DF93CDB7B4
:1001F000DEB729970FB6F894DEBF0FBECDBF8C01D6
:100200007B01AE014F5F5F4F41DD882339F0AE01C6
:100210004F5F5F4FB701C801B7DF02C080E894EEBF
:1002200029960FB6F894DEBF0FBECDBFDF91CF91F8
:100230001F910F91FF90EF900895813824EE92075F
:100240006CF0BC01882777FD8095982F0E94A190C3
:1002500020E030E040E05CE30C94359260E070E038
:100260008EEF92EC0895BDDFE8CF0F931F93CF93ED
:10027000DF93CDB7DEB728970FB6F894DEBF0FBE79
:10028000CDBF8C01462FBE016F5F7F4F8EDC882370
:1002900031F0BE016F5F7F4FC801E5DF04C060E051
:1002A00070E08EEF92EC28960FB6F894DEBF0FBE8A
:1002B000CDBFDF91CF911F910F9108951F920F92A3
:1002C0000FB60F9211242F933F938F939F93AF9369
:1002D000BF938091960E9091970EA091980EB09139
:1002E000990E3091950E23E0230F2D3720F40196BF
:1002F000A11DB11D05C026E8230F0296A11DB11D49
:100300002093950E8093960E9093970EA093980E3F
:10031000B093990E80919A0E90919B0EA0919C0E95
:10032000B0919D0E0196A11DB11D80939A0E9093E0
:100330009B0EA0939C0EB0939D0EBF91AF919F9189
:100340008F913F912F910F900FBE0F901F90189596
:100350002FB7F8946091960E7091970E8091980E39
:100360009091990E2FBF08953FB7F89480919A0EFF
:1003700090919B0EA0919C0EB0919D0E26B5A89BCE
:1003800005C02F3F19F00196A11DB11D3FBF662783
:10039000782F892F9A2F620F711D811D911D42E0C8
:1003A000660F771F881F991F4A95D1F70895CF923E
:1003B000DF92EF92FF92CF93DF936B017C01D4DF4A
:1003C000EB01C114D104E104F10481F00E94098F12
:1003D000CBDF6C1B7D0B683E734098F381E0C81A3D
:1003E000D108E108F108C851DC4FEBCFDF91CF9184
:1003F000FF90EF90DF90CF9008958230910538F014
:10040000880F991F880F991F05970197F1F7089595
:10041000789484B5826084BD84B5816084BD85B5DF
:10042000826085BD85B5816085BDEEE6F0E08081A6
:1004300081608083E1E8F0E01082808182608083C7
:10044000808181608083E0E8F0E08081816080834A
:10045000E1EBF0E0808184608083E0EBF0E080817C
:1004600081608083E1E9F0E0808182608083808127
:1004700081608083E0E9F0E0808181608083E1EA4F
:10048000F0E0808182608083808181608083E0EA07
:10049000F0E0808181608083E1E2F1E08081826030
:1004A0008083808181608083E0E2F1E080818160EF
:1004B0008083EAE7F0E080818460808380818260CD
:1004C00080838081816080838081806880831092B6
:1004D000C10008958093A5040895863308F08653DB
:1004E00020917B00982F9870277F922B90937B0010
:1004F00087702091A50490E4299F90011124822BFC
:1005000080937C0080917A00806480937A0080914F
:100510007A0086FDFCCF809178002091790090E0F0
:10052000922B089590E0FC013197E231F10508F03B
:100530004CC0EB56FF4F0C94B693809180008F77A0
:1005400003C0809180008F7D80938000089580910A
:100550008000877FF9CF84B58F7702C084B58F7D07
:1005600084BD08958091B0008F7703C08091B00062
:100570008F7D8093B0000895809190008F7707C0A1
:10058000809190008F7D03C080919000877F809341
:10059000900008958091A0008F7707C08091A000FF
:1005A0008F7D03C08091A000877F8093A000089575
:1005B000809120018F7707C0809120018F7D03C03B
:1005C00080912001877F809320010895CF93DF934E
:1005D00090E0FC01EF56F34F2491FC01E952F34FF8
:1005E0008491882349F190E0880F991FFC01EF5A0C
:1005F000F24FA591B491895C924FFC01C591D491C1
:100600009FB7611108C0F8948C91209582238C9338
:10061000888182230AC0623051F4F8948C91322F81
:10062000309583238C938881822B888304C0F8942F
:100630008C91822B8C939FBFDF91CF9108950F9364
:100640001F93CF93DF931F92CDB7DEB7282F30E0F3
:10065000F901E55BF34F8491F901EF56F34F1491E3
:10066000F901E952F34F04910023C1F0882319F0F6
:10067000698358DF6981E02FF0E0EE0FFF1FE95C2E
:10068000F24FA591B4919FB7F8948C91611103C07A
:100690001095812301C0812B8C939FBF0F90DF9118
:1006A000CF911F910F910895CF93DF93282F30E0C2
:1006B000F901E55BF34F8491F901EF56F34FD491C3
:1006C000F901E952F34FC491CC2389F081112ADF5B
:1006D000EC2FF0E0EE0FFF1FE35EF24FA591B49117
:1006E0002C912D2381E090E021F480E002C080E095
:1006F00090E0DF91CF9108950F931F93762F90E0B4
:10070000FC01EF56F34F6491FC01E952F34FE49181
:100710007111762FF0E0EE0FFF1FE35EF24F85912F
:10072000949189019A013F70472F0E9488076115B3
:1007300071058105910531F06F5F7F4F8F4F9F4F9E
:100740009F7003C060E070E0CB011F910F9108958E
:10075000FC01818D228D90E0805C9F4F821B91096E
:100760008F7399270895FC01918D828D981731F030
:10077000828DE80FF11D858D90E008958FEF9FEF3A
:100780000895FC01918D828D981761F0828DDF01B3
:10079000A80FB11D5D968C91928D9F5F9F73928F74
:1007A00090E008958FEF9FEF089588E995E8892BF1
:1007B00039F080E090E0892B19F0BAD1811123C083
:1007C00080E090E0892B41F080E090E0892B21F0DF
:1007D0000E94000081111AC083E496E8892B39F049
:1007E00080E090E0892B19F04ED2811112C08EEE7C
:1007F00096E8892B99F080E090E0892B79F0EED291
:1008000081110AC008950E940000DACF0E94000002
:10081000E3CF0E940000EBCF0C9400000895FC0190
:10082000848DDF01A80FB11DA35ABF4F2C91848D79
:1008300090E001968F739927848FA689B7892C93AE
:10084000A089B1898C9180648C93938D848D981349
:1008500006C00288F389E02D80818F7D8083089512
:10086000CF93DF93EC01888D8823C1F0EA89FB895F
:10087000808185FD05C0A889B9898C9186FD0EC04F
:100880000FB607FCF5CF808185FFF2CFA889B98923
:100890008C9185FFEDCFCE01C2DFE8CFDF91CF9104
:1008A0000895CF92DF92FF920F931F93CF93DF9320
:1008B0001F92CDB7DEB76C0181E0D60158968C93BC
:1008C00058975B969C915B975C968C915C9798137C
:1008D00007C05096ED91FC915197808185FD2DC008
:1008E000F601038D10E00F5F1F4F0F731127F02EDD
:1008F000F601848DF81210C00FB607FCF9CFD601AF
:100900005096ED91FC915197808185FFF1CFC60102
:10091000698385DF6981ECCF838DE80FF11DE35A90
:10092000FF4F6083D6015B960C935B975296ED91D7
:10093000FC915397808180620CC0D6015696ED9150
:10094000FC91579760835096ED91FC91519780816F
:100950008064808381E090E00F90DF91CF911F91C0
:100960000F91FF90DF90CF900895BF92CF92DF92CA
:10097000EF92FF92CF93DF93EC016A017B01B22EDD
:10098000E889F98982E08083411581EE5807610585
:100990007105A1F060E079E08DE390E0A701960198
:1009A0000E94789321503109410951095695479584
:1009B00037952795211580E1380798F0E889F9895E
:1009C000108260E874E88EE190E0A70196010E9431
:1009D000789321503109410951095695479537952A
:1009E0002795EC85FD853083EE85FF852083188E65
:1009F000EC89FD89B082EA89FB89808180618083EE
:100A0000EA89FB89808188608083EA89FB8980810B
:100A100080688083EA89FB8980818F7D8083DF9174
:100A2000CF91FF90EF90DF90CF90BF900895CF933C
:100A3000DF93EC01E881F9810284F385E02D1995BB
:100A4000EA89FB8980818F7E8083EA89FB898081A6
:100A5000877F8083EA89FB8980818F778083EA8919
:100A6000FB8980818F7D80838A8D898FDF91CF91F3
:100A700008951F920F920FB60F9211240BB60F928A
:100A80002F938F939F93EF93FF93E091AE0EF0918E
:100A9000AF0E8081E091B40EF091B50E82FD12C0D0
:100AA00090818091B70E8F5F8F732091B80E82175F
:100AB00051F0E091B70EF0E0E256F14F958F809340
:100AC000B70E01C08081FF91EF919F918F912F917F
:100AD0000F900BBE0F900FBE0F901F9018951F9296
:100AE0000F920FB60F9211240BB60F922F933F93D4
:100AF0004F935F936F937F938F939F93AF93BF9326
:100B0000EF93FF938EE99EE08ADEFF91EF91BF9114
:100B1000AF919F918F917F916F915F914F913F9195
:100B20002F910F900BBE0F900FBE0F901F90189536
:100B30008EE99EE00DDE21E0892B09F420E0822F72
:100B400008951092A10E1092A00E88EE93E0A0E0FE
:100B5000B0E08093A20E9093A30EA093A40EB09346
:100B6000A50E8EE59AE090939F0E80939E0E85ECE5
:100B700090E09093AB0E8093AA0E84EC90E090935B
:100B8000AD0E8093AC0E80EC90E09093AF0E80930E
:100B9000AE0E81EC90E09093B10E8093B00E82EC9B
:100BA00090E09093B30E8093B20E86EC90E0909319
:100BB000B50E8093B40E1092B70E1092B80E10922C
:100BC000B90E1092BA0E08951F920F920FB60F929F
:100BD00011240BB60F922F938F939F93EF93FF9354
:100BE000E0914B0FF0914C0F8081E091510FF0910B
:100BF000520F82FD12C090818091540F8F5F8F73CE
:100C00002091550F821751F0E091540FF0E0E55C10
:100C1000F04F958F8093540F01C08081FF91EF9129
:100C20009F918F912F910F900BBE0F900FBE0F9041
:100C30001F9018951F920F920FB60F9211240BB6AA
:100C40000F922F933F934F935F936F937F938F9365
:100C50009F93AF93BF93EF93FF938BE39FE0DFDD11
:100C6000FF91EF91BF91AF919F918F917F916F9184
:100C70005F914F913F912F910F900BBE0F900FBE40
:100C80000F901F9018958BE39FE062DD21E0892B88
:100C900009F420E0822F089510923E0F10923D0F2C
:100CA00088EE93E0A0E0B0E080933F0F9093400F78
:100CB000A093410FB093420F8EE59AE090933C0FC2
:100CC00080933B0F85ED90E09093480F8093470F02
:100CD00084ED90E090934A0F8093490F80ED90E06F
:100CE00090934C0F80934B0F81ED90E090934E0FBB
:100CF00080934D0F82ED90E09093500F80934F0FB3
:100D000086ED90E09093520F8093510F1092540F04
:100D10001092550F1092560F1092570F08951F9270
:100D20000F920FB60F9211240BB60F922F938F9341
:100D30009F93EF93FF93E091E80FF091E90F80818B
:100D4000E091EE0FF091EF0F82FD12C09081809143
:100D5000F10F8F5F8F732091F20F821751F0E091A6
:100D6000F10FF0E0E852F04F958F8093F10F01C042
:100D70008081FF91EF919F918F912F910F900BBEEA
:100D80000F900FBE0F901F9018951F920F920FB6E5
:100D90000F9211240BB60F922F933F934F935F93B3
:100DA0006F937F938F939F93AF93BF93EF93FF9333
:100DB00088ED9FE034DDFF91EF91BF91AF919F915E
:100DC0008F917F916F915F914F913F912F910F90F4
:100DD0000BBE0F900FBE0F901F90189588ED9FE0EF
:100DE000B7DC21E0892B09F420E0822F08951092CE
:100DF000DB0F1092DA0F88EE93E0A0E0B0E0809372
:100E0000DC0F9093DD0FA093DE0FB093DF0F8EE524
:100E10009AE09093D90F8093D80F85E391E0909357
:100E2000E50F8093E40F84E391E09093E70F8093C4
:100E3000E60F80E391E09093E90F8093E80F81E360
:100E400091E09093EB0F8093EA0F82E391E090930F
:100E5000ED0F8093EC0F86E391E09093EF0F80937A
:100E6000EE0F1092F10F1092F20F1092F30F1092FA
:100E7000F40F0895CF92DF92EF92FF920F931F939A
:100E8000CF93DF937C016A01EB0100E010E00C15C9
:100E90001D0571F06991D701ED91FC910190F081F0
:100EA000E02DC7011995892B19F00F5F1F4FEFCF68
:100EB000C801DF91CF911F910F91FF90EF90DF90CC
:100EC000CF9008956115710581F0DB010D90002030
:100ED000E9F7AD0141505109461B570BDC01ED917B
:100EE000FC910280F381E02D199480E090E0089558
:100EF000EF92FF920F931F93CF93DF938C017B01AF
:100F0000C0E0D0E0F701EC0FFD1F6491662359F0BB
:100F1000F801A081B181ED91FC91C8011995892B4F
:100F200011F02196EFCFCE01DF91CF911F910F915C
:100F3000FF90EF900895DC01ED91FC91DB01149698
:100F40004D915C9115976D917C910280F381E02D1C
:100F50001994B8CFDC01ED91FC910190F081E02D66
:100F600019946AE67AE0AECF0F931F93CF93DF9385
:100F7000EC01BEDF8C01CE01F4DF800F911FDF9109
:100F8000CF911F910F9108950F931F93CF93DF93EC
:100F9000EC01D1DF8C01CE01E4DF800F911FDF91E6
:100FA000CF911F910F9108950F931F93CF93DF93CC
:100FB000EC0188DF8C01CE01D4DF800F911FDF911F
:100FC000CF911F910F9108950F931F93CF93DF93AC
:100FD000EC01C0DF8C01CE01C4DF800F911FDF91D7
:100FE000CF911F910F9108958F929F92AF92BF92D0
:100FF000CF92DF92EF92FF920F931F93CF93DF93E5
:10100000CDB7DEB7A1970FB6F894DEBF0FBECDBF48
:101010007C01C42EE52FCB01D22E19A221E02D1583
:1010200010F02AE0D22E8E010F5D1F4F8D2C912CD7
:10103000A12CB12C6C2D7E2FA50194010E947893D8
:101040008C2DD29E80191124015011098A3014F47C
:10105000805D01C0895CF80180832115310541055F
:10106000510521F0C22EE32FCA01E4CFB801C70118
:1010700029DFA1960FB6F894DEBF0FBECDBFDF917A
:10108000CF911F910F91FF90EF90DF90CF90BF9085
:10109000AF909F908F900895CF92DF92EF92FF9242
:1010A0000F931F93CF93DF93EC016A017B0121150E
:1010B000310579F4E881F9810190F081E02D642F08
:1010C000DF91CF911F910F91FF90EF90DF90CF9024
:1010D00019942A303105D9F477FF18C06DE23ADF50
:1010E0008C0144275527BA014C195D096E097F0907
:1010F0002AE0CE0179DF800F911FDF91CF911F9100
:101100000F91FF90EF90DF90CF9008952AE0B70104
:10111000A601CE01DF91CF911F910F91FF90EF902B
:10112000DF90CF9061CF9A01AB01662757FD6095A4
:10113000762FB2CF0F931F93CF93DF93EC019A01D9
:10114000AB01662757FD6095762FA6DF8C01CE0197
:1011500008DF800F911FDF91CF911F910F910895AC
:101160000F931F93CF93DF93EC0196DF8C01CE0199
:10117000F8DE800F911FDF91CF911F910F9108959D
:101180002115310541F4DC01ED91FC910190F081D4
:10119000E02D642F199428CF0F931F93CF93DF93E3
:1011A000EC019A01462F50E060E070E0E9DF8C012D
:1011B000CE01D7DE800F911FDF91CF911F910F914C
:1011C00008950F931F93CF93DF93EC01D9DF8C0128
:1011D000CE01C7DE800F911FDF91CF911F910F913C
:1011E00008954F925F926F927F928F929F92AF92EB
:1011F000BF92CF92DF92EF92FF920F931F93CF9304
:10120000DF93EC016A017B01B22E9A01AB01C701A9
:10121000B6010E942993882319F06DE67AE026C072
:1012200026013701E89477F82FEF3FEF4FE75FE7AC
:10123000C301B2010E94299381110CC02FEF3FEF2F
:101240004FE75FE7C301B201ACD618161CF461E7A3
:101250007AE00CC02FEF3FEF4FE75FE4C701B60124
:101260000E9476911816A4F465E77AE0CE01DF912A
:10127000CF911F910F91FF90EF90DF90CF90BF9093
:10128000AF909F908F907F906F905F904F901ACE0D
:101290002FEF3FEF4FE75FECC701B60182D687FD26
:1012A000E3CF20E030E0A901C701B6017AD687FF7D
:1012B00009C06DE2CE014EDE8C01F7FAF094F7F82A
:1012C000F09402C000E010E0A12C60E070E080E04B
:1012D0009FE3AB1439F020E030E040E251E465D602
:1012E000A394F7CF9B01AC01C701B60194D56B0164
:1012F0007C01F9D62B013C0122D79B01AC01C7012F
:10130000B60188D56B017C012AE0B301A201CE01B0
:101310006BDE080F191FBB2031F06DE077E0CE01C6
:10132000D1DD080F191F7B2C772021F120E030E060
:1013300040E251E4C701B6010E9435926B017C0185
:10134000CDD64B01AA2497FCA094BA2C2AE030E019
:10135000B501A401CE01A0DE080F191FC501B4011B
:10136000F0D69B01AC01C701B60154D56B017C01DD
:101370007A94DACFC801DF91CF911F910F91FF903E
:10138000EF90DF90CF90BF90AF909F908F907F9025
:101390006F905F904F90089524CF0F931F93CF933A
:1013A000DF93EC011EDF8C01CE01DBDD800F911F8E
:1013B000DF91CF911F910F9108950F931F93CF93BA
:1013C000DF93EC010E94A881688779878A879B87D1
:1013D000E881F9810680F781E02DCE01199597FF0C
:1013E00015C00E94A881088519852A853B85601B48
:1013F000710B820B930B0C811D812E813F81601735
:1014000071078207930720F38FEF9FEFDF91CF9152
:101410001F910F910895FC01448355836683778360
:101420000895CF92DF92EF92FF920F931F93CF9385
:10143000DF937C016A01EB0100E010E00C151D0553
:1014400041F0C701BADF97FD04C089930F5F1F4FBA
:10145000F5CFC801DF91CF911F910F91FF90EF90D1
:10146000DF90CF9008954F925F926F927F928F920C
:101470009F92AF92BF92CF92DF92EF92FF920F9323
:101480001F93CF93DF934C01EB0186E0849F800193
:10149000859F100D1124060F171FFB01E017F107A0
:1014A00008F582819381892B19F13696F7CF408117
:1014B000518164817581DA01A60FB71F2C91332702
:1014C00027FD30958217930709F56F5F7F4F75836E
:1014D0006483228133816217730751F03696E017D7
:1014E000F10728F3C40169DF97FD46C0FE01F7CF7D
:1014F000EC1BFD0BF595E7952BEA3AEAE29FC0015C
:10150000E39F900DF29F900D112438C06115710575
:1015100029F3A480B58095012150310935832483B6
:10152000DA01A20FB31FAC91BB27A7FDB0958A17B4
:101530009B07F9F421153105C9F06A017B01E21A14
:10154000F30AE40EF51E412C512CD6016D906D016D
:10155000D7017D907D01671006C0BFEF4B1A5B0A73
:101560004216530690F34216530699F6B582A482AA
:10157000B5CF232B71F6B2CF8FEF9FEFDF91CF91D5
:101580001F910F91FF90EF90DF90CF90BF90AF90A1
:101590009F908F907F906F905F904F900895CF9322
:1015A000DF9300D000D0CDB7DEB7FE01319626E044
:1015B000DF011D922A95E9F77A8369835C834B8367
:1015C00041E050E0BF014FDF21E0892B09F020E02E
:1015D000822F26960FB6F894DEBF0FBECDBFDF91E7
:1015E000CF910895DCCFFC01808191810C94CE9441
:1015F000CF93DF93EC0188819981009711F00E94CD
:10160000CE94198218821D821C821B821A82DF915D
:10161000CF9108950F931F93CF93DF93EC018B012C
:101620006F5F7F4F888199810E945D95009731F0AF
:10163000998388831B830A8381E001C080E0DF9166
:10164000CF911F910F910895CF93DF93EC01888183
:101650009981892B29F08A819B818617970758F4F5
:10166000CE01D8DF882341F08C819D81892B19F42C
:10167000E881F981108281E0DF91CF910895EF92A6
:10168000FF920F931F93CF93DF93EC017B018A01AD
:10169000BA01DADF811103C0CE01AADF07C01D83C2
:1016A0000C83B701888199810E948F96CE01DF91CA
:1016B000CF911F910F91FF90EF900895FC0111823F
:1016C000108213821282158214826115710551F005
:1016D000FB0101900020E9F7AF0141505109461B81
:1016E000570BCDCF0895EF92FF920F931F93CF9397
:1016F000DF93EC017B018A01BA01A6DF811103C0EF
:10170000CE0176DF07C01D830C83B70188819981E4
:101710000E947696CE01DF91CF911F910F91FF909D
:10172000EF9008950F931F93CF93DF938C01EB01FC
:10173000FC0180819181009799F0428153812C8135
:101740003D814217530750F0688179810E948F963E
:101750008C819D81F8019583848313C00E94CE946F
:1017600088819981F801918380838A819B81938309
:1017700082838C819D8195838483198218821B8248
:101780001A821D821C82DF91CF911F910F910895C3
:10179000CF93DF93EC01FB018617970751F060812F
:1017A00071816115710521F04481558168DF01C0A7
:1017B0001FDFCE01DF91CF910895FC0111821082CD
:1017C0001382128215821482E3CFCF93DF93EC0150
:1017D0008617970709F0A6DFCE01DF91CF91089514
:1017E000CF93DF93EC018617970709F09BDFCE01BB
:1017F000DF91CF910895CF93DF93EC0161157105CF
:1018000059F0FB0101900020E9F7AF014150510967
:10181000461B570B34DF01C0EBDECE01DF91CF91C9
:101820000895CF93DF931F921F92CDB7DEB7FC01CF
:1018300011821082138212821582148269831A82A5
:10184000BE016F5F7F4FD7DF0F900F90DF91CF9179
:1018500008950F931F93CF93DF93CDB7DEB76297B1
:101860000FB6F894DEBF0FBECDBF8C01CB01F801DF
:1018700011821082138212821582148250E0BE01FE
:101880006F5F7F4F0E94CD96BE016F5F7F4FC80193
:10189000B2DF62960FB6F894DEBF0FBECDBFDF9108
:1018A000CF911F910F9108950F931F93CF93DF93C3
:1018B000CDB7DEB7A2970FB6F894DEBF0FBECDBF8F
:1018C0008C01CB01BA01F8011182108213821282BD
:1018D0001582148230E0AE014F5F5F4F0E94E196A7
:1018E000BE016F5F7F4FC80186DFA2960FB6F894E6
:1018F000DEBF0FBECDBFDF91CF911F910F91089535
:10190000EF92FF920F931F93CF93DF93CDB7DEB784
:10191000A1970FB6F894DEBF0FBECDBF7C01CB01FF
:10192000BA01F70111821082138212821582148289
:1019300042E0420F8E010F5F1F4F78D7BC01C701F5
:101940005ADFA1960FB6F894DEBF0FBECDBFDF9170
:10195000CF911F910F91FF90EF900895EF92FF921A
:101960000F931F93CF93DF93CDB7DEB7A1970FB639
:10197000F894DEBF0FBECDBF7C01CB01BA01F701E9
:1019800011821082138212821582148242E0420F69
:101990008E010F5F1F4F4AD7BC01C7012CDFA196F4
:1019A0000FB6F894DEBF0FBECDBFDF91CF911F9170
:1019B0000F91FF90EF9008950F931F93CF93DF93B4
:1019C0001F921F92CDB7DEB78C016115710559F0DA
:1019D000CB0169837A830E947D96AC0169817A810B
:1019E000C80181DE01C004DEC8010F900F90DF91B5
:1019F000CF911F910F910895FC01118210821382E3
:101A0000128215821482D8CFEF92FF920F931F9308
:101A1000CF93DF93EC017B010C811D816115710572
:101A200011F480E015C04115510589F0040F151F10
:101A3000B8010ADE8823A9F3288139818C819D8130
:101A4000B701820F931F0E948F961D830C8381E044
:101A5000DF91CF911F910F91FF90EF900895FB01BF
:101A60004481558160817181CFCF6115710551F03D
:101A7000FB0101900020E9F7AF0141505109461BDD
:101A8000570BC2CF80E00895CF93DF931F921F9230
:101A9000CDB7DEB769831A8241E050E0BE016F5FC7
:101AA0007F4FB2DF0F900F90DF91CF910895CF93CA
:101AB000DF93EC01FB014481558160817181A4DFDA
:101AC000811102C0CE0194DDCE01DF91CF91089546
:101AD000CF93DF93EC016115710561F0FB0101907B
:101AE0000020E9F7AF0141505109461B570B8CDF2D
:101AF000811102C0CE017CDDCE01DF91CF9108952E
:101B0000FA01DB0114964D915C911597DC01149656
:101B10002D913C911597241B350B2E173F0788F00C
:101B20008D919C91009769F0DB016D917C9161151D
:101B3000710539F08E0F9F1F0E94969621E0892B28
:101B400009F020E0822F0895FC0144815581FB01BA
:101B5000248135814217530718F040E050E0D0CF80
:101B600080E00895FC01248135816217730748F4F1
:101B700080819181009729F0FC01E60FF71F808199
:101B8000089580E00895EECF0F931F93CF93DF93D6
:101B9000EB0141155105E9F02097D9F0FC01648172
:101BA000758126173707A0F4621B730B8A01015059
:101BB00011096017710708F48B01FC0160817181C4
:101BC000620F731FA801CE010E94A496C00FD11FFF
:101BD0001882DF91CF911F910F910895AF92BF921C
:101BE000CF92DF92EF92FF920F931F93CF93DF93E9
:101BF0007B01EA01FB01448155814115510569F1E1
:101C0000FC01248135812115310539F1241735076F
